:100000000C943E280C946F280C946F280C946F2845
:100010000C946F280C946F280C946F280C946F2804
:100020000C946F280C946F280C946F280C946F28F4
:100030000C946F280C946F280C946F280C946F28E4
:100040000C946F280C947C7F0C946F280C946F2870
:100050000C946F280C946F280C9453BF0C948AF75F
:100060000C946F280C949E4B0C946F280C946F2862
:100070000C946F280C946F280C946F280C946F28A4
:100080000D94A00C0C946F280C946F280C946F287E
:100090000C946F280C946F280C946F280C946F2884
:1000A0000C946F280C946F280D94730C0C946F288B
:1000B0000C946F280C946F280C946F280D94460CA8
:1000C0000C946F280C946F280C946F280C946F2854
:1000D0000C946F280C946F280C946F280C946F2844
:1000E0000C946F28F3C554C48AC42FC68AC48AC42A
:1000F0008AC48AC48AC48AC48AC48AC48AC48AC490
:100100008AC48AC48AC48AC48AC48AC48AC48AC47F
:100110008AC48AC48AC48AC48AC48AC48AC48AC46F
:1001200029C68AC48AC48AC48AC48AC48AC48AC4BE
:100130008AC402C68AC48AC48AC48AC48AC48AC4D5
:100140008AC48AC48AC48AC446C687C407F60AF623
:10015000F9F5FDF503F641F60EF612F618F61CF663
:1001600020F626F62AF62EF641F634F638F63CF658
:10017000A6F6ABF6B0F6BAF6C4F63DF7CEF6D6F66E
:10018000DEF6E8F6F2F6FCF60BF715F73DF71FF78B
:1001900029F733F7084AD73B3BCE016E84BCBFFD3D
:1001A000C12F3D6C74319ABD56833DDA3D00C77F47
:1001B00011BED9E4BB4C3E916BAAAABE00000080E0
:1001C0003F05A84CCDB2D44EB93836A9020C50B96F
:1001D000918688083CA6AAAA2ABE000000803F009B
:1001E0000D943D120D94AB020D94F6030D945D0138
:1001F0000D94311A0D9412014E414E494E495459F5
:10020000494E46CDCCCC3D0AD7233C17B7D13877E1
:10021000CC2B329595E6241FB14F0A0000204100F7
:1002200000C84200401C4620BCBE4CCA1B0E5AAE41
:10023000C59D7400407A10F35A00A0724E18090050
:1002400010A5D4E80000E87648170000E40B54023B
:100250000000CA9A3B000000E1F505000080969876
:1002600000000040420F000000A0860100000010C6
:100270002700000000E80300000000640000000008
:10028000000A00000000000100000000002C76D8E9
:1002900088DC674F0823DFC1DFAE59E1B1B796E5CF
:1002A000E3E453C63AE651997696E8E6C28426EB33
:1002B000898C9B62ED407C6FFCEFBC9C9F40F2BA46
:1002C000A56FA5F490055A2AF75C936B6CF9676DDE
:1002D000C11BFCE0E40D47FEF520E6B500D0ED9033
:1002E0002E0300943577050080841E080000204E00
:1002F0000A000000C80C333333330F986E12831199
:1003000041EF8D2114893BE65516CFFEE6DB18D16F
:10031000844B381BF77C1D901DA4BBE42420328441
:10032000725E228100C9F124ECA1E53D27434F4DC7
:100330004D554E49434154494F4E00445259525530
:100340004E004552524F525300494E464F004543CE
:10035000484F0047322F473320626164207061723A
:10036000616D65746572730A00536C6565702E2E3D
:100370002E005A2070726F6265206F75742E206295
:1003800065640A005A2070726F6265206F75742E62
:100390002062656400473238205A20466F726269D5
:1003A0006464656E0A00473238205A20466F7262D4
:1003B000696464656E00205A3A200020593A200092
:1003C00042656420583A20004D65736820706F695B
:1003D0006E742063616E6E6F742062652072657347
:1003E0006F6C7665640A0043522D313020563320FD
:1003F00072656164792E00526573756D696E672050
:100400007072696E7400436C69636B20746F207244
:100410006573756D652E2E2E004E6F206D6F76659F
:100420002E00456E642066696C65206C6973740AE1
:1004300000426567696E2066696C65206C6973743B
:100440000A005446207072696E74696E6720627982
:10045000746520004E6F74205446207072696E746B
:10046000696E670A002569730025696D2025697327
:10047000002569682025696D202569730025696458
:10048000202569682025696D202569730025697913
:1004900020256964202569682025696D20256973F8
:1004A000005072696E742074696D653A2000507254
:1004B0006F7465637465642050696E0A00457874D2
:1004C00072756465722025730043522D31302056B9
:1004D000332072656164792E004E03490342033B69
:1004E000032D036F66660044454255473A004B4969
:1004F0004C4C45442E20004D3131332053006F6B5E
:100500000043522D3130205633204F66662E002F87
:100510002F20004D31343520533C696E6465783EA0
:10052000206F7574206F662072616E6765202830B9
:100530002D31290A0053657474696E672054726105
:1005400076656C20416363656C65726174696F6E7A
:100550003A200053657474696E6720526574726145
:10056000637420416363656C65726174696F6E3A90
:10057000200053657474696E67205072696E742030
:10058000416363656C65726174696F6E3A200053F4
:10059000657474696E67205072696E7420616E6450
:1005A0002054726176656C20416363656C6572618D
:1005B00074696F6E3A2000000136372603FF3C3D18
:1005C000380EFF2E303E13FFFF0C0809FFFFFF1A05
:1005D0001C18FFFF08440AFF43FFFFFFFFFFFF2037
:1005E0006F7574206F662072616E67650A005365CF
:1005F00072766F20003A200020536572766F2000DB
:1006000020643A0020693A0020703A0043290A0029
:1006100061626C656420286D696E2074656D702060
:1006200000436F6C64206578747275646573206133
:10063000726520003A20007A5F6D696E3A20202DA5
:100640003230207A5F6D61783A20203230005A20B3
:100650004F666673657420004E6F2063617365207A
:100660006C696768740A004163746976652045782F
:100670007472756465723A2000556E6B6E6F776E9A
:1006800020636F6D6D616E643A2022004B494C4CC3
:1006900045442E200053544F505045442E200050C6
:1006A00072696E7465722073746F70706564206413
:1006B000756520746F206572726F72732E204669A3
:1006C0007820746865206572726F7220616E642094
:1006D000757365204D39393920746F2072657374D4
:1006E0006172742E202854656D7065726174757224
:1006F000652069732072657365742E2053657420BC
:1007000069742061667465722072657374617274B5
:10071000696E67290A004E6F204C696E65204E7520
:100720006D626572207769746820636865636B73B6
:10073000756D2C204C617374204C696E653A2000F5
:100740004E6F20436865636B73756D2077697468BD
:10075000206C696E65206E756D6265722C204C612F
:100760007374204C696E653A2000636865636B732F
:10077000756D206D69736D617463682C204C6173B5
:1007800074204C696E653A20004C696E65204E7588
:100790006D626572206973206E6F74204C61737492
:1007A000204C696E65204E756D6265722B312C2070
:1007B0004C617374204C696E653A20004D313130C4
:1007C000004D3331004D383420582059205A2045EF
:1007D0000054462072656164206572726F720A006F
:1007E000446F6E65207072696E74696E6720666909
:1007F0006C650A0020496E76616C696420657874C6
:1008000072756465722000000000000000000000A6
:1008100000000000009B4300009B430000CD4353B9
:10082000544F505045442E20005072696E746572CA
:100830002073746F707065642064756520746F2018
:100840006572726F72732E20466978207468652015
:100850006572726F7220616E6420757365204D3908
:10086000393920746F20726573746172742E202878
:1008700054656D706572617475726520697320725C
:10088000657365742E2053657420697420616674E5
:1008900065722072657374617274696E67290A00EB
:1008A00053544F502063616C6C65642062656361D2
:1008B000757365206F6620424C546F7563682065C0
:1008C00072726F72202D207265737461727420775A
:1008D000697468204D3939390A0047302046333071
:1008E0003030205831353020593135300042696C74
:1008F000696E656172204C6576656C696E6720472C
:100900007269643A0A0020706F736974696F6E20AF
:100910006F7574206F662072616E67652E0A003FE6
:1009200050726F62652000486F6D652025732573D6
:100930002573206669727374002066697273740A85
:10094000005A0059005800486F6D65200052756EBE
:100950006E696E6720696E204452592D52554E20A3
:100960006D6F64650A00473239204175746F20420B
:100970006564204C6576656C696E670A00284229BB
:1009800061636B00284629726F6E740028522969D2
:1009900067687400284C29656674003F28562965ED
:1009A00072626F7365206C6576656C20697320696F
:1009B0006D706C61757369626C652028302D342907
:1009C0002E0A00426164205A2076616C75650A0027
:1009D0004E6F2062696C696E65617220677269642E
:1009E0000A0046696C652064656C657465643A004C
:1009F00044656C6574696F6E206661696C65642C12
:100A00002046696C653A20006F70656E20666169EA
:100A10006C65642C2046696C653A2000202F00200C
:100A200042403A0020403A0048656174696E672090
:100A3000646F6E652E0020573A00457874727564B5
:100A400065722025730043522D31302056332072B9
:100A5000656164792E0042656420646F6E652E00C6
:100A600020573A004265642048656174696E672EBC
:100A700000205A3A0020593A0020436F756E7420C6
:100A8000583A0020453A00205A3A0020593A005876
:100A90003A004361703A454D455247454E43595FD0
:100AA0005041525345523A300A004361703A434133
:100AB00053455F4C494748545F4252494748544E5A
:100AC0004553533A300A004361703A544F47474CFC
:100AD000455F4C49474854533A300A004361703AE5
:100AE000534F4654574152455F504F5745523A3045
:100AF0000A004361703A4C4556454C494E475F44A5
:100B00004154413A310A004361703A5A5F50524FA2
:100B100042453A310A004361703A4155544F4C45C1
:100B200056454C3A310A004361703A5052494E548E
:100B30005F4A4F423A310A004361703A50524F4780
:100B4000524553533A300A004361703A4155544F6D
:100B50005245504F52545F54454D503A310A00436C
:100B600061703A454550524F4D3A310A004649525C
:100B70004D574152455F4E414D453A4D61726C694A
:100B80006E20437265616C69747920334420534F41
:100B9000555243455F434F44455F55524C3A687444
:100BA0007470733A2F2F6769746875622E636F6D66
:100BB0002F4D61726C696E4669726D776172652F37
:100BC0004D61726C696E2050524F544F434F4C5FD1
:100BD00056455253494F4E3A312E30204D414348ED
:100BE000494E455F545950453A43522D31302056B5
:100BF000332045585452554445525F434F554E5447
:100C00003A3120555549443A63656465326132662C
:100C10002D343161322D343734382D396231322D53
:100C20006335356336326633363766660A00205AD6
:100C300000205900580020204D61783A2000205AA9
:100C400000205900580020204D696E3A20004F6E58
:100C500020004F666600536F667420656E6473747F
:100C60006F70733A200020643A0020693A002070C7
:100C70003A004B64200023646566696E6520204459
:100C8000454641554C545F004B692000236465661E
:100C9000696E65202044454641554C545F004B70B9
:100CA000200023646566696E6520204445464155F1
:100CB0004C545F00504944204175746F74756E65E3
:100CC0002066696E697368656421205075742074AC
:100CD0006865206C617374204B702C204B69206117
:100CE0006E64204B6420636F6E7374616E74732046
:100CF00066726F6D2062656C6F7720696E746F200D
:100D0000436F6E66696775726174696F6E2E680AEB
:100D100000504944204175746F74756E652066619A
:100D2000696C6564212074696D656F75740A005083
:100D30004944204175746F74756E65206661696CF5
:100D40006564212054656D706572617475726520EB
:100D5000746F6F20686967680A00204B643A20004E
:100D6000204B693A2000204B703A20000A20436C47
:100D7000617373696320504944200A002054753A16
:100D80002000204B753A2000206D61783A20002029
:100D90006D696E3A200020643A2000206269617318
:100DA0003A20004F66660A0046616465204865691E
:100DB0006768742000426564204C6576656C696ED6
:100DC0006720004661696C656420746F20656E6100
:100DD000626C6520426564204C6576656C696E675F
:100DE0000A004D65736820706F696E742063616ED0
:100DF0006E6F74206265207265736F6C7665640A2D
:100E0000004D34323120696E636F727265637420F5
:100E1000706172616D657465722075736167650AD2
:100E2000004F666673657473206170706C696564E9
:100E3000004572723A20546F6F206661722100542F
:100E40006F6F206661722066726F6D2072656665D5
:100E500072656E636520706F696E740A00627573E7
:100E6000793A2070617573656420666F7220696ECF
:100E70007075740A00627573793A207061757365D4
:100E80006420666F7220757365720A0062757379EB
:100E90003A2070726F63657373696E670A004B491D
:100EA0004C4C45442E20004B494C4C2063617573DB
:100EB0006564206279204B494C4C20627574746FD4
:100EC0006E2F70696E0A004B494C4C45442E200031
:100ED0004B494C4C206361757365642062792074C2
:100EE0006F6F206D75636820696E616374697665E4
:100EF0002074696D65202D2063757272656E742093
:100F0000636F6D6D616E643A2000506C656173654E
:100F1000207265736574005052494E544552204802
:100F2000414C544544005072696E7465722068618A
:100F30006C7465642E206B696C6C28292063616C6D
:100F40006C6564210A0062696E004D3131372049B9
:100F50004E56414C494420444154412E00473932B9
:100F6000205A2573204525730062696E0000000039
:100F7000000000000000000000000048420000489F
:100F80004200008040000000005761726E696E6789
:100F90003A20486F6D696E672042756D7020446914
:100FA0007669736F72203C20310A0002020400004F
:100FB000A0400000A0400000004000009B43000053
:100FC0009B430000CD43FFFFFF20204D38353120EB
:100FD0005A005A2D50726F6265204F6666736574B1
:100FE00020286D6D293A0A00204400204900202065
:100FF0004D33303420500020440020490020204D43
:101000003330312050005049442073657474696E48
:1010100067733A0A00204600204200204800202042
:101020004D3134352053004D6174657269616C2017
:1010300068656174757020706172616D6574657248
:10104000733A0A00205A0020204D343230205300D9
:101050004175746F20426564204C6576656C696EDD
:10106000673A0A00205A0020590020204D323036BD
:10107000205800486F6D65206F66667365743A0A84
:1010800000204500205A002059002058002042002E
:1010900020540020204D32303520530041647661C9
:1010A0006E6365643A20533C6D696E5F6665656486
:1010B000726174653E20543C6D696E5F7472617636
:1010C000656C5F66656564726174653E20423C6D67
:1010D000696E5F7365676D656E745F74696D655F7A
:1010E0006D733E20583C6D61785F78795F6A6572F8
:1010F0006B3E205A3C6D61785F7A5F6A65726B3E29
:1011000020453C6D61785F655F6A65726B3E0A00E1
:1011100020540020520020204D3230342050004115
:101120006363656C65726174696F6E2028756E69A2
:1011300074732F7332293A20503C7072696E745F59
:10114000616363656C3E20523C72657472616374C6
:101150005F616363656C3E20543C74726176656CBC
:101160005F616363656C3E0A00204500205A0020E1
:10117000590020204D3230312058004D6178696D82
:10118000756D20416363656C65726174696F6E2073
:1011900028756E6974732F7332293A0A002045004E
:1011A000205A0020590020204D3230332058004D65
:1011B0006178696D756D20666565647261746573CB
:1011C0002028756E6974732F73293A0A0020450030
:1011D000205A0020590020204D39322058005374E5
:1011E0006570732070657220756E69743A0A00200C
:1011F000204D3230302044300A0020204D32303033
:101200002044002044697361626C65640A00466989
:101210006C616D656E742073657474696E67733A82
:101220000020204D3134392043203B20556E697415
:101230007320696E2043656C736975730A00202002
:10124000473231202020203B20556E69747320697D
:101250006E206D6D0A007A5F6D696E3A2000795FCD
:101260006D696E3A2000785F6D696E3A20005265B4
:10127000706F7274696E6720656E6473746F70202E
:101280007374617475730A004D36303020486F7482
:10129000656E6420746F6F20636F6C6420746F20C0
:1012A0006368616E67652066696C616D656E740A5E
:1012B000000000000000000000000000000000002E
:1012C000000000000000000000000000000000001E
:1012D000000000000000000000000000000000000E
:1012E00000000000000000000000000000000000FE
:1012F00000000000000000000000000000000000EE
:1013000000000000000000000000000000000000DD
:1013100000000000000000000000000000000000CD
:1013200000000000000000000000000000000000BD
:101330000000000080000008000000000000000025
:101340000000000080000008000000000000000015
:101350000000209E9DE773C8000000000000000010
:101360000000359291249248000000000000000027
:101370000000151E912493C800000000000000002A
:1013800000001B10912492000000000000000000EB
:1013900000000A1E9DE493C8000000000000000049
:1013A000000000000000000000000000000000003D
:1013B000000000000000000000000000000000002D
:1013C000000000000000000000000000000000001D
:1013D000000000000000000000000000000000000D
:1013E00000000000000000000000000000000000FD
:1013F00000000000000000000000000000000000ED
:1014000000000000000000000000000000000000DC
:1014100000000000000000000000000000000000CC
:1014200000000000000000000000000000000000BC
:1014300000000000000000000000000000000000AC
:10144000000000000000000000000000000000009C
:10145000000000000000000000000000000000008C
:10146000000000000000000000000000000000007C
:10147000000000000000000000000000000000006C
:10148000000000000000000000000000000000005C
:101490000000000FFDFFC0FF80C0600FFFF80F00CD
:1014A0000000001FFDFFE3FF80C0600FFFF81E007B
:1014B0000000003C0180678001C0600E0E1E3C00F1
:1014C000000000700180670001E0600E0E0F7800E0
:1014D0000000006001806E0003E0600E0E07F00067
:1014E0000000006001BFEFFF8370600E0E03E0009C
:1014F00000000060019FCFFF8738600E0E01C00022
:1015000000000060018E0E000718600E0E01C00082
:1015100000000070018707000E1E600E0E01C00063
:101520000000003C018387800C0E600E0E01C0009D
:101530000000001FFD81C3FF9CFE7FEE0E01C00076
:101540000000000FFD80E0FFBDFF7FEE0E01C00038
:10155000000000000000000000000000000000008B
:10156000000000000000000000000000000000007B
:10157000000000000000000000000000000000006B
:10158000000000000000000000000000000000005B
:10159000000000000000000000000000000000004B
:1015A000000000000000000000000000000000003B
:1015B000000000000000000000000000000000002B
:1015C000000000000000000000000000000000001B
:1015D000000000000000000000000000000000000B
:1015E00000000000000000000000000000000000FB
:1015F00000000000000000000000000000000000EB
:1016000000000000000000000000000000000000DA
:1016100000000000000000000000000000000000CA
:1016200000000000000000000000000000000000BA
:1016300000000000000000000000000000000000AA
:10164000000000000000000000000000000000009A
:10165000000000000000000000000000000000008A
:10166000000000000000000000000000000000007A
:10167000000000000000000000000000000000006A
:10168000000000000000000000000000000000005A
:10169000000000000000000000000000000000004A
:1016A000000000000000000000000000000000003A
:1016B0000025753A2530327500253032753A2530CF
:1016C00032750025756420253032753A2530327523
:1016D000005A0059005800092000000000000000D6
:1016E000000000000000003FFFF0000000000000CC
:1016F0000000000000000038007000000000000042
:101700000000000000000030FC300000000000007D
:101710000000000000000020FC100000000000009D
:101720000000000000000020781000000000000011
:10173000000000000000002030107BC08C22600000
:10174000000000000000002C00D08A219222901F8F
:10175000E00000104100002E31D082209222103F84
:10176000F00000082080002F7BD083DE9222603FB3
:10177000F00000082080002F7BD082809222103F52
:10178000F00000104100002E31D08A409214901FCA
:10179000E00000208200002C00D07221CC08601FE5
:1017A000E000004104000020301000000000003F75
:1017B000F000004104000020781000000000003F0D
:1017C000F000002082000020FC1000000000003F1C
:1017D000F000001041000030FC3000000000000F5D
:1017E000C00000000000003800700000000000078A
:1017F000800000FFFFC0003FFFF00000000000037A
:10180000000000FFFFC0000000000000000000001A
:10181000000000000000003FFFF00000000000009A
:101820000000000000000038007000000000000010
:1018300000000000000000338730000000000000BE
:10184000000000000000002787900000000000005A
:10185000000000000000002F87D000000000000002
:10186000000000000000002F87D07BC08C226000A9
:10187000000000000000002F03D08A219222901F58
:10188000E000000820800020301082209222103FCB
:10189000F000000410400020781083DE9222603FA8
:1018A000F000000410400020781082809222103F47
:1018B000F00000082080002030108A409214901F11
:1018C000E00000104100002F03D07221CC08601FFF
:1018D000E00000208200002F87D000000000003FC1
:1018E000F00000208200002F87D000000000003FA1
:1018F000F000001041000027879000000000003F2A
:10190000F000000820800033873000000000000F46
:10191000C000000000000038007000000000000758
:10192000800000FFFFC0003FFFF000000000000348
:10193000000000FFFFC00000000024F4D43050C3BA
:101940008E20C2A24017828B7011127A910D816C89
:10195000D90AA861E108C7586607615143061E4BC2
:101960005D05C145A7041A411104093D9803713969
:1019700031034036DB0265339102D4305402802EAD
:101980001D02632CEE01752AC501B028A0011027A5
:1019900081018F2564012B244B01E0223401AC210D
:1019A0001F018D200D01801FFC00841EED00971D7E
:1019B000DF00B81CD200E61BC600201BBC00641A66
:1019C000B200B219A8000A19A0006A189900D1172C
:1019D000910040178B00B516840031167E00B315B8
:1019E00079003A157300C7146F0058146A00EE139B
:1019F00066008813630025135E00C7125B006C123B
:101A0000570015125400C111510070114F002111DF
:101A10004B00D61049008D104700461044000210BC
:101A20004200C00F4000800F3E00420F3C00060FF6
:101A30003B00CB0E3800930E37005C0E3500270EAE
:101A40003400F30D3200C10D3100900D3000600DF7
:101A50002E00320D2D00050D2C00D90C2B00AE0CE4
:101A60002900850C29005C0C2700350C27000E0C82
:101A70002600E80B2400C40B2400A00B23007D0BE0
:101A800023005A0B2100390B2100180B2000F80A03
:101A90001F00D90A1E00BB0A1E009D0A1D00800AF5
:101AA0001D00630A1C00470A1B002C0A1B00110AB8
:101AB0001A00F7091A00DD091900C4091900AB0959
:101AC0001900920917007B091800630917004C09D7
:101AD000160036091600200916000A091500F50837
:101AE0001500E0081400CC081400B8081400A4087D
:101AF0001400900813007D0812006B0813005808AA
:101B000012004608120034081100230811001208C0
:101B1000110001081100F0071000E0071000D007C5
:101B20001000C0071000B0070F00A10710009107B8
:101B30000E0083070F0074070F0065070E0057079C
:101B40000E0049070E003B070D002E070E00200770
:101B50000D0013070D0006070D00F9060C00ED0639
:101B60000D00E0060C00D4060C00C8060C00BC06F4
:101B70000C00B0060C00A4060B0099060C008D06A4
:101B80000B0082060B0077060B006C060B0061064B
:101B90000A0057060B004C060A0042060A003806E7
:101BA0000A002E060A0024060A001A060A00100679
:101BB000090007060A00FD050900F4050900EB0508
:101BC0000900E2050900D9050900D0050900C7058B
:101BD0000900BE050900B5050800AD050800A5050A
:101BE00009009C050800940508008C050800840580
:101BF00008007C050800740508006C0507006505F1
:101C000008005D050700560508004E05070047055A
:101C100007004005080038050700310507002A05C0
:101C20000700230507001C050600160507000F0521
:101C300007000805060002050700FB040600F5047E
:101C40000700EE040600E8040600E2040700DB04D7
:101C50000600D5040600CF040600C9040600C3042C
:101C60000600BD040600B7040600B1040500AC047C
:101C70000600A6040600A00405009B0406009504C7
:101C80000500900406008A04050085040500800410
:101C900006007A04050075040500700405006B0455
:101CA000050066040500610405005C040500570496
:101CB0000500520405004D040500480405004304D6
:101CC00005003E0404003A04050035040500300414
:101CD00004002C04050027040400230405001E044E
:101CE00004001A04040016040500110404000D0485
:101CF0000400090405000404040000040400FC03BB
:101D00000400F8030400F4030400F0030400EC03EF
:101D10000400E8030400E4030400E0030400DC031F
:101D20000400D8030400D4030400D0030400CC034F
:101D30000400C8030300C503030024F404D9201BD6
:101D4000C40C5C0E9804C4095F0265077101F405B8
:101D5000F900FB04B30048048700C103690058037D
:101D6000550003034500BE023A00840231005302CD
:101D70002A002902250004022000E4011C00C801F9
:101D80001900AF01170098011400840113007101BC
:101D900010006101100051010E0043010D003601D9
:101DA0000B002B010B0020010B00150109000C0199
:101DB000090003010800FB000800F3000800EB0025
:101DC0000700E4000600DE000600D8000600D2008E
:101DD0000600CC000500C7000500C2000500BD00DC
:101DE0000400B9000400B5000400B1000400AD0017
:101DF0000400A9000400A5000300A20003009F0046
:101E000004009B000300980003009500020093006B
:101E10000300900003008D0002008B000300880087
:101E200002008600020084000300810002007F009F
:101E300002007D0002007B000200790002007700B2
:101E400001007600020074000200720001007100BF
:101E500002006F0002006D0001006C0002006A00C9
:101E600001006900020067000100660001006500D2
:101E700001006400020062000100610001006000D6
:101E800001005F0002005D0001005C0001005B00DA
:101E900001005A00010059000100580001005700DC
:101EA00001005600010055000100540001005300DC
:101EB00000005300010052000100510001005000D9
:101EC00001004F0001004E0000004E0001004D00D7
:101ED00001004C0001004B0000004B0001004A00D3
:101EE00001004900010048000000480001004700CF
:101EF00001004600000046000100450000004500CA
:101F000001004400010043000000430001004200C2
:101F100000004200010041000000410001004000BB
:101F200001003F0000003F0001003E0000003E00B5
:101F300001003D0000003D0001003C0000003C00AD
:101F400000003C0001003B0000003B0001003A00A3
:101F500000003A000100390000003900010038009B
:101F60000000380000003800010037000000370092
:101F70000100360000003600000036000100350088
:101F8000000035000000350001003400000034007E
:101F90000000340001003300000033000000330073
:101FA0000100320000003200000032000100310068
:101FB000000031000000310001003000000030005E
:101FC0000000300001002F0000002F0000002F0053
:101FD00000002F0001002E0000002E0000002E0047
:101FE00001002D0000002D0000002D0000002D003C
:101FF00001002C0000002C0000002C0000002C0030
:1020000001002B0000002B0000002B0000002B0023
:1020100001002A0000002A0000002A0000002A0017
:10202000010029000000290000002900000029000B
:1020300000002900010028000000280000002800FE
:1020400000002800000028000100270000002700F1
:1020500000002700000027000000270001002600E4
:1020600000002600000026000000260000002600D8
:1020700001002500000025000000250000002500CB
:1020800000002500000025000100240000002400BD
:1020900000002400000024000000240001002300B0
:1020A00000002300000023000000230000002300A4
:1020B0000000230000002300010022000000220095
:1020C0000000220000002200000022000000220088
:1020D000010021000000210000002100000021007B
:1020E000000021000000210000002100010020006C
:1020F0000000200000002000000020000000200060
:1021000000002000000020000000200001001F004F
:1021100000001F0000001F0000001F0000001F0043
:1021200000001F0000001F0001001E0000001E0034
:1021300000001E0000001E0000004D383420582012
:1021400059205A2045006265640A002C2073797377
:1021500074656D2073746F707065642120486561CB
:102160007465725F49443A200048656174696E671E
:10217000206661696C65640048656174696E6720FA
:102180006661696C65640048656174696E672066A4
:1021900061696C65640048656174696E6720666199
:1021A000696C65640057726974696E6720746F208A
:1021B00066696C653A20006F70656E206661696CB7
:1021C00065642C2046696C653A20006F70656E204E
:1021D0006661696C65642C2046696C653A2000462E
:1021E000696C652073656C65637465640A002053CF
:1021F000697A653A200046696C65206F70656E6586
:10220000643A20006F70656E206661696C65642CAD
:102210002046696C653A20002066696C653A2000AA
:102220004E6F7720002220706F7300222070617241
:10223000656E743A2200535542524F5554494E45EB
:102240002043414C4C207461726765743A22004B04
:10225000494C4C45442E2000747279696E67207495
:102260006F2063616C6C207375622D67636F6465AA
:102270002066696C6573207769746820746F6F20BD
:102280006D616E79206C6576656C732E204D4158BA
:10229000206C6576656C2069733A0043616E6E6FE1
:1022A00074206F70656E20737562646972200054CB
:1022B000462063617264206F6B0A006F70656E5216
:1022C0006F6F74206661696C65640A00766F6C7567
:1022D0006D652E696E6974206661696C65640A00BB
:1022E0004572726F723A00544620696E69742066B6
:1022F00061696C0A006175746F25692E67004D3243
:1023000034004D323320257300524553554D45203E
:102310004F5054494F4E533A00524553554D452066
:102320004F5054494F4E533A00524553554D452056
:102330004F5054494F4E533A00526573756D6520A6
:102340007072696E7400526573756D652070726984
:102350006E7400526573756D65207072696E7400DD
:1023600045787472756465206D6F72650045787488
:1023700072756465206D6F7265004578747275645E
:1023800065206D6F7265005A204F66667365740034
:102390005A204F6666736574005A204F66667365EF
:1023A000740056656C6F636974790056656C6F6371
:1023B0006974790056656C6F636974790041636371
:1023C000656C65726174696F6E00416363656C650D
:1023D000726174696F6E00416363656C65726174EC
:1023E000696F6E004A65726B004A65726B004A65E0
:1023F000726B0053746570732F6D6D00537465704C
:10240000732F6D6D0053746570732F6D6D004520D3
:10241000696E206D6D33004520696E206D6D33004F
:102420004520696E206D6D330046696C2E2044692D
:10243000612E0046696C2E204469612E0046696C4D
:102440002E204469612E004F6666004F6E200043C7
:10245000616E6E6F7420656E746572207375626450
:1024600069723A2000022E2E0041626F757420506E
:1024700072696E7465720041626F75742050726982
:102480006E7465720041626F7574205072696E746B
:102490006572007777772E637265616C6974792E47
:1024A000636F6D007777772E6378737733642E636D
:1024B0006F6D007777772E637265616C6974792E22
:1024C000636F6D00457874727564657273203100B6
:1024D0004578747275646572732031004578747242
:1024E0007564657273203100426175643A20313140
:1024F0003532303000426175643A20313135323046
:102500003000426175643A20313135323030004359
:102510007265616C6974792056322E350043522DF4
:102520003130205633424C546F75636800312E3180
:102530002E362E30424C00437265616C69747920EE
:1025400033440048656174696E67206661696C6533
:10255000640048656174696E67206661696C6564D2
:102560000048656174696E67206661696C65640026
:102570004D696E696D756D2054656D7020697320AD
:1025800020313730004D696E696D756D2054656D71
:10259000702069732020313730004D696E696D7588
:1025A0006D2054656D7020697320203137300042F2
:1025B00061636B004261636B004261636B0000000A
:1025C0002200250028002B002E00310034000201DB
:1025D0000000050108010B01000020002300260077
:1025E00029002C002F003200000100000301060129
:1025F0000901050505050705080808080202020289
:102600000A0A08080404040401010101010101018E
:102610000303030303030303040707070C0C0C0C59
:102620000C0C0C0C02020202060606060606060642
:102630000B0B0B0B0B0B0B0B0102102020080810CF
:102640002040102040800201020108040201010222
:1026500004081020408080402010080402018004FB
:102660000201804020100804020108040201010256
:10267000040810204080010204081020408000005F
:102680000A0B02090C0D0E080703040100000000EC
:10269000000000000000000000000000000000003A
:1026A00000000000000000000000121110000000F7
:1026B000000000000000000000000000000000001A
:1026C000000000002020506C616E6E6572427566DD
:1026D00066657242797465733A20002046726565BA
:1026E000204D656D6F72793A2000436F6D70696C93
:1026F00065643A2041707220323720323032300A1D
:1027000000207C20417574686F723A2043522D314D
:10271000302056330A00323032302D30342D3237EB
:1027200000204C61737420557064617465643A20B4
:1027300000312E312E362E30424C5F56332E310A68
:10274000004D61726C696E0020536F667477617220
:10275000652052657365740A00205761746368646C
:102760006F672052657365740A002042726F776E3E
:10277000206F75742052657365740A002045787463
:1027800065726E616C2052657365740A00506F77D4
:10279000657255700A0073746172740A0065727212
:1027A0006F722077726974696E6720746F20666932
:1027B0006C650A00456E6473746F70732025632026
:1027C000256320256320256300205A3A0020593ACA
:1027D0000020583A00656E6473746F7073206869E6
:1027E000743A2000446F6E6520736176696E6720CD
:1027F00066696C652E0A004D323900290A00206294
:10280000797465733B206372632000536574746947
:102810006E67732053746F726564202800202863EC
:10282000616C63756C6174656429210A0020213D27
:102830002000454550524F4D20435243206D69734F
:102840006D61746368202D202873746F726564292C
:102850002000290A002062797465733B206372634B
:1028600020002073746F7265642073657474696EE0
:10287000677320726574726965766564202800202C
:102880004D61726C696E3D563431290A0028454508
:1028900050524F4D3D00454550524F4D2076657288
:1028A00073696F6E206D69736D6174636820004891
:1028B000617264636F6465642044656661756C74FD
:1028C0002053657474696E6773204C6F616465642E
:1028D0000A00F4010000F401000064000000E803B5
:1028E00000000000FA430000FA430000A04000008E
:1028F000C8410000A0420000A0420000C843EC1103
:10290000BF43416363656C00416363656C00416371
:1029100063656C00412D7265747261637400412DB2
:102920007265747261637400412D726574726163C3
:102930007400412D74726176656C00412D74726172
:1029400076656C00412D74726176656C00416D6135
:1029500078205800416D6178205800416D617820E1
:102960005800416D6178205900416D61782059000F
:10297000416D6178205900416D6178205A00416DA8
:102980006178205A00416D6178205A00416D61786C
:10299000204500416D6178204500416D61782045FA
:1029A0000056782D6A65726B0056782D6A65726BD9
:1029B0000056782D6A65726B0056792D6A65726BC8
:1029C0000056792D6A65726B0056792D6A65726BB7
:1029D00000567A2D6A65726B00567A2D6A65726BA5
:1029E00000567A2D6A65726B0056652D6A65726BAA
:1029F0000056652D6A65726B0056652D6A65726BAF
:102A0000005873746570732F6D6D00587374657022
:102A1000732F6D6D005873746570732F6D6D005951
:102A200073746570732F6D6D005973746570732FB7
:102A30006D6D005973746570732F6D6D005A7374EA
:102A40006570732F6D6D005A73746570732F6D6DA3
:102A5000005A73746570732F6D6D004573746570E3
:102A6000732F6D6D004573746570732F6D6D004528
:102A700073746570732F6D6D004361726420696EAD
:102A800073657274656400A8A9AAAB00436172649F
:102A900020696E73657274656400436172642072AC
:102AA000656D6F76656400A8A9ACAD004361726482
:102AB0002072656D6F766564004D6F76696E672E66
:102AC0002E2E004572723A204368616E676520467B
:102AD000696C616D656E74005072696E742070610E
:102AE00075736564004572723A204368616E67656C
:102AF0002046696C616D656E7400000C0B00FE076A
:102B00000192032120FFFF0AFF07FF0000000600DB
:102B10000A0107070602008080808080008003028F
:102B200002060105A0A00507070600005050F85056
:102B3000F850500507070600002078A07028F02004
:102B4000050707060000C0C81020409818050707B1
:102B50000600006090A040A89068020303060104EC
:102B6000C04080030707060100204080808040208D
:102B7000030707060100804020202040800505054E
:102B800006000120A870A8200505050600012020E8
:102B9000F820200203030602FFC040800501010661
:102BA0000003F8020202060200C0C0050505060087
:102BB000010810204080050707060000708898A8CB
:102BC000C8887003070706010040C040404040E04D
:102BD000050707060000708808708080F805070761
:102BE000060000F81020100808F00507070600008E
:102BF00010305090F81010050707060000F880F01C
:102C000008088870050707060000708080F0888833
:102C100070050707060000F808102020202005078F
:102C2000070600007088887088887005070706000E
:102C30000070888878080870020505060200C0C088
:102C400000C0C00206060602FFC0C000C0408004EB
:102C500007070600001020408040201005030306EF
:102C60000002F800F804070706000080402010204A
:102C70004080050707060000708808102000200526
:102C8000070706000070880868A8A87005070706EF
:102C90000000708888F8888888050707060000F01B
:102CA0008888F08888F00507070600007088808013
:102CB000808870050707060000F08888888888F0FB
:102CC000050707060000F88080F08080F8050707F8
:102CD000060000F88080F08080800507070600006D
:102CE000708880B888887005070706000088888883
:102CF000F88888880107070602008080808080802D
:102D000080050707060000381010101090600507B6
:102D1000070600008890A0C0A0908805070706005D
:102D200000808080808080F805070706000088D832
:102D3000A8888888880507070600008888C8A8989A
:102D400088880507070600007088888888887005CD
:102D50000707060000F08888F080808005070706D6
:102D6000000070888888A89068050707060000F0B2
:102D70008888F0A09088050707060000788080709A
:102D80000808F0050707060000F820202020202072
:102D90000507070600008888888888887005070767
:102DA00006000088888888885020050707060000EC
:102DB0008888888888A850050707060000888850FA
:102DC0002050888805070706000088888850202042
:102DD00020050707060000F80810204080F80307C8
:102DE00007060000E08080808080E0050505060081
:102DF000018040201008030707060000E020202083
:102E00002020E00503030600042050880501010688
:102E10000000F802020206020580400505050600D2
:102E20000070087888780507070600008080B0C821
:102E30008888F00505050600007080808870050709
:102E400007060000080868988888780505050600C8
:102E5000007088F880700507070600003048E040E1
:102E60004040400506060600FF7088887808700517
:102E700007070600008080B0C88888880107070619
:102E80000200800080808080800308080601FF2007
:102E90000020202020A04004070706010080809029
:102EA000A0C0A090030707060100C040404040407A
:102EB000E0050505060000D0A8A8A8A80505050698
:102EC0000000B0C88888880505050600007088885D
:102ED00088700506060600FFF08888F080800506E9
:102EE000060600FF788888780808050505060000B2
:102EF000B0C880808005050506000070807008F06D
:102F00000407070600004040E0404040300505054A
:102F100006000088888898680505050600008888EE
:102F20008850200505050600008888A8A8500505DA
:102F30000506000088502050880506060600FF8818
:102F40008888780870050505060000F8102040F80C
:102F5000030707060100204040804040200107078A
:102F600006020080808080808080030707060100C1
:102F70008040402040408005020206000368900027
:102F8000000006000A0000000C000A0000000C000F
:102F90000A0000000C000A0000000C000A000000FB
:102FA0000C000A0000000C000A0000000C000A00DF
:102FB00000000C000A0000000C000A0000000C00D9
:102FC0000A0000000C000A0000000C000A000000CB
:102FD0000C000A0000000C000A0000000C000A00AF
:102FE00000000C000A0000000C000A0000000C00A9
:102FF0000A0000000C000A0000000C000A0000009B
:103000000C000A0000000C000A0000000C000A007E
:1030100000000C000A0000000C000A0000000C0078
:103020000A0000000C000A0000000C000A0000006A
:103030000C000A0B0B160C00FFFFE002000200045C
:10304000000D0014802440C4200400040004000B80
:103050000B160C00FFF9008A00ABE0AC40AA40AAB6
:1030600040AA40AA80210052808C600B0B160C00F5
:10307000FF240024003F80440084000400FFE00A95
:103080000011002080C0600B0B160C00FF240024F0
:10309000003FC044000400FFE009000900112021A6
:1030A0002040E00B0B160C00FF20003DE05120916A
:1030B000201120FF201120292025E0452080000B31
:1030C0000B160C00FF20807FC00840FFE01100209D
:1030D000805F4080203F8000007FC00B0B160C00FB
:1030E000FF224047E09480E4802FE04480F4800792
:1030F000E03480C48007E00B0B160C00FF04808FC7
:10310000E0490019002FC0090009002FC0490089BB
:10311000000FE00B0B160C00FF10003F8051000E5B
:10312000003180C0603F8024803F8024803F800B3E
:103130000B160C00FF2280FA4007E0FA808A808A92
:1031400080FA802280B280AAA064E00B0B160C00EB
:10315000FF222047409280EFE0220047C0EC40076A
:10316000C03440C7C004400B0B160C00FF08000F12
:10317000C008000800FFE008000E000980084008B1
:103180000008000A0B160C00FFFF80008000808002
:10319000808080FF8080008000804080407FC00B66
:1031A0000B160C00FF47C04100EFE04100450069ED
:1031B00060C9204D6049204FE0C8200B0B160C0061
:1031C000FF0800040004000A000A000A00110011B0
:1031D000002080404080200B0B160C00FF22402274
:1031E00000F7E0220023E03520E520254028802953
:1031F0004072200B0A140C00004440444044407FBD
:10320000C004000400842084208420FFE00B0B16FF
:103210000C00FF040000007FC00400040004007FD5
:10322000C0040004000400FFE00B0B160C00FFFFBD
:10323000E0110001C0FE00488025000400FFE015F9
:10324000002480C4600B0B160C00FF11007FC044EB
:10325000407FC044407FC00400FFE004000400043D
:1032600000090B160C00FF1000FF8080808080FF9B
:103270008080808080FF8080808080FF800B0B16A4
:103280000C00FF7100010003E0F9202120412051D2
:10329000208920FA20022004C00B0B160C00FF7FAF
:1032A000C01100110011001100FFE01100110021F8
:1032B00000210041000B0B160C00FF21002200F43E
:1032C0004057E0502057C094405440244057C09489
:1032D000400B0B160C00FF11000A007FC004000415
:1032E00000FFE004000A0011002080C0600A0B16F5
:1032F0000C00FF5FC0004084408440BF4084408C8D
:10330000409440A4408C4081C00B0B160C00FF245D
:103310000027C024002400FFE00000144024804760
:10332000000C0070000B0B160C00FF248004800FB3
:10333000C0E48024803FE024802480288050008FD7
:10334000E00B0B160C00FF08000800FF8088808847
:1033500080FF8088808880FFA0882007E00B0B1604
:103360000C00FF27802480F480248074806C80A46B
:1033700080248024A028A030600A0B160C00FFFFD8
:10338000C0804080409E40924092409E408040805D
:1033900040FFC080400B0B160C00FF7FC044005F55
:1033A000C050405FC050405FC042004A805240A6BB
:1033B000200B0B160C00FF040007E004007FC04048
:1033C00040404040407FC00000524089200B0B1617
:1033D0000C00FF4780248004800480E86020002FD8
:1033E000C024402280310026C00B0B160C00FF7F4A
:1033F000C04A407FC00400FFE004003F80208024DA
:10340000802480FFE00B0B160C00FF22004FE048E9
:10341000204FE0C8004FE04AA05AA06FE04AA04801
:10342000600B0B160C00FFF3C024402A80F1002231
:103430008065E07220A540208023002C000B0B1635
:103440000C00FF0400FFE080200000FFE0040024E7
:103450000027C0240054008FE00B0B160C00FF73F4
:10346000E01080510023E0FA202AA022A022A02010
:1034700080214062200B0B160C00FF2200F78022F7
:10348000803680E2A025A024606820000052408998
:10349000200B0B160C00FF73C0420042007BE04A79
:1034A000404A407A404A404240444088400B0B1614
:1034B0000C00FF0800FFE008001FC030405FC09014
:1034C000401FC01040104010C00B0B160C00FF0234
:1034D000007FE0420042005FC0420047004A805245
:1034E00040622082000B0B160C00FFF3C096409147
:1034F00080A660A10097C091009500E7E08100815F
:10350000000B0B160C00FF0F8088804F8008808F07
:103510008040001FC03540554095403FE00B0B16E2
:103520000C00FF27E02080F880208020803880E099
:103530008020802080208061800B0B160C00FF1FF4
:10354000E0910057C0144017C0944057C011005577
:1035500040992023000B0B160C00FF208027E0F27F
:1035600040218022403420E2402240224022406418
:10357000400B0B160C00FF410041004FE0E92049D1
:103580002049206FE0C92049204920CFE00B0B16CD
:103590000C00FF2100F1004FE0A920F9202FE039B5
:1035A00020E92029202FE028200B0B160C00FF8F8C
:1035B000E049200920CBA049204FE048204BA04AF9
:1035C000A06BA050E00B0B160C00FF7FC004004462
:1035D00040244024800400FFE004000400040004B0
:1035E000000B0B160C00FF820042001FE0C2005FC0
:1035F000C052405FC047004A805240BFE00B0B16EC
:103600000C00FF04007FE048807FE048804F80404E
:10361000005FC04840478098600B0B160C00FF010C
:1036200000EFE0A100A440AFE0A440AFE0A920E992
:103630002002800C600B0B160C00FF14C0F6A0BC1F
:1036400060A780A880BFE0A920EFE009200FE00973
:10365000200B0B160C00FF7F80408042806280545C
:10366000804880488054A062A0406080200B0B16E8
:103670000C00FF04007FE040207FE040007DE0542C
:10368000204CA0546064A08D600B0B160C00FF82D0
:10369000005FE0040008409FE040200A800A804A62
:1036A000A092A022600B0B160C00FF41004FE0E837
:1036B00020428044406820C7C0410041004100CF03
:1036C000E00B0B160C00FF50207D209120FF2011F5
:1036D000207D205520552054205C2010E00B0B1637
:1036E0000C00FF3F8020803F802080FFE048007B6F
:1036F000C0494079404880FB600B0B160C00FF046A
:103700000004000400248024404440442084200419
:103710000004001C000B0B160C00FF040004000446
:1037200000FFE004000A000A00110011002080C020
:1037300060090A140A0000888049000800FF800020
:103740008000807F8000800080FF800B0B160C00C3
:10375000FF21001200FFE0000078804A807A804A52
:10376000807A80488059800B0B160C00FF27C00020
:10377000000000EFE02100220024402FE020205034
:10378000008FE00B0B160C00FF20802700F90021B2
:10379000C077002100F9E027007120A92020E00B6C
:1037A0000B160C00FF10401040FDE0104038C035F3
:1037B00040524094401040104010C00B0B160C00BB
:1037C000FF0040F8400BE008408840524051402143
:1037D000405040484089C00A0B160C00FF8400840A
:1037E000408480F5008600840084009400A440C4D6
:1037F0004083C00B0B160C00FF11207D001100FF51
:10380000E02900FD4049407C8008A0FD600A200BB3
:103810000B160C00FF17C02440244067C0A1002FE6
:10382000E0210023802540292021000B0B160C00ED
:10383000FF0800FFE0100027C020806100AFE021FA
:10384000002100210023000B0B160C00FF24002F89
:10385000E0B400A480A4A0AAC02A80288029403215
:103860004024200B0B160C00FF7FE080003FC0209F
:10387000403FC010001FC010402880470038E00BB8
:103880000B160C00FF7FE04000400040004000406D
:1038900000400040004000400080000B0B160C0070
:1038A000FFFFE004007FC044407FC044407FC0442D
:1038B0000024001800E7E00B0B160C00FF11E0FDE0
:1038C00000450029E0FD4011407D401140554092E7
:1038D0004034400B0B160C00FF21005FE04000CF8E
:1038E000C040004FC040004FC048404FC048400B50
:1038F0000B160C00FF04007FC040407FC040407F9B
:10390000C040407FC004405220BFA00B0B160C00EB
:10391000FF7FC044407FC044407FC004001B00E0E4
:10392000E01100110061000B0B160C00FFFFE0041A
:103930000008007FE049204F2049204F20492049BE
:10394000207FE00B0B160C00FFFDE056407940385D
:103950008055409220FFE0040027C02400FFE00BC8
:103960000B160C00FFFB8052007BE01240FA401463
:10397000403F8020803F8020803F800B0B160C0052
:10398000FF1FE0200027C06440A7C020002FE028D0
:103990002027C0210023000B0B160C00FFF3E08250
:1039A000208220FA20822082208A20B220C2E002D7
:1039B0000002000B0B160C00FF248046A095C0E40B
:1039C0008027E04480F5C006A03480C48007E00B67
:1039D0000B160C00FF27C0410087E0E02022804545
:1039E00080F2800FE03080C14002200B0B160C00EB
:1039F000FF02000200220023C02200220022002237
:103A00000022002200FFE0090B160C00FF0800084E
:103A100000FF80888088808880FF808880888088F8
:103A200080FF800B0B160C00FF210053A04100F714
:103A3000E0510053C0564053C05A4053C042400B5F
:103A40000B160C00FF7FC0040004000400FFE00A16
:103A5000000A0012002220422081E00B0B160C000D
:103A6000FF110021002FE06100A380238025402565
:103A7000402920210021000B0B160C00FFF7E094D9
:103A800020F42097E09480F48097E09480F4A0964E
:103A90006004200B0B160C00FF7BE0948004007F79
:103AA000C00400FFE00100FFE02100110007000B4F
:103AB0000B160C00FF210047C091002FE06080AF83
:103AC000E0208024802280208023800B0B160C00B5
:103AD000FF27C02440F7C02EE02AA03EE0E1002FDF
:103AE000E02380254069200B0B160C00FF140027F3
:103AF000E02A006200A3C02200220023E02200226C
:103B000000220000060900FE070192032120FFFFAA
:103B100008FF07FF0000000600000107070602007B
:103B200080808080800080030202060105A0A0053D
:103B300007070600005050F850F8505005070706D8
:103B400000002078A07028F020050707060000C0BC
:103B5000C810204098180507070600006090A04094
:103B6000A89068020303060104C04080030707060B
:103B7000010020408080804020030707060100806C
:103B800040202020408005050506000120A870A8DF
:103B9000200505050600012020F820200203030669
:103BA00002FFC04080050101060003F80202020680
:103BB0000200C0C005050506000108102040800570
:103BC0000707060000708888888888700307070642
:103BD000010040C040404040E0050707060000707B
:103BE0008808708080F8050707060000F81020108C
:103BF0000808F005070706000010305090F8101074
:103C0000050707060000F880F00808887005070718
:103C1000060000708080F0888870050707060000A5
:103C2000F80810202020200507070600007088886B
:103C30007088887005070706000070888878080873
:103C400070020505060200C0C000C0C002060606DC
:103C500002FFC0C000C0408004070706000010201B
:103C60004080402010050303060002F800F8040716
:103C7000070601008040201020408005070706004D
:103C800000708808102000200507070600007088D3
:103C90000868A8A870050707060000708888F888DB
:103CA0008888050707060000F08888F08888F005F6
:103CB0000707060000708880808088700507070667
:103CC0000000F08888888888F0050707060000F85B
:103CD0008080F08080F8050707060000F88080F0FB
:103CE000808080050707060000708880B88888708B
:103CF000050707060000888888F888888801070774
:103D00000602008080808080808005070706000012
:103D1000381010101090600507070600008890A06A
:103D2000C0A0908805070706000080808080808002
:103D3000F805070706000088D8A88888888805073E
:103D4000070600008888C8A8988888050707060025
:103D50000070888888888870050707060000F0884A
:103D600088F080808005070706000070888888A892
:103D70009068050707060000F08888F0A090880585
:103D80000707060000788080700808F0050707061E
:103D90000000F820202020202005070706000088CA
:103DA00088888888887005070706000088888888C2
:103DB0008850200507070600008888888888A85052
:103DC00005070706000088885020508888050707E7
:103DD000060000888888502020200507070600007C
:103DE000F80810204080F8030707060100E08080F3
:103DF000808080E005050506000180402010080352
:103E00000707060100E02020202020E0050303062C
:103E10000004205088050101060000F80202020695
:103E200002058040050505060000700878887805C1
:103E300007070600008080B0C88888F005050506E1
:103E40000000708080887005070706000008086879
:103E5000988888780505050600007088F880700548
:103E600007070600003048E04040404005060606CF
:103E700000FF7088887808700507070600008080BA
:103E8000B0C888888801070706020080008080800B
:103E900080800308080601FF200020202020A04089
:103EA000040707060000808090A0C0A090030707C9
:103EB000060100C04040404040E005050506000006
:103EC000D0A8A8A8A8050505060000B0C88888885D
:103ED000050505060000708888887005060606003E
:103EE000FFF08888F080800506060600FF78888845
:103EF000780808050505060000B0C8808080050523
:103F00000506000070807008F004070706000040F6
:103F100040E040404030050505060000888888984C
:103F200068050505060000888888502005050506F7
:103F300000008888A8A850050505060000885020C4
:103F400050880506060600FF8888887808700505F1
:103F500005060000F8102040F803070706010020BE
:103F6000404080404020010707060200808080809A
:103F70008080800307070601008040402040408089
:103F80000502020600026890000000060000000022
:103F9000000600000000000600000000000600000F
:103FA00000000006000000000006000000000006FF
:103FB00000000000000600000000000600000000F5
:103FC00000060000000000060000000000060000DF
:103FD00000000006000000000006000000000006CF
:103FE00000000000000600000000000600000000C5
:103FF00000060000000000060000000000060000AF
:10400000000000060000000000060000000000069E
:104010000000000000060000000000060000000094
:10402000000600000000000600000000000600007E
:10403000000000060000000000060000000000066E
:104040000000000000060000000000060000000064
:1040500000060000010707060200800080808080C3
:10406000800507070600002070A8A0A8702005079B
:1040700007060000304040E04050A8050505060056
:10408000008870507088050707060000885020F8E7
:1040900020F82001070706020080808000808080D1
:1040A00005080806000030482050502090600301A9
:1040B00001060107A0050707060000F888B8B8B890
:1040C00088F8050707060001700878887800F80569
:1040D00005050600012850A050280503030600012D
:1040E000F8080802020206020640800507070600DB
:1040F00000F888A88898A8F8050101060006F804C9
:104100000404060003609090600507070600002085
:1041100020F8202000F804050506000360902040E8
:10412000F0030505060003E020E020E0020202069D
:10413000020640800508080600FF8888888898E8FD
:1041400080800507070600007898987818181802EC
:104150000202060202C0C00202020602FF40800301
:10416000050506000340C04040E0050707060001C2
:10417000708888887000F8050505060001A05028A1
:1041800050A00507070600008890A858B808080541
:1041900007070600008890B84898203805080806E8
:1041A0000000C040C048D8380808050707060000CE
:1041B000200020408088700508080600004020008C
:1041C0007088F888880508080600001020007088AC
:1041D000F888880508080600002050007088F888D4
:1041E000880508080600006890007088F88888052F
:1041F00008080600005000708888F88888050808BC
:104200000600002050207088F888880507070600FF
:10421000003860A0B8E0A0B80508080600FF708864
:10422000808088702060050808060000402000F8A3
:1042300080F080F8050808060000081000F880F0FB
:1042400080F8050808060000205000F880F080F88B
:104250000507070600005000F880F080F803080802
:10426000060100804000E0404040E00308080601ED
:1042700000204000E0404040E00308080601004004
:10428000A000E0404040E0030707060100A000E076
:10429000404040E0050707060000704848E84848ED
:1042A0007005080806000068900088C8A89888056E
:1042B0000808060000402070888888887005080873
:1042C000060000102070888888887005080806009D
:1042D0000020500070888888700508080600006873
:1042E00090007088888870050808060000500070EB
:1042F0008888888870050505060001885020508848
:104300000508080600FF1070A8A8A8A870400508B6
:1043100008060000402088888888887005080806FC
:10432000000010208888888888700508080600002A
:104330002050008888888870050808060000500012
:104340008888888888700508080600001020885032
:10435000202020200509090600FFC0407048487051
:104360004040E00408080601FF609090A09090E0B3
:10437000800508080600004020007008788878054D
:1043800008080600001020007008788878050808E2
:10439000060000205000700878887805080806009C
:1043A00000689000700878887805070706000050BC
:1043B00000700878887805080806000020502070F2
:1043C00008788878050606060000D02878A0A8504E
:1043D0000506060600FF7080887020600508080644
:1043E00000004020007088F8807005080806000072
:1043F0001020007088F88070050808060000205022
:10440000007088F88070050707060000500070886B
:10441000F8807003080806010080400040C040405A
:10442000E003080806010020400040C04040E003CF
:10443000080806010040A00040C04040E003070714
:10444000060100A00040C04040E00507070600004C
:10445000A040A01078887005080806000068900049
:10446000B0C88888880508080600004020007088C9
:104470008888700508080600001020007088888869
:1044800070050808060000205000708888887005B4
:104490000808060000689000708888887005070783
:1044A0000600005000708888887005050506000128
:1044B0002000F800200507070600FF1070A8A8A834
:1044C0007040050808060000402000888888986829
:1044D00005080806000010200088888898680508EC
:1044E000080600002050008888889868050707069D
:1044F0000000500088888898680509090600FF10A8
:104500002000888888F808700407070601FFC0406B
:1045100060506040E00508080600FF500088888869
:10452000780870496E666F2073637265656E00EC83
:10453000EDEEEF00496E666F2073637265656E0085
:1045400054756E6500CFF00054756E65004C616E59
:104550006775616765004C616E6775616765004CE2
:10456000616E677561676500506175736520707273
:10457000696E7400F1F2CAF30050617573652070C2
:1045800072696E74005072696E742066726F6D206D
:10459000544600AFB0005072696E742066726F6D41
:1045A000205446004E6F205446206361726400F927
:1045B000A8004E6F2054462063617264004D36306F
:1045C0003020423000537065656400D1D2005370D2
:1045D00065656400466C6F7700CCADD1D200466C47
:1045E0006F77004261627973746570205A0042618E
:1045F000627973746570205A0042616279737465E0
:1046000070205A0070012C0190012701B001220195
:10461000C0011D01F00118011002130130020E014A
:104620006002090190020401C002FF000003FA00C9
:104630004003F5008003F000D003EB002004E60007
:104640007004E100E004DC004005D700C005D200A2
:104650004006CD00D006C8008007C3003008BE0069
:10466000F008B900C009B400B00AAF00B00BAA004E
:10467000D00CA500000EA000500F9B00C0109600AB
:104680005012910000148C00C0158700B0178200F2
:10469000B0197D00D01B7800001E730040206E0012
:1046A00090226900F024640040275F0090295A009E
:1046B000E02B5500102E500020304B0010324600E9
:1046C000E033410090353C0010373700703832003D
:1046D000A0392D00B03A2800A03B2300603C1E000A
:1046E000103D1900903D1400103E0F00703E0A006E
:1046F000C03E0500003F0000403FFBFF803FF6FF4B
:10470000C03FF1FF544845524D414C2052554E4157
:1047100057415900546865726D616C2052756E6125
:10472000776179004572723A204D494E54454D509B
:1047300020424544004572723A204D494E54454D41
:1047400050004D494E54454D50207472696767655D
:10475000726564004572723A204D415854454D507F
:1047600020424544004572723A204D415854454D0F
:1047700050004D415854454D50207472696767652B
:10478000726564004D61696E00AEAFB0004D616945
:104790006E004D6F7665205800C1B22058004D6FF5
:1047A00076652058004D6F7665205900C1B22059BA
:1047B000004D6F76652059004D6F7665205A00C117
:1047C000B2205A004D6F7665205A00457874727594
:1047D00064657200CCADBA00457874727564657218
:1047E000004E6F7A7A6C6500D3D4004E6F7A7A6C83
:1047F000650042656400C4C7004265640046616E9E
:1048000020737065656400D5D6D1D20046616E20F4
:10481000737065656400436F6E74726F6C00D8D9F5
:1048200000436F6E74726F6C004D6F74696F6E0031
:10483000DFB2004D6F74696F6E0050726570617207
:104840006500A4A5005072657061726500526573C1
:10485000756D65207072696E7400F4F5CAF30052CC
:104860006573756D65207072696E740053746F7036
:10487000207072696E7400F2F6CAF30053746F70A0
:10488000207072696E74005052494E542050415548
:10489000534544005052494E5420504155534544CD
:1048A000005052494E542050415553454400202059
:1048B0004E6F7A7A6C653A200020204E6F7A7A6CBF
:1048C000653A200020204E6F7A7A6C653A2000000D
:1048D000060900FE000000000001090008FE0000BB
:1048E00005080806000040F0C88888987810050878
:1048F00008060000C0F88888888888F8050505063D
:1049000000012030F830200508080600002070F86B
:1049100020202020E00509090600FF2070A8A8B883
:10492000888870200509090600FFE080C0B0A8282B
:104930003028280509090600FFF8A8888888888893
:10494000A8F8050A0A0600FE205050505088A8A872
:10495000887003030306000340A040456E676C693E
:10496000736800456E676C69736800456E676C69B3
:104970007368004368696E657365004368696E65B6
:104980007365004368696E6573650050726568659C
:10499000617420504C4120636F6E660050726568F0
:1049A00065617420504C4120BEBF0050726568653F
:1049B000617420504C4120636F6E660050726568D0
:1049C0006561742041425320636F6E6600507265CA
:1049D000686561742041425320BEBF005072656813
:1049E0006561742041425320636F6E660054656DAB
:1049F000706572617475726500C9D20054656D701E
:104A0000657261747572650053746F7265207365A9
:104A10007474696E67730053746F7265206D656D91
:104A20006F72790053746F72652073657474696E68
:104A3000677300566D6178205800566D6178205874
:104A400000566D6178205800566D617820590056E7
:104A50006D6178205900566D6178205900566D615E
:104A600078205A00566D6178205A00566D61782082
:104A70005A00566D6178204500566D6178204500DA
:104A8000566D6178204500566D696E00566D696EF1
:104A900000566D696E005654726176206D696E0025
:104AA0005654726176206D696E005654726176209C
:104AB0006D696E007C3C3E5E2B3D3F2F5B5D3B2C69
:104AC0002A225C0020746F6F206C6F6E67206578FF
:104AD00074727573696F6E2070726576656E746539
:104AE000640A0020636F6C64206578747275736962
:104AF0006F6E2070726576656E7465640A00507220
:104B0000656865617420504C4120456E64005072A8
:104B1000656865617420504C4120456E6400507298
:104B2000656865617420504C4120456E6400507288
:104B3000656865617420504C412042656400507284
:104B4000656865617420504C4120C4C7005072658F
:104B50006865617420504C41204265640050726564
:104B6000686561742041425320456E64005072654F
:104B7000686561742041425320456E64005072653F
:104B8000686561742041425320456E64005072652F
:104B9000686561742041425320426564005072652B
:104BA000686561742041425320C4C7005072656833
:104BB00065617420414253204265640047323800E9
:104BC0004175746F20686F6D6500BBBCBD00417599
:104BD000746F20686F6D6500426564204C65766572
:104BE0006C696E6700B1B2CFD000426564204C653D
:104BF00076656C696E67004D3432380053657420F9
:104C0000686F6D65206F66667365747300BEBFBBA9
:104C1000BCBDC0C10053657420686F6D65206F66B0
:104C200066736574730044697361626C65207374A4
:104C300065707065727300B5B6B7B8B9BA004469EB
:104C40007361626C65207374657070657273004384
:104C500068616E67652066696C616D656E7400439E
:104C600068616E67652066696C616D656E7400438E
:104C700068616E67652066696C616D656E7400437E
:104C80006F6F6C646F776E00C8C900436F6F6C64A0
:104C90006F776E005072656865617420504C4100FA
:104CA000C3C420504C410050726568656174205047
:104CB0004C4100507265686561742041425300C3E5
:104CC000C4204142530050726568656174204142BE
:104CD00053004D3834004732380A47323900656E88
:104CE0007175657565696E672022006563686F3A46
:104CF000002E0A006F70656E206661696C65642C19
:104D00002046696C653A200057726974696E6720A5
:104D1000746F2066696C653A20004D6F766520617E
:104D200078697300C1B2CE004D6F766520617869F5
:104D300073004D6F76652031306D6D00C1B220314A
:104D4000306D6D004D6F76652031306D6D004D6FAB
:104D5000766520316D6D00C1B220316D6D004D6FF3
:104D6000766520316D6D004D6F766520302E316D8A
:104D70006D00C1B220302E316D6D004D6F76652013
:104D8000302E316D6D0046696C616D656E7400E0AA
:104D9000E10046696C616D656E7400424C546F753C
:104DA000636800424C546F75636800424C546F75E1
:104DB0006368004C6F61642073657474696E677317
:104DC000004C6F6164206D656D6F7279004C6F618E
:104DD000642073657474696E677300496E697469E1
:104DE000616C697A6520454550524F4D00496E69A6
:104DF0007469616C697A6520454550524F4D004990
:104E00006E697469616C697A6520454550524F4DF1
:104E10000050726F62696E67206661696C65640A32
:104E20000050726F62696E67206661696C6564002C
:104E3000205A3A200020593A200042656420583A0E
:104E400020002E0A0046696C652862696E2920647C
:104E5000656C657465640044656C6574696F6E2883
:104E600062696E29206661696C656400000021003A
:104E7000240027002A002D0030003300010100002B
:104E8000040107010A014572726F7220777269741A
:104E9000696E6720746F20454550524F4D210A00BE
:104EA0005072696E742070617573656400473020BC
:104EB00046333030302058302059300000473932E6
:104EC00020452573004730205A2573004D31303975
:104ED00020532569004D31343020532569004D3170
:104EE00030362053323535004730205A257300477D
:104EF0003238205830205930004D31303920532578
:104F000069004D31393020532569005072696E7443
:104F10002061626F7274656400506F7765722D4C0A
:104F20006F7373205265636F766572793F00A4A535
:104F3000F4F5CAF3203F00506F7765722D4C6F7304
:104F400073205265636F766572793F0052657365B1
:104F50007420424C546F7563680052657365742009
:104F6000424C546F75636800526573657420424CFF
:104F7000546F75636800424C546F756368205365C5
:104F80006C662D5465737400424C546F75636820D1
:104F900053656C662D5465737400424C546F756391
:104FA000682053656C662D54657374004465706C9D
:104FB0006F7920424C546F756368004465706C6F64
:104FC0007920424C546F756368004465706C6F794A
:104FD00020424C546F7563680053746F7720424CC5
:104FE000546F7563680053746F7720424C546F752B
:104FF00063680053746F7720424C546F7563680088
:105000004D32383020503020533930004D32383056
:1050100020503020533130004D3238302050302075
:1050200053313230004D3238302050302053313639
:105030003000526573656E643A20006F6B00207417
:105040006F6F206C6F6E6720657874727573696F0F
:105050006E2070726576656E7465640A0020636FF9
:105060006C6420657874727573696F6E20707265F8
:1050700076656E7465640A00F800F00011241FBEA6
:10508000CFEFD1E2DEBFCDBF00E00CBF15E0A0E066
:10509000B2E0E6E6FBE502E00BBF02C007900D922E
:1050A000A839B107D9F72BE1A8E9B5E001C01D92F5
:1050B000AD37B207E1F718E2CDE3D8E200E006C071
:1050C00021970109802FFE010F94152DCC33D107B4
:1050D00080E00807A9F70F9415140D94A22D0C94E5
:1050E00000002F923F924F925F926F927F928F9229
:1050F0009F92AF92BF92CF92DF92EF92FF920F9367
:105100001F93CF93DF93CDB7DEB7CF55D1090FB63D
:10511000F894DEBF0FBECDBF0091CE1120E6029FF6
:1051200080011124025B1F4E8091471280FF1AC03C
:10513000EBEEFCE484917F013FEFE31AF30A811167
:1051400002C0780104C00E94F245F701F3CFD701F5
:105150008D917D01882319F00E94F245F8CF8AE0F5
:105160000E94F24581E090E09093460680934506C8
:105170001092B7051092B6058FE38093C005109288
:10518000BF051092BE0584E0E2EBF5E0DF011D9261
:105190008A95E9F7F80180810F5F1F4F8032D1F3C4
:1051A0008E34C9F4818190ED980F9A3020F08D32C1
:1051B00011F08B3281F4DF0112969D012F5F3F4F7A
:1051C0008C9180538A3010F4D901F7CFFD011196EC
:1051D00080818032D9F3F0934E06E0934D067F0133
:1051E000BFEFEB1AFB0A10816AE270E0C7010F946F
:1051F0006A2D009731F0FC01319780818032E1F314
:1052000011821D3431F1143521F1173411F1EBEE17
:10521000FCE484918F010F5F1F4F882321F00E94CF
:10522000F245F801F6CF60914D0670914E0689E780
:1052300096E00F94200D82E20E94F2458AE00E94DF
:10524000F24510924606109245060F94420A0C94BD
:105250000640C701FC01208101962032D9F320537A
:105260002A30A8F61093C00580E090E06AE03196FD
:10527000DF0111972C91022E000C330B20533109C2
:10528000689FA001699F500D1124C901840F951FCB
:10529000208120532A3058F39093BF058093BE0598
:1052A000DF0131962C912032D9F31D34D1F48E31A7
:1052B000910591F03CF48731910571F08C319105A5
:1052C00081F40AC08537910564F08737910524F091
:1052D000803AE3E09E0729F4B093B705A093B605A2
:1052E0007DC01092B7051092B60500914D06EE24D0
:1052F000E394F12CFD0131962C91222309F46EC028
:105300002132A9F41D3499F48032910581F4F0938F
:10531000B705E093B60563E270E0CF010F946A2D04
:10532000009711F40C94C332DC011C9257C0215435
:105330002A31A0F5AF01FA0130814F5F5F4F303263
:10534000D1F340ED430F4A3040F043ED430F42307C
:1053500020F03B3211F00C94173FAF01622F70E048
:10536000DB0133E0B595A7953A95E1F7AE54BA4F16
:105370002770670102C0CC0CDD1C2A95E2F796016C
:105380003C91232B2C934115510511F0401B01C07A
:1053900040E0DB01A856BA4F4C930AC02091B605F5
:1053A0003091B705232B21F4B093B705A093B60530
:1053B000208121542A3110F4DF019CCFDF01AD019F
:1053C0004F5F5F4F2C9120532A3010F4DA01F7CF52
:1053D000FD01119620812032D9F3EECF8091C005D6
:1053E0008D3411F40C94C332843511F40C94DC3EEA
:1053F000873409F00CCF2090BE053090BF052CE11A
:105400002216310409F4C7C58CF444E02416310493
:105410003CF452E025163104B4F537FE2AC011CF12
:1054200084E02816310409F471C50BCF9AE22916DD
:10543000310409F4DBC75CF4BDE12B16310409F437
:10544000E6C6EEE12E16310409F4E4C6FACEFBE519
:105450002F16310409F463C72CE52216310409F430
:1054600063C73AE52316310409F0EBCE1092BD056F
:10547000E8CE80910B02882309F4E3CE0E94CF503E
:105480000F940707DECE80910B02882309F4D9CE52
:105490000E94CF5082E50E949D45882309F43CC1BB
:1054A0000E943B454B015C0180914119909142194A
:1054B000A0914319B09144198CA79DA7AEA7BFA78F
:1054C000209145193091461940914719509148193A
:1054D00028AB39AB4AAB5BAB80913F089091400859
:1054E000A0914108B09142088CAF9DAFAEAFBFAF65
:1054F0002091430830914408409145085091460856
:105500002CAB3DAB4EAB5FAB20E030E0A901C50159
:10551000B4010F947B23882309F42AC12CAD3DAD3F
:105520004EAD5FAD6CA57DA58EA59FA50F947B2389
:1055300081110DC02CA93DA94EA95FA968A979A91F
:105540008AA99BA90F947B23882309F411C111E038
:1055500032E02316310409F010E020E030E0A90128
:10556000C501B4010F947B23881F8827881F181753
:1055700059F080E090E0A0E8BFEB28968CAF9DAF9B
:10558000AEAFBFAF28970AC020E030E040E85FE34D
:1055900028962CAF3DAF4EAF5FAF28972CA53DA509
:1055A0004EA55FA56CAD7DAD8EAD9FAD0F94142A59
:1055B00068AF79AF8AAF9BAF28A939A94AA95BA97F
:1055C0006CA97DA98EA99FA90F94142A6B017C0157
:1055D00028AD39AD4AAD5BADCA01B9010F94E023E6
:1055E0002B013C01A7019601C701B6010F94E023EE
:1055F0009B01AC01C301B2010F94152A0F94812CB9
:1056000024966CAF7DAF8EAF9FAF249720E030E043
:1056100040E05FE30F94E0232B013C01A5019401DE
:10562000C501B4010F94E0234B015C01A301920179
:10563000C301B2010F94E0239B01AC01C501B40189
:105640000F94142A0F94812C28962CAD3DAD4EADAD
:105650005FAD28970F94E0234B015C01C701B601B1
:10566000905824962CAD3DAD4EAD5FAD24970F9470
:10567000F12AA50194010F94E0236B017C012CAD6C
:105680003DAD4EAD5FAD6CA57DA58EA59FA50F94DC
:10569000152A20E030E040E05FE30F94E0239B0117
:1056A000AC01C701B6010F94152A2CA53DA54EA546
:1056B0005FA50F94142A6B017C012CA93DA94EA96A
:1056C0005FA968A979A98AA99BA90F94152A20E046
:1056D00030E040E05FE30F94E0232B013C0124968F
:1056E0002CAD3DAD4EAD5FAD249768AD79AD8AADC3
:1056F0009BAD0F94F12AA50194010F94E0239B0127
:10570000AC01C301B2010F94152A28A939A94AA9ED
:105710005BA90F94142A14C089E40E949D45882334
:1057200029F00E943B456B017C0103C0C12CD12CA8
:1057300076018AE40E949D458823E9F00E943B455A
:105740006CAF7DAF8EAF9FAF20E030E0A901C70105
:10575000B6010F947B2381111BC020E030E0A9012A
:105760006CAD7DAD8EAD9FAD0F947B23811110C0CC
:10577000E0EEF2E2B8C320E030E0A901C701B601D3
:105780000F947B238823A1F31CAE1DAE1EAE1FAE6B
:10579000D701C601B0588CA79DA7AEA7BFA72CAD57
:1057A0003DAD4EAD5FAD505828AB39AB4AAB5BABAE
:1057B0009C01AD01BC01CD010F94E0234B015C01C4
:1057C00028A939A94AA95BA9CA01B9010F94E02304
:1057D0009B01AC01C501B4010F94152A0F94812CD3
:1057E00068966CAF7DAF8EAF9FAF6897809141197F
:1057F00090914219A0914319B09144198CAB9DAB83
:10580000AEABBFABA7019601BC01CD010F94152A29
:1058100028966CAF7DAF8EAF9FAF2897209145192A
:1058200030914619409147195091481924962CAF50
:105830003DAF4EAF5FAF24972CAD3DAD4EAD5FADEC
:1058400024966CAD7DAD8EAD9FAD24970F94152A37
:105850006C966CAF7DAF8EAF9FAF6C9780913F0819
:1058600090914008A0914108B09142082C968CAFCD
:105870009DAFAEAFBFAF2C9728962CAD3DAD4EADD2
:105880005FAD2897BC01CD010F94142A6B017C01F8
:1058900020914308309144084091450850914608B2
:1058A00060962CAF3DAF4EAF5FAF60976C962CAD5E
:1058B0003DAD4EAD5FAD6C9760966CAD7DAD8EAD80
:1058C0009FAD60970F94142A4B015C018091491998
:1058D00090914A19A0914B19B0914C1964968CAFD4
:1058E0009DAFAEAFBFAF64979C01AD01609147081B
:1058F000709148088091490890914A080F94142AA1
:1059000068AF79AF8AAF9BAFA70196016CA57DA563
:105910008EA59FA50F94E0232B013C01A5019401C6
:1059200068A979A98AA99BA90F94E0239B01AC01DE
:10593000C301B2010F94152A2B013C01A50194016A
:105940006CA57DA58EA59FA50F94E0234B015C015E
:10595000A701960168A979A98AA99BA90F94E023B8
:105960009B01AC01C501B4010F94142AA30192015B
:105970000F94882A6B017C0120E030E0A9010F948C
:105980007B2387FF0AC02BED3FE049EC50E4C701C1
:10599000B6010F94152A6B017C0192E0291631049F
:1059A00051F42BED3FE049EC50E4C701B6010F94F0
:1059B000142A6B017C0120E030E0A901C701B60187
:1059C0000F947B23811126C02C962CAD3DAD4EAD9E
:1059D0005FAD2C976CA97DA98EA99FA90F947B23FD
:1059E000811118C060962CAD3DAD4EAD5FAD609796
:1059F00024966CAD7DAD8EAD9FAD24970F947B2327
:105A0000811108C08BEDC82E8FE0D82E89ECE82ECE
:105A100080E4F82EA701960168966CAD7DAD8EAD41
:105A20009FAD68970F94E0239B01AC010F94E02396
:105A30004B015C0128AD39AD4AAD5BADCA01B9017E
:105A40000F94E0239B01AC01C501B4010F94152A0A
:105A50000F94812C4B015C012FE632E143E85AE3BD
:105A60000F947B2387FD39C2C501B4010F948A2BA3
:105A70000F945E2B22967FAF6EAF2297DB01AB2B8C
:105A800031F4E1E0F0E02296FFAFEEAF22974090D4
:105A90004D1950904E1960904F19709050192296E0
:105AA0002EAD3FAD2297B90180E090E00F947F23A7
:105AB0004B015C019B01AC01C701B6010F94F12AB7
:105AC0006CAB7DAB8EAB9FABA501940168AD79AD9E
:105AD0008AAD9BAD0F94F12A68966CAF7DAF8EAF07
:105AE0009FAF6897A301920160914B0870914C0899
:105AF00080914D0890914E080F94142AA5019401AD
:105B00000F94F12AA0966CAF7DAF8EAF9FAFA09798
:105B10002CA93DA94EA95FA9CA01B9010F94E023A0
:105B200020E030E040E05FE30F94E0239B01AC0114
:105B300060E070E080E89FE30F94142A2C966CAF2D
:105B40007DAF8EAF9FAF2C9764968CAD9DADAEAD03
:105B5000BFAD649789879A87AB87BC874D865E8681
:105B60006F86788A60911B0270911C02072E000CD0
:105B7000880B990B0F94812320918C0230918D0218
:105B800040918E0250918F020F94E0232AE037ED6E
:105B900043E25CE30F94E02360966CAF7DAF8EAF81
:105BA0009FAF60970E947EF79B01AC0128533F4F47
:105BB0004F4F5F4F64962CAF3DAF4EAF5FAF6497D2
:105BC0004CA45DA46EA47FA422242394312C39E13B
:105BD00038AF22964EAD5FAD22974215530509F4BA
:105BE00038C10E94D47B0E947EF7DC01CB01649611
:105BF0002CAD3DAD4EAD5FAD6497821B930BA40BF6
:105C0000B50BB7FD11C00E947EF79B01AC01285374
:105C10003F4F4F4F5F4F64962CAF3DAF4EAF5FAFDE
:105C2000649780E00E947C6738AD315038AF3323F1
:105C300009F441C028A939A94AA95BA92C966CADE1
:105C40007DAD8EAD9FAD2C970F94E0236B017C0151
:105C50009201A3016CA97DA98EA99FA90F94E023AD
:105C6000A70196010F94152A6B017C019201A301F3
:105C70002C966CAD7DAD8EAD9FAD2C970F94E0232F
:105C80004B015C0128A939A94AA95BA96CA97DA986
:105C90008EA99FA90F94E0239B01AC01C501B4011B
:105CA0000F94142A2B013C01C601D70188AB99AB94
:105CB000AAABBBAB4DC0B10180E090E00F947F2355
:105CC0002CA93DA94EA95FA90F94E0234B015C01CB
:105CD0000F94EE2A6B017C01C501B4010F94772C5F
:105CE0004B015C01A70196016CA57DA58EA59FA522
:105CF0000F94E0232B013C012CAD3DAD4EAD5FADCB
:105D0000C501B4010F94E023A30192010F94152A59
:105D10002B013C01A50194016CA57DA58EA59FA535
:105D20000F94E0234B015C012CAD3DAD4EAD5FAD5A
:105D3000C701B6010F94E0239B01AC01C501B4017A
:105D40000F94142A68AB79AB8AAB9BAB49E148AF9F
:105D50009201A30128966CAD7DAD8EAD9FAD2897C5
:105D60000F94152A69837A838B839C8328A939A988
:105D70004AA95BA96C966CAD7DAD8EAD9FAD6C975D
:105D80000F94152A6D837E838F83988768962CAD38
:105D90003DAD4EAD5FAD689769857A858B859C85F5
:105DA0000F94152A69877A878B879C87A0962CADDC
:105DB0003DAD4EAD5FADA0976D857E858F85988991
:105DC0000F94152A6D877E878F87988B80918B0221
:105DD000882321F0CE0101960E94EB63C0906C08ED
:105DE00089819A81AB81BC8188A399A3AAA3BBA313
:105DF0008D819E81AF81B8858CA39DA3AEA3BFA3E7
:105E000089859A85AB85BC8588A799A7AAA7BBA7D2
:105E1000AE01485D5F4FBE016C5D7F4FCE01809645
:105E20000E940EE26096ECACFDAC0EAD1FAD60972B
:105E30009E01235F3F4FAE01485D5F4FBE016C5D29
:105E40007F4FCE0180960E94F1D45FEF251A350A6C
:105E5000C0CEC0906C0880913F0890914008A091FE
:105E60004108B091420888A399A3AAA3BBA380913B
:105E7000430890914408A0914508B09146088CA32E
:105E80009DA3AEA3BFA38091470890914808A0911D
:105E90004908B0914A0888A799A7AAA7BBA7AE014D
:105EA000485D5F4FBE016C5D7F4FCE0180960E94C2
:105EB0000EE26096ECACFDAC0EAD1FAD60972BE42E
:105EC00038E0AE01485D5F4FBE016C5D7F4FCE0193
:105ED00080960E94F1D40E9448430E94AF45B1C908
:105EE0000E94F245F80184918F010F5F1F4F8111CD
:105EF000F7CFE3E5F3E084918F010F5F1F4F882315
:105F000009F49FC90E94F245F801F5CF80E50E948F
:105F10009D45882329F00E94FB446B017C0103C04E
:105F2000C12CD12C760183E50E949D45882361F028
:105F30000E943B4520E030E04AE754E40F94E02320
:105F40000F945E2B6B017C010E94717F8091360261
:105F5000811105C060E089E693E00E94CFB30E9402
:105F6000AF4580912A1090912B10A0912C10B091E8
:105F70002D10C80ED91EEA1EFB1E0E947EF7DC0102
:105F8000CB018C199D09AE09BF09B7FF5AC980E042
:105F90000E947C67F2CF0E94717F80E00E943D41A9
:105FA0000E94D34511E01093151088E50E946E45BC
:105FB000E82E89E50E946E45082F8AE50E946E450D
:105FC000F82EE11004C0011104C0182705C001110A
:105FD00002C010E001C0182F0E943E43111105C0FD
:105FE000E11003C0002309F440C020E030E040EAA3
:105FF00050E460917C1670917D1680917E16909190
:106000007F160F94152A6093470870934808809371
:10601000490890934A082091491930914A194091B2
:106020004B1950914C190F943B2C18165CF41982A3
:106030001A821B821C82BE016F5F7F4F87E498E04B
:106040000E94AB42111105C0E11003C0011107C04D
:106050000CC080E090E00E94AE621123B9F381E0B1
:1060600090E00E94AE62111103C0FF2009F4BEC08F
:1060700080911610882321F08091171081111FC084
:1060800060E086EA93E00E94CFB3EBEEFCE48491FB
:106090008F010F5F1F4F811103C0E5E9F3E004C0DA
:1060A0000E94F245F801F3CF84918F010F5F1F4FDB
:1060B000882309F49BC00E94F245F801F5CF0E94A5
:1060C000B444409074165090751660907616709097
:1060D00077168090781690907916A0907A16B090E6
:1060E0007B1620E030E046E153E4C501B4010F9493
:1060F000152A6B017C0160934308709344088093D8
:106100004508909346088091491990914A19A091A9
:106110004B19B0914C198093470890934808A0936D
:106120004908B0934A0820E030E046E153E4C30157
:10613000B2010F94152A20E030E04CE352E40F94B2
:10614000142A60933F08709340088093410890930D
:106150004208A30192010F94142A2B013C012FE65F
:1061600032E143E85AEB0F943B2C87FF02C00C94BA
:10617000283F21E230E04BE953E4C301B2010F9420
:106180007B23181614F40C94283FA5019401C70131
:10619000B6010F94142A6B017C012FE632E143E82B
:1061A0005AEB0F943B2C87FF02C00C94283F21E24E
:1061B00030E04BE953E4C701B6010F947B23181676
:1061C00014F40C94283F19821A821B821C829E01AF
:1061D0002F5F3F4F49E459E163E478E08FE398E0B3
:1061E0000E94BA4182E090E00E94AE620E94B444F4
:1061F0008091D911809315100E94BA4583E0809355
:1062000035020E94575B81E00E943D411AC80E94FE
:106210006A5217C8C0904119D0904219E0904319B2
:10622000F090441988E50E949D45811109C020E045
:1062300030E04CE352E4C701B6010F94152A02C0C6
:106240000E943B4568A379A38AA39BA3C0904519EC
:10625000D0904619E0904719F090481989E50E94BE
:106260009D45811108C020E030E0A901C701B601B9
:106270000F94152A02C00E943B456B017C01698383
:106280007A838B839C83209174163091751640918C
:1062900076165091771668A179A18AA19BA10F94D7
:1062A000142A4B015C012AEF3EEF4BE352E40F94BA
:1062B0003B2C87FF02C00C94212921E230E04BE9FE
:1062C00053E4C501B4010F947B23181614F40C9405
:1062D0002129209178163091791640917A165091A3
:1062E0007B16C701B6010F94142A6B017C012FE6BF
:1062F00032E143E85AEB0F943B2C87FF02C00C9429
:10630000212921E230E04BE953E4C701B6010F94A3
:106310007B23181614F40C9421290C94463F81E039
:106320008093BD050C94212985E40E949D45B82EDB
:10633000811102C00E94717FA1EB8A2EA2E09A2EE9
:10634000B1E4CB2EB9E1DB2E13E3E12E18E0F12E00
:1063500000E010E0A12C33243394D4018D914D0141
:106360000E949D45882359F1F6014080518062804A
:1063700073800E943B45D6016D937D938D939C93D2
:1063800013970330E1F0023011F430921810A3019A
:1063900092010F94142A9B01AC01F7016081718175
:1063A000828193810F94152AD7016D937D938D93EC
:1063B0009C931397C8010E94AD43AA24A3940F5F36
:1063C0001F4FB4E0CB0ED11CE4E0EE0EF11C043004
:1063D000110519F6AA2019F00E94B44403C0B110A7
:1063E0000E94A6F10E94575B0C94212980910B0218
:1063F000882311F40C94212989E40E949D45182FCB
:10640000882321F00E940B45062F01C000E08AE49A
:106410000E949D45E82E882321F00E940B45F62E10
:1064200001C0F12C112311F0053028F4EE2089F081
:10643000F4E0FF1570F4E8ECF3E084918F010F5F56
:106440001F4F882311F40C9421290E94F245F80172
:10645000F4CF0E943E43112339F12091D5113091A0
:10646000D6110203B001039F700D11248091D11148
:106470009091D211680F791F072E000C880B990B91
:106480000F948123209174163091751640917616E1
:10649000509177160F94152A60933F087093400827
:1064A0008093410890934208EE2041F12091D7114A
:1064B0003091D8114F2D4203B001439F700D11242C
:1064C0008091D3119091D411680F791F072E000C81
:1064D000880B990B0F9481232091781630917916AF
:1064E00040917A1650917B160F94152A60934308B9
:1064F00070934408809345089093460880E50E9475
:106500006E458823E1F00E942C458823C1F01123B9
:10651000B1F020E030E04CE352E460913F0870912C
:10652000400880914108909142080F94142A60938A
:106530003F0870934008809341089093420886E496
:106540000E949D458823D9F00E943B456B017C0148
:1065500020E030E0A9010F943B2C181684F420E0D1
:1065600030E040E752E4C701B6010F94F12A60938E
:106570008C0270938D0280938E0290938F020F9401
:1065800007070C9421298091BE059091BF0586379D
:10659000910509F455C70CF0E3C08D34910509F459
:1065A00091C40CF056C08931910509F4DBC21CF589
:1065B0008431910509F4CAC17CF48131910509F453
:1065C00050C22CF4029708F4C4C10C9421294297BC
:1065D00009F45EC60C9421298631910509F499C20B
:1065E0000CF491C28731910509F499C2489709F4D6
:1065F000ACC20C9421298F31910509F469C394F43C
:106600008B31910509F4D3C20CF4B2C28C319105DF
:1066100009F40AC34E9711F00C9421290E94545892
:106620000C9421298A32910509F408C42CF480972E
:1066300009F404C30C9421298B34910509F43EC458
:106640008C34910511F00C9421290E948DF10C9449
:1066500021298B36910509F400C60CF054C085350C
:10666000910509F448C68CF58235910509F407C6F1
:1066700014F58135910511F00C9421290E94A7C2CF
:106680000E94717F0F94F70610926E1B10926D1B83
:106690000E94A6F210921C1210921B1268EE73E078
:1066A00080E090E00E940EB160E081E095E00E9401
:1066B000CFB30C9421298335910509F4E4C58435C1
:1066C000910509F4E5C50C9421298836910509F452
:1066D000FDC37CF48C35910511F00C94212961EBFC
:1066E000C62E62E0D62E71E5E72E79E1F72E10E096
:1066F0001DC68936910509F444C58A36910509F409
:106700008DC50C9421298037910509F4E7C484F4E0
:106710008D36910509F47AC50CF4DCC48E369105EA
:1067200009F420C48F36910509F42FC40C94212953
:106730008237910509F47AC60CF4D8C483379105E1
:1067400009F47AC68537910511F00C94212960E08F
:106750008091B6059091B7050E94ECB30C94212965
:106760008D3251E0950711F40C94933D0CF06DC0FF
:106770008B3C910509F495C7A4F58139910509F47D
:10678000A7C684F48837910509F495C60CF48FC622
:106790008937910509F496C68C38910509F4D3C45C
:1067A0000C9421298E3B910509F434C534F48B39BE
:1067B000910509F402C50C942129883C910509F43E
:1067C00003C7893C910511F00C942129B1EBEB2E04
:1067D000B2E0FB2E0AED11E18AEEC82E81E1D82E3F
:1067E00047C78C3D910511F40C94643CA4F48D3C96
:1067F000910509F4DEC70CF470C78E3C910511F4C5
:106800000C94463C833D910511F00C9421290E9483
:1068100011620C942129823E910511F40C948F3C55
:106820003CF48D3D910511F40C94733C0C9421299A
:106830008831B1E09B0711F40C94BE3C8C3291403E
:1068400011F40C946B3D0C942129853AF1E09F07DB
:1068500011F40C946F3EB4F5803931E0930711F4D4
:106860000C94633EC4F48F3251E0950711F40C94FC
:106870005F3E14F40C940E3E8033B1E09B0711F49C
:106880000C94973D8336914011F00C942129E0EE51
:10689000F2E20C94B73E8239F1E09F0711F40C94B8
:1068A0006B3E14F40C94673E8A3931E0930709F487
:1068B00019C4843A914011F00C9421290E94F45992
:1068C0000C942129873F51E0950711F40C947B3EED
:1068D000FCF4843FB1E09B0711F40C94733E4CF43C
:1068E0008C3A914011F00C9421290E94165C0C9472
:1068F0002129853F21E0920711F40C94773E863FD1
:10690000914011F00C9421290E94599E0C94212948
:10691000833543E09407B1F04CF48835924011F090
:106920000C9421290E942E710C942129803AB3E005
:106930009B0709F4C0C1873E934011F40C94CA3EF2
:106940000C942129EBEEFCE40C948A3EE1E3F4E0A4
:106950009AC0A090B605B090B70580E50E949D450D
:10696000882359F00E94FB446B017C0111E0672BE6
:10697000682B692B31F410E004C010E0C12CD12C3D
:10698000760183E50E949D458823F1F00E943B45F6
:1069900020E030E04AE754E40F94E0230F945E2BAC
:1069A0006B017C01111112C0672B682B692B71F4EC
:1069B000A114B10459F0D5018C91882339F061E01C
:1069C000C5010E94ECB307C0112391F360E086E09B
:1069D00094E00E94CFB383E090E0909346068093CA
:1069E000450681E080931A120E94717F0E94AF4594
:1069F000C114D104E104F104E1F080912A109091D6
:106A00002B10A0912C10B0912D10C80ED91EEA1E8B
:106A1000FB1E0E947EF7DC01CB018C199D09AE099B
:106A2000BF09B7FF1AC080911A1281110C94973FC9
:106A300014C080911A12882321F080E00E947C67A4
:106A4000F8CF8091C11360E0882319F087EF93E0BD
:106A500002C087EE93E00E94CFB310921A120C94FA
:106A6000212960E089E194E00E94CFB35F988A9881
:106A70009FB7F894809108018E7F809308019FBF93
:106A800012980C94212984918F010F5F1F4F882346
:106A900021F00E94F245F801F6CF1092661610928E
:106AA000651682EF93E10E94DBCF8BE1E2EFF3E129
:106AB000DE01159601900D928A95E1F78091F01311
:106AC0009091F1139C838B8385EC92E09A83898368
:106AD00040E050E0BE016F5F7F4F84E294E00E948F
:106AE000888ACE0101960E943B64E2E2F4E0849140
:106AF0008F010F5F1F4F882311F40C9421290E94EE
:106B0000F245F801F4CF0E940A890E9443640C9474
:106B100021291092C1131092C2130C942129E091E3
:106B2000B605F091B7058081882329F0803209F4F9
:106B300010823196F8CF40E061E08091B6059091E7
:106B4000B7050E94918C0C9421290E94A6F2809195
:106B5000C213882319F081E08093C1130E9467F269
:106B60000C9421291092C1130E948DF10C942129BB
:106B70008091C213882311F40C94212983E50E948B
:106B80009D45882311F40C9421290E940B45AB01EB
:106B9000BC0140935C1650935D1660935E16709333
:106BA0005F168CE895E10E94FFFE0C9421298091EC
:106BB000C213811103C0E4E5F4E02AC0E2E4F4E08A
:106BC00084918F010F5F1F4F882321F00E94F245AF
:106BD000F801F6CF60915C1670915D1680915E169B
:106BE00090915F164AE00E94B4468FE20E94F245FF
:106BF000609158167091591680915A1690915B16B3
:106C00004AE00E94B4468AE00E94F2450C94212991
:106C100084918F010F5F1F4F882311F40C94212959
:106C20000E94F245F801F4CF40E060E08091B605A3
:106C30009091B7050E94918C0C9421298091C113E9
:106C400081110E94717FE090B605F090B70580E554
:106C50000E946E45182F882319F00E942C45182F8A
:106C60008091C213882311F40C942129412F61E0F3
:106C7000C7010E94918C83E50E949D45882381F085
:106C80000E940B45AB01BC0140935C1650935D160E
:106C900060935E1670935F168CE895E10E94FFFE8C
:106CA0008091C213882319F081E08093C1131111E0
:106CB0000C94212953CF8091B6059091B70521E01E
:106CC0002093C01340E060E00E94918C0C94212935
:106CD0000E94528A7B018C0120E831E541E050E0BE
:106CE0000F94B729C9016DE671E00F94EE2C4B01AA
:106CF0005C01C801B70120E13EE040E050E00F94A4
:106D0000B729CA01B90128E130E040E050E00F9412
:106D1000B729762E672EC62ED72EFCE32F2E312CC8
:106D2000412C512CC801B701A20191010F94B72940
:106D3000F62EE72ECA01B901A20191010F94B729DD
:106D4000CB018E010F5F1F4F8114910499F0EF92D8
:106D5000FF927F936F936F927F92BF92AF929F92B9
:106D60008F928DE894E09F938F931F930F930F94CE
:106D7000152313C0A114B104B1F0EF92FF927F93D9
:106D80006F936F927F92BF92AF928DE794E09F9343
:106D90008F931F930F930F9415230FB6F894DEBFB4
:106DA0000FBECDBF30C0CD2879F0EF92FF927F9318
:106DB0006F936F927F9281E794E09F938F931F93DD
:106DC0000F930F941523E9CF892B69F0EF92FF926F
:106DD0007F936F9389E694E09F938F931F930F9314
:106DE0000F941523DACFEF92FF9285E694E09F93FC
:106DF0008F931F930F930F9415230F900F900F9065
:106E00000F900F900F9060E0C8010E94ECB3EBEE82
:106E1000FCE484917F019FEFE91AF90A882321F0AD
:106E20000E94F245F701F5CFB80181EA94E00F9492
:106E3000200D8AE00E94F2450C94212983E50E94EE
:106E40009D45882311F40C9421290E941B45E82EAE
:106E500080E50E949D45882311F40C9421290E940D
:106E60000B45162FC62ED72ED7FE02C00C94212913
:106E7000E7EBF5E08491181303C0E0EEF2E20AC0FC
:106E80003196A5E0EF3DFA07A9F70C949C3F0E94CC
:106E9000F245F80184918F010F5F1F4F8111F7CFE9
:106EA000EEEAF4E084918F010F5F1F4F882311F405
:106EB0000C9421290E94F245F801F4CF0E9467F258
:106EC0000C9421290E94B1E80C94212988E690E0D5
:106ED0000E941F4781110C9421298091471283FF42
:106EE00002C00C94212983E50E949D458823B1F1BD
:106EF0000E943B450F94592BCB010E943BB30E944B
:106F00003B4520E030E04AEA52E40F947B23181618
:106F10003CF00E94B1E860E089EC94E00E94CFB3BD
:106F20000E943B4520912112309122124091231260
:106F3000509124120F943B2C181684F483E393E0B1
:106F40009F938F938DEB94E09F938F931F920E945A
:106F500067EB0F900F900F900F900F900F94CB0D49
:106F60000C9421298EE40E949D45882311F40C94F1
:106F700021290E940B456093051B7093061B80938B
:106F8000071B9093081B0C94212983E50E946E45F2
:106F9000882359F083E50E949D45882319F00E94BB
:106FA0001B4501C080E080934712EBEEFCE4849126
:106FB0008F010F5F1F4F811103C0E7EEF4E004C0A3
:106FC0000E94F245F801F3CF84918F010F5F1F4FAC
:106FD000882321F00E94F245F801F6CF80914712F4
:106FE000811103C0E3EEF4E034C0E9EDCE2EE4E01D
:106FF000DE2EE12CF12C20E08091471290E00E2C47
:1070000002C0959587950A94E2F780FF17C0BB24CC
:10701000B394B20E222319F08CE20E94F245F601DD
:1070200085919491FC0184918F010F5F1F4F8823FC
:1070300021F00E94F245F801F6CF2B2DBFEFEB1A9D
:10704000FB0AE2E0CE0ED11CF5E0EF16F104A1F64A
:107050003CC084918F010F5F1F4F8823B1F10E94C4
:10706000F245F801F6CF8AE50E946E45882309F4BF
:107070006FC60E943B456B017C0120E030E040EA96
:1070800051EC0F943B2C87FD57C620E030E040EADE
:1070900051E4C701B6010F947B2318160CF44CC6BB
:1070A000C092E416D092E516E092E616F092E7164A
:1070B0000E94D5F26091E4167091E5168091E61673
:1070C0009091E71642E00E94A04A8AE00E94F245B1
:1070D0000C942129109294020C9421298EEE94E0B4
:1070E0000E9411670E949E5A0C94212983E50E94F8
:1070F0009D45811103C0EBEEFCE40DC00E941B45D1
:10710000809300028D3310F40C9421298CE380933A
:1071100000020C94212984918F010F5F1F4F882357
:1071200021F00E94F245F801F6CF4091000250E0B4
:1071300060E070E087EF94E00F94CD0C8AE00E944D
:10714000F2450C9421298091471283FF02C00C94D0
:10715000212983E50E949D45882311F40C9421295F
:107160000E943B450F94592B6E37710514F06DE763
:1071700070E070936C1B60936B1B0E945BC20C945D
:10718000212989E690E00E941F47811111C0EEEF8E
:10719000F4E084918F010F5F1F4F882321F00E943C
:1071A000F245F801F6CF0E94154C8AE00E94F245A4
:1071B000109246061092450629C783E50E949D4518
:1071C000882311F40C9421290E941B4580934B06BF
:1071D0008D3318F08CE380934B060E947EF76B0191
:1071E0007C0120914B0630E0A8EEB3E00F94052A15
:1071F000C60ED71EE81EF91EC0924706D09248065A
:10720000E0924906F0924A060C9421290E94314EE0
:107210000C9421290E94944C0C94212983E50E940E
:107220009D45882339F00E940B458B016F3F710506
:1072300019F010F00FEF10E080E50E949D458111DC
:1072400006C010936E1B00936D1B0C9421290E94A5
:107250001B4581110C942129F4CF80E50E949D45A6
:10726000811106C010926E1B10926D1B0C94212987
:107270000E940B45672B11F00C942129F3CF10923B
:10728000BC050C94212981E08093BC050C94212934
:1072900083E50E949D458823A1F00E943B4520E0A4
:1072A00030E04AE754E40F94E0230F945E2B6093A0
:1072B00001027093020280930302909304020C94E3
:1072C000212988E50E946E4581114FC689E50E94FB
:1072D0006E4581114AC68AE50E946E45811145C6F8
:1072E00085E40E946E45811140C60E94717F0F9413
:1072F000F7060C94212983E50E946E45882311F43A
:107300000C9421290E943B4520E030E04AE754E4F8
:107310000F94E0230F945E2B60934F0670935006FA
:1073200080935106909352060C942129D6018D9199
:107330006D010E946E45882309F46DC0133009F079
:1073400063C00E943B454B015C0120E030E040EA15
:1073500051E40F947B2387FF4EC0A50194016091F7
:107360005D1970915E1980915F19909160190F9469
:10737000F12A2B013C019B01AC016091021270913A
:10738000031280910412909105120F94E0236093F0
:107390000212709303128093041290930512A301BA
:1073A000920160919B1270919C1280919D1290911C
:1073B0009E120F94E02360939B1270939C12809313
:1073C0009D1290939E126091511B7091521B80915F
:1073D000531B9091541B0F947F23A30192010F9490
:1073E000E0230F945E2B6093511B7093521B80938C
:1073F000531B9093541B80925D1990925E19A0923A
:107400005F19B092601907C00E943B45F701608385
:107410007183828393831F5FF4E0EF0EF11C1430BD
:1074200009F084CF0F94190F0C9421290E94717FC9
:107430000E94575B0C9421290E94CE5A0C9421295A
:1074400085E40E946E45882381F00E942C458823A4
:1074500061F0EBEEFCE484918F010F5F1F4F8823F6
:1074600021F00E94F245F801F6CF81E40E946E45BA
:10747000882381F00E942C45882361F0EFE0F5E03D
:1074800084918F010F5F1F4F882321F00E94F245E6
:10749000F801F6CF0091B6051091B705D8018D918E
:1074A0008D01882309F411CE0E94F245F7CF0E9486
:1074B000896C0C94212981E0809315108093D91157
:1074C0000C942129109215101092D9110C94212995
:1074D00083E50E949D45882319F00E940B4502C058
:1074E00060E070E07B01FF24B2E0EB16F104DCF019
:1074F000E0EEF2E284918F010F5F1F4F811103C014
:10750000E3E1F5E004C00E94F245F801F3CF849175
:107510008F010F5F1F4F882311F40C9421290E94C3
:10752000F245F801F4CF88E40E949D458823A9F034
:107530000E940B456A3A71053CF06530E1E07E0738
:107540002CF064E071E002C06AEA70E0F701EE0F2F
:10755000FF1FE158FD4E7183608386E40E949D45C4
:107560008823A9F00E940B45F701EE0FFF1FED578E
:10757000FD4E718360836F3F710519F014F06FEF5A
:1075800070E077FF02C060E070E07183608382E4A6
:107590000E949D45882311F40C9421290E940B45DB
:1075A0006530710534F06F3671052CF06EE670E0D1
:1075B00002C065E070E0F701EE0FFF1FE558FD4ED9
:1075C000718360830C94212988EC90E00E941F470E
:1075D00081110C94212984E40E946E45882309F4CA
:1075E00043C00E943B456B017C0111E020E030E08C
:1075F000A9010F947B23811101C010E010930910A1
:1076000020E030E0A901C701B6010F947B23882355
:1076100059F10091B80510E00E943B45000F111F81
:10762000000F111FF801EB5FFF4E608371838283AF
:10763000938320E030E0A90160910510709106105D
:1076400080910710909108100F947B2381110CC03A
:1076500080E090E0A0EEBFE38093051090930610C9
:10766000A0930710B09308100F94F6030C942129EF
:10767000D7018D917D010E946E45882349F00E94BB
:107680003B450F945E2BF801608371838283938363
:107690000C5F1F4FC016D10659F70F94FB0D0C94C9
:1076A0002129A1EBEA2EA2E0FA2E0FE812E1D70180
:1076B0008D917D010E946E45882339F00E943B45E3
:1076C000F80160837183828393830C5F1F4FF2E123
:1076D0000F391F0761F70C94212983E50E946E453D
:1076E0008823D9F00E943B45AB01BC014093F211C5
:1076F0005093F3116093F4117093F5114093EA11D4
:107700005093EB116093EC117093ED118FE895E0BD
:107710000F94EA0C8AE00E94F24580E50E946E45D3
:10772000882399F00E943B45AB01BC014093F211C4
:107730005093F3116093F4117093F51182E795E083
:107740000F94EA0C8AE00E94F24582E50E946E45A1
:10775000882399F00E943B45AB01BC014093EE1198
:107760005093EF116093F0117093F11183E595E060
:107770000F94EA0C8AE00E94F24584E50E946E456F
:10778000882311F40C9421290E943B45AB01BC01D4
:107790004093EA115093EB116093EC117093ED114B
:1077A00085E395E00F94EA0C8AE00E94F2450C9480
:1077B000212983E50E946E45882351F00E943B45B4
:1077C00060938B1270938C1280938D1290938E1213
:1077D00084E50E946E45882351F00E943B456093EA
:1077E0008712709388128093891290938A1282E490
:1077F0000E946E45882351F00E94FB446093AC12B6
:107800007093AD128093AE129093AF1288E50E94F0
:107810006E45882351F00E943B456093F6117093AA
:10782000F7118093F8119093F91189E50E946E4544
:10783000882351F00E943B456093FA117093FB112D
:107840008093FC119093FD118AE50E946E45882378
:1078500051F00E943B456093FE117093FF1180939D
:1078600000129093011285E40E946E45882311F462
:107870000C9421290E943B456093021270930312DD
:1078800080930412909305120C942129F1EBEF2EB2
:10789000F2E0FF2E00E010E0D7018D917D010E9403
:1078A0006E45882331F00E943B45AB01BC01C80105
:1078B000AAD70F5F1F4F0330110571F70E94B44420
:1078C0000E94575B0C94212983E50E949D458823E3
:1078D00011F40C9421290E940B4570931C026093B3
:1078E0001B020C9421298DED90E00E941F4781110D
:1078F0000C94212983E50E949D45882311F40C9462
:1079000021290091B80510E00E940B45000F111FBE
:10791000F801E75EFD4F718360830C94212980E5B7
:107920000E946E45882311F40C9421290E940B4576
:10793000F62EC62ED72E83E50E949D45882321F082
:107940000E940B458B0102C00FEF1FEFC80101968B
:10795000039710F00C942129D7FE02C00C94212922
:10796000E7EBF5E08FED95E02491F21611F40C941D
:10797000212931968E179F07B9F71FC380E50E9412
:107980006E45882311F40C9421290E940B456B014C
:107990007C015B01672B19F000EE12E281C083E5E8
:1079A0000E946E45811103C0EBEEFCE408C00E940A
:1079B0000B4580E993E10F94990B0C942129849154
:1079C0008F010F5F1F4F882321F00E94F245F801BD
:1079D000F6CF60E070E088EF95E00F94070D80919E
:1079E000921328E532E06901C81AD10887FDD394C3
:1079F000CC0CDD1CCC0CDD1C0D2C000CEE08FF08A3
:107A00008091911328E830E02901481A510887FD38
:107A10005394440C551C440C551C052C000C660852
:107A20007708809190138F3FC1F090E0FC01EE0F3A
:107A3000FF1F8E0F9F1FFC01ED5DFC4EA180B280E9
:107A400033E0AA0CBB1C3A95E1F744E0B694A79446
:107A50004A95E1F7B2E0AB0EB11C95012F5F3F4FA5
:107A6000C901330FAA0BBB0B9C01AD0124193509C9
:107A700046095709A4EBB0E00F94F529A701960138
:107A800024193509460957090F94D929B90185EFF9
:107A900095E00F94070D8AE00E94F2450C9421298D
:107AA000F8018491882329F00F5F1F4F0E94F2454F
:107AB000F7CFB6018EEE95E00F94070D0FED15E0B0
:107AC000F8018491882311F40C9421290F5F1F4F32
:107AD0000E94F245F5CF83E50E949D45882311F071
:107AE0009AD702C064E071E079A368A380E50E94A0
:107AF0009D45882331F08FD76938F3E17F0730F453
:107B000002C068EE73E07A83698304C088E893E179
:107B10009A838983BE01605E7F4FCE0101960E94E9
:107B200059F10C9421290E9473610C94212980E55C
:107B3000D5D7882349F09FD760938B0D70938C0D18
:107B400080938D0D90938E0D89E4C8D7882379F0AA
:107B500092D72CEA35EC47E25EE30F94E023609382
:107B6000870D7093880D8093890D90938A0D84E41E
:107B7000B5D7882379F07FD72CEA35EC47E25EE36E
:107B80000F94F12A6093830D7093840D8093850D7B
:107B90009093860DEBEEFCE484918F010F5F1F4FF5
:107BA000882321F00E94F245F801F6CF40918B0D19
:107BB00050918C0D60918D0D70918E0D88E096E046
:107BC0000F94EA0C2CEA35EC47E25EE36091870DF6
:107BD0007091880D8091890D90918A0D0F94F12AF2
:107BE000AB01BC0184E096E00F94EA0C2CEA35EC82
:107BF00047E25EE36091830D7091840D8091850D65
:107C00009091860D0F94E023AB01BC0180E096E0DB
:107C10000F94EA0C8AE0E6D70C94212983E55ED71D
:107C2000182F882369F027D70F94592B70931802C7
:107C30006093170221E0672B09F020E020932512C2
:107C400080E54CD7882359F0209117023091180213
:107C5000232B09F001D7809325120C9421291111AF
:107C60000C942129EBEEFCE484918F010F5F1F4FF0
:107C7000882319F0B7D7F801F7CF80912512882310
:107C800019F063E674E002C06FE273E081E296E00F
:107C90000F94200D609117027091180280E196E018
:107CA0000F94070DECE0F6E084918F010F5F1F4FFA
:107CB000882311F40C94212995D7F801F5CF0E945F
:107CC000245D0C9421290E94717F0C94212981E06C
:107CD00049D40C94212980E045D40C9421290E9498
:107CE00058590C9421290E94BFA40C9421290E9468
:107CF000A29F0C94212983E5F1D6882311F0ACD6FC
:107D000001C081E091E089270E94EB6C0C9421294D
:107D100069D7F80184918F010F5F1F4F8111F8CF50
:107D2000EEE4F6E084918F010F5F1F4F882309F482
:107D30009AC958D7F801F6CFE7E3F6E084918F01AE
:107D40000F5F1F4F882309F4C0C94CD7F801F6CF45
:107D50004091E4165091E5166091E6167091E71691
:107D600084E396E00F94EA0CB0C93CD7F801849103
:107D70008F010F5F1F4F8111F8CFE8E5F6E0849186
:107D80008F010F5F1F4F882311F40C9421292AD7EC
:107D9000F801F5CF81E080930B021092BC1283E5CD
:107DA0009DD6811104C00F94610A0C94212954D6E8
:107DB00081110C942129F7CFF090BE05FF20F9F036
:107DC000EBEEFCE484918F010F5F1F4F882319F0C5
:107DD00009D7F801F7CF84E505D76F2D70E080E073
:107DE00090E04AE0C1D780E2FDD60EE313E0D8016F
:107DF0008D918D01882309F468C9F4D6F8CF1092CB
:107E00006C08EBEEFCE484918F010F5F1F4F882319
:107E100019F0E8D6F801F7CF60916C0870E087E6BA
:107E200096E00F94070D8AE0DDD60C94212940914D
:107E3000B6055091B705452B39F4AF0141505109B2
:107E40005093B7054093B60540E050E00C94AE293E
:107E500060E084E893E00E94CFB3EBEEFCE4849111
:107E60008F010F5F1F4F811103C0E2E7F3E003C0F2
:107E7000B9D6F801F4CF84918F010F5F1F4F88238B
:107E800011F40C94F630AED6F801F5CF80E0F5D1C0
:107E90008AD683E523D6882309F447C0DDD521E0BF
:107EA000482FBE016F5F7F4FCE0180960E9440F346
:107EB0006B017C019B01AC010F94C32C811130C07C
:107EC0002CEA35EC47E257E368A179A18AA19BA18E
:107ED0000F94152AAB01BC0180EC93E00F94EA0CDF
:107EE0002CEA35EC47E257E369817A818B819C81EA
:107EF0000F94152AAB01BC018BEB93E00F94EA0CB5
:107F00002CEA35EC47E257E3C701B6010F94152A76
:107F1000AB01BC0186EB93E00F94EA0C8AE062D6D9
:107F200029D60E94575B0C94212981E0B8CF80E0CC
:107F30000E947C670C94093561E0812F0E9442F613
:107F40006E2D812F0E942A9EF12CB701812F0E9455
:107F50007EF6B9E0CB16D10411F00C942129F092F1
:107F60006E1BE0926D1B0C9421290E94717F88E5A5
:107F7000B5D5882319F05F9A1092161089E5AED511
:107F8000882319F08A9A109217108AE5A7D58823BA
:107F900051F09FB7F89480910801816080930801A7
:107FA0009FBF1092181085E499D5882311F40C9482
:107FB00021290F94F5060C9421290E94717F60E01D
:107FC0008F2D0E9442F60F3FEFEF1E0759F48F2DC1
:107FD0000E94019E31E020E0892B09F030E0032F60
:107FE000122F05C00130110571F401E010E08F2D52
:107FF0000E94019E8017910711F40C94212980E0C2
:108000000E947C67F4CF00E010E0F1CFC15ADF4F4F
:108010000FB6F894DEBF0FBECDBFDF91CF911F9199
:108020000F91FF90EF90DF90CF90BF90AF909F9017
:108030008F907F906F905F904F903F902F9008951A
:1080400090912E10E92FF0E0EA5DFF4E80839F5F54
:10805000943018F490932E1002C010922E1080913C
:10806000CF118F5F8093CF110895089580E090E045
:1080700008958FB7F8949091041B2091031B9217D9
:1080800059F0E92FF0E0ED57F54E208130E09F5F89
:108090009F779093041B02C02FEF3FEF8FBFC90162
:1080A0000895CF92EF92FF920F931F93CF93DF9398
:1080B000CDB7DEB72C970FB6F894DEBF0FBECDBF9D
:1080C000C0906C08E1E4F9E180859185A285B385D3
:1080D00044815581668177810081118122813381BC
:1080E00009831A832B833C834D835E836F83788758
:1080F00089879A87AB87BC87AE01475F5F4FBE0118
:108100006B5F7F4FCE0101960E940EE2E0908C02E1
:10811000F0908D0200918E0210918F022DE439E1D2
:10812000AE01475F5F4FBE016B5F7F4FCE0101968F
:108130000E94F1D42C960FB6F894DEBF0FBECDBFCF
:10814000DF91CF911F910F91FF90EF90CF90089505
:108150000F931F93CF93DF93EC010E947EF70E8164
:108160001F8128853985011511052105310559F52E
:108170002C852223A9F13A8521502C8721E0230F59
:108180002A874D85241301C01A86FE0124E0329F00
:10819000E00DF11D112406851785208931890A8398
:1081A0001B832C833D83DC01CB01800F911FA11D1C
:1081B000B11D8E839F83A887B9878C819D81892B70
:1081C00079F0409A0DC0DC01CB01801B910BA20B12
:1081D000B30BB7FD05C040981E821F821886198612
:1081E000DF91CF911F910F910895CF92DF92EF927F
:1081F000FF92CF936B017C01C091AB126093A712E9
:108200007093A8128093A9129093AA122DEB37E3D2
:1082100046E855EB0F943B2C87FD0AC02DEB37E366
:1082200046E855E3C701B6010F947B2318164CF4BA
:10823000A701960160E070E080E89FE30F94F12AC7
:1082400003C060E070E0CB016093A3127093A412AE
:108250008093A5129093A612CC2349F082E090E07F
:10826000CF91FF90EF90DF90CF900D94F107CF91D9
:10827000FF90EF90DF90CF9008951F93CF93DF93FF
:10828000CDB7DEB72C970FB6F894DEBF0FBECDBFCB
:10829000882331F02091D5113091D611232BF9F09C
:1082A0009091AB128917D9F0182F8CE0E5EBF2E032
:1082B000DE01119601900D928A95E1F7CE010196AB
:1082C0000F943D081093AB12111105C082E090E0AD
:1082D0000F94F10704C081E499E10E948FE12C968C
:1082E0000FB6F894DEBF0FBECDBFDF91CF911F91C7
:1082F0000895CF92DF92EF92FF9280E0BEDF10925E
:10830000D8111092D7111092D6111092D511109247
:10831000D4111092D3111092D2111092D11140E8C1
:1083200056E125E0C12CD12C80ECE82E8FE7F82E09
:1083300080E090E0FA01E80FF91FC082D182E2826A
:10834000F382049684319105A9F721504C5E5F4F6A
:108350002111EECFFF90EF90DF90CF900895BC01F8
:1083600080E993E10F94990B67E771E080E090E07A
:108370000C940EB14F925F926F927F928F929F9268
:10838000AF92BF92CF92DF92EF92FF920F931F9323
:10839000CF93DF935C014B018A01E90140908C028D
:1083A00050908D0260908E0270908F02FA012081B1
:1083B0003181428153816091491970914A198091AC
:1083C0004B1990914C190F947B2387FF2DC0C880C7
:1083D000D980EA80FB8020E030E0A901B601C70126
:1083E0000F947B23811108C0E1E8FFE0859195910E
:1083F000A591B4916C017D01C601D70180938C02D7
:1084000090938D02A0938E02B0938F02F801808129
:108410009181A281B3818093491990934A19A093C5
:108420004B19B0934C193DDEC880D980EA80FB809F
:1084300020E030E0A901C701B6010F947B23811130
:1084400008C0C0908702D0908802E0908902F09026
:108450008A02C0928C02D0928D02E0928E02F0923B
:108460008F02F50180819181A281B38180934119AE
:1084700090934219A0934319B0934419F401808159
:108480009181A281B3818093451990934619A0935D
:108490004719B093481905DEF801208131814281E6
:1084A00053816091491970914A1980914B199091AB
:1084B0004C190F943B2C18169CF5D880E980FA8053
:1084C000CB8120E030E0A9016D2D7E2D8F2D9C2FDA
:1084D0000F947B2381110AC0E1E8FFE0859195911B
:1084E000A591B491D82EE92EFA2ECB2F8D2D9E2D4D
:1084F000AF2DBC2F80938C0290938D02A0938E029F
:10850000B0938F02F80180819181A281B381809321
:10851000491990934A19A0934B19B0934C19C1DD96
:108520000E94717F40928C0250928D0260928E0266
:1085300070928F02DF91CF911F910F91FF90EF907A
:10854000DF90CF90BF90AF909F908F907F906F9073
:108550005F904F9008959B01AC0165E479E181E45F
:1085600099E108CFCF92DF92EF92FF921F93CF93C2
:10857000DF93CDB7DEB72C970FB6F894DEBF0FBEF2
:10858000CDBF90911910981709F469C0182F80E099
:1085900090E0A0E2B1E48D839E83AF83B887C09062
:1085A000E416D090E516E090E616F090E71620E08D
:1085B00030E0A901C701B6010F947B2387FF0CC0EF
:1085C000A701960160E070E080E291E40F94142A24
:1085D0006D837E838F8398872D813E814F8158855F
:1085E0006091491970914A1980914B1990914C19D9
:1085F0000F947B2387FF0AC019821A821B821C8278
:10860000BE016F5F7F4FCE010596A5DF80914119B6
:1086100090914219A0914319B091441989879A8782
:10862000AB87BC878091451990914619A091471955
:10863000B09148198D839E83AF83B88719821A82BF
:108640001B821C829E012F5F3F4F49E459E1BE010E
:108650006B5F7F4FCE0109968DDE1093191080E07D
:108660002C960FB6F894DEBF0FBECDBFDF91CF9131
:108670001F91FF90EF90DF90CF90089580E1E1E4AB
:10868000F9E1AFE3B8E001900D928A95E1F7089522
:1086900080E1EFE3F8E0A1E4B9E101900D928A9561
:1086A000E1F708958F929F92AF92BF92CF92EF928F
:1086B000FF920F931F93CF93DF93CDB7DEB72C9725
:1086C0000FB6F894DEBF0FBECDBF4B015C01C0906A
:1086D0006C08EFE3F8E080859185A285B38544813D
:1086E00055816681778100811181228133810983DF
:1086F0001A832B833C834D835E836F8378878987BE
:108700009A87AB87BC87AE01475F5F4FBE016B5F47
:108710007F4FCE0101960E940EE2850174012BE489
:1087200038E0AE01475F5F4FBE016B5F7F4FCE0108
:1087300001960E94F1D42C960FB6F894DEBF0FBEBE
:10874000CDBFDF91CF911F910F91FF90EF90CF9010
:10875000BF90AF909F908F900895CF92DF92EF924D
:10876000FF920F931F93CF93DF93EC01CC0FDD1F8C
:10877000CC0FDD1FFE01E65EFF4E20E030E0A901D8
:1087800060817181828193810F94152AFE01ED5CD5
:10879000F74F20813181428153810F94152A6B015B
:1087A0007C01FE01EC58F94E6083718382839383D0
:1087B000FE01E95FF74F25913591459154918E0166
:1087C000075C194F0F94152AF80160837183828327
:1087D0009383FE01ED5EF74F2591359145915491BC
:1087E000C75DDD4FC701B6010F94152A68837983F1
:1087F0008A839B83DF91CF911F910F91FF90EF9020
:10880000DF90CF9008958F929F92AF92BF92EF9298
:10881000FF920F931F93CF93DF938C014A015B016B
:10882000EC01CC0FDD1FCC0FDD1FCE018F5B964E10
:108830007C01C65EDF4E288139814A815B81C5019A
:10884000B4010F94142AF7012081318142815381B0
:108850000F94152AF7016083718382839383888242
:108860009982AA82BB82C801DF91CF911F910F919B
:10887000FF90EF90BF90AF909F908F906ECFCF936F
:10888000FC0120812B33A1F02091CF11243080F402
:10889000C62FBC0180912E10F0E68F9FC0011124DD
:1088A000825B9F4E0F947E2D8C2FCADB81E001C02E
:1088B00080E0CF910895DF92EF92FF920F931F9384
:1088C000CF93DF93CDB7DEB76E970FB6F894DEBFC8
:1088D0000FBECDBF6091F60F7091F70F6115710556
:1088E00049F14DE150E0CE0101967C010F94EC225C
:1088F0001E8EF7018F010E191F09D190DD2019F08E
:108900009AE0D912F7CFF701E00FF11F1082C701EB
:108910000E9482EB882371F0DD20A9F00F5F1F4FCA
:108920008091F60F9091F70F080F191F1093F70F12
:108930000093F60F81E02091F60F3091F70F232B73
:1089400029F480E003C000E010E0F0CF6E960FB68F
:10895000F894DEBF0FBECDBFDF91CF911F910F9175
:10896000FF90EF90DF9008950F931F93CF93DF93C5
:10897000CDB7DEB72C970FB6F894DEBF0FBECDBFD4
:10898000E1E4F9E180859185A285B3854481558133
:1089900066817781008111812281338109831A8365
:1089A0002B833C834D835E836F83788789879A8787
:1089B000AB87BC87AE01475F5F4FBE016B5F7F4FE8
:1089C000CE0101960E940EE22DE439E1AE01475F2F
:1089D0005F4FBE016B5F7F4FCE0101960F94560E25
:1089E0002C960FB6F894DEBF0FBECDBFDF91CF91AE
:1089F0001F910F9108958091C1059091C205009734
:108A000031F04AE050E060E070E00D94C22160E097
:108A100070E0CB0108958091C1059091C205009747
:108A200031F04AE050E060E070E00D94952060E0A5
:108A300070E0CB010895EFDF97FD0AC0ECDF6F3FD8
:108A400071058105910509F02CF4E5DF862F089565
:108A500080E008958FEF08958091C1059091C2053F
:108A6000892B31F0E8DF91E0811103C090E001C073
:108A700091E0892F08950F931F93CF938091C105A3
:108A80009091C2050097F1F0FC018F01C1912C2F4C
:108A90002F7D89F0C53411F0C536B9F7F801108281
:108AA00060E070E00F94411FF801C083562F472FFC
:108AB000382F292F0BC060E070E0CF911F910F91EC
:108AC0000D94411F50E040E030E020E0652F742F0E
:108AD000832F922FCF911F910F91089581548A3146
:108AE00050F5482F50E0FA0193E0F595E7959A95F7
:108AF000E1F7EE54FA4F208130E0877002C03595DF
:108B000027958A95E2F7822F817020FF15C0FA0120
:108B1000E856FA4F9081992339F020914D06309113
:108B20004E06290F311D02C020E030E03093C2050F
:108B30002093C105089580E00895D0DF882341F097
:108B400081E02091C1053091C205232B09F480E01A
:108B50000895FC01238121110C947ECE08950E947A
:108B60007EF760932A1070932B1080932C109093B3
:108B70002D1008958091300690913106A091320613
:108B8000B091330680938C0290938D02A0938E0255
:108B9000B0938F0280912E0690912F0690931C0225
:108BA00080931B02DCCF80918C0290918D02A0916A
:108BB0008E02B0918F028093300690933106A0937D
:108BC0003206B093330680911B0290911C02909361
:108BD0002F0680932E0684E690E090931C028093EB
:108BE0001B02BDCF9091C00095FFFCCF8093C600C3
:108BF00008950F931F93CF93C82F882329F04A9984
:108C00000DC08AE090E002C08AE590E0A8DBCC23AA
:108C100019F08CE390E0A3DBC0E052C08CE390E05D
:108C20009EDB8AE090E09BDB8AE590E098DB6CEDD0
:108C300075E080E090E00E940EB14A9BE2CFE0EE4A
:108C4000F2E284918F010F5F1F4F882319F0CADF72
:108C5000F801F7CFE0EAF8E084918F010F5F1F4F32
:108C6000882319F0BFDFF801F7CF0E94A7C2C09197
:108C70000B02CC2321F1E0EEF2E284918F010F5F31
:108C80001F4F882319F0AEDFF801F7CFE9E2F8E0D3
:108C900084918F010F5F1F4F882319F0A3DFF80124
:108CA000F7CF60E08FE198E00E94CFB36EE571E00E
:108CB00080E090E00E940EB110920B0201C0C1E072
:108CC0008C2FCF911F910F910895CF92DF92EF9249
:108CD000FF921F93CF93DF93CDB7DEB728970FB6E0
:108CE000F894DEBF0FBECDBF6D837E838F839887E0
:108CF00069017A0181E07DDF882311F081E026C0DF
:108D000020E030E040E752E4C701B6010F94F12AB9
:108D100069837A838B839C83BE016F5F7F4FCE0113
:108D2000059619DC80914D10182F147082FF04C035
:108D300080E05FDF8111E2CF10924D1082E090E081
:108D40000F94F10711DE81E0111180E028960FB633
:108D5000F894DEBF0FBECDBFDF91CF911F91FF9082
:108D6000EF90DF90CF9008958F929F92AF92BF9235
:108D7000EF92FF920F931F93CF93DF93CDB7DEB7A0
:108D8000A0970FB6F894DEBF0FBECDBF6115710579
:108D90008105910589F100E0842E912CA12CB12C44
:108DA000102FEE24E394F12CEC0EFD1EE00EF11CCE
:108DB00007FDFA94A50194010F94B729F701608388
:108DC000B901CA010F5F611571058105910541F770
:108DD0001F3F21F1E1E0F0E0EC0FFD1FE10FF11D7D
:108DE00017FDFA9580818A3010F097E301C090E377
:108DF000890FF8DE1150ECCF80E3A0960FB6F894FF
:108E0000DEBF0FBECDBFDF91CF911F910F91FF90BD
:108E1000EF90BF90AF909F908F90E4CEA0960FB64A
:108E2000F894DEBF0FBECDBFDF91CF911F910F91A0
:108E3000FF90EF90BF90AF909F908F900895EF922A
:108E4000FF920F931F93CF93DF937C0184E575DE30
:108E5000D82F882321F1EFDDC82F1816E4F4EBEEAC
:108E6000FCE484918F010F5F1F4F882319F0BADE55
:108E7000F801F7CF8DE4B6DEB70180E090E04AE07C
:108E800073DF6C2FCC0F770B84EF97E00F94070DF7
:108E90008AE0A8DE08C08093B805D0E004C08091C5
:108EA0006C088093B8058D2FDF91CF911F910F91A2
:108EB000FF90EF900895CF92DF92EF92FF926B01B7
:108EC0007C0197FF0AC08DE28DDEF094E094D0948F
:108ED000C094C11CD11CE11CF11C4AE0C701B601C1
:108EE000FF90EF90DF90CF903FCFFF920F931F93B3
:108EF000CF93DF93F82E092F162FE0EEF2E2849144
:108F0000EF012196882319F06DDEFE01F8CFEF2DD9
:108F1000F02F8491EF012196882319F063DEFE0182
:108F2000F8CF6091051B7091061B8091071B9091F3
:108F3000081BC1DF8AE056DE11110F94610A1092FE
:108F4000280610922706DF91CF911F910F91FF9075
:108F500008952F923F924F925F926F927F928F92DD
:108F60009F92AF92BF92CF92DF92EF92FF920F93B8
:108F70001F93CF93DF931F92CDB7DEB79CDC811197
:108F8000CBC28091CF11843008F065C072D89C01AB
:108F900097FD61C0982F00912706109128068A300E
:108FA00019F09D3009F021C1109229060115110513
:108FB00041F3F801E953FA4F1082109228061092FB
:108FC000270627EC35E08901F90180812F5F3F4FAB
:108FD0008032C9F38E3409F072C078016AE270E021
:108FE000C8010F946A2D6C01E114F10409F4ADC0BD
:108FF0006CEB77E0C8010F94FB225C01892B09F030
:1090000061C04AE050E060E070E0C70101960F9453
:1090100095206093C3057093C4058093C505909314
:10902000C6054090051B5090061B6090071B709072
:10903000081BFFEF4F1A5F0A6F0A7F0A6415750558
:109040008605970509F449C0AB2809F046C061E0E0
:1090500089E897E04ADF8091C113882309F45CC254
:109060008091CF11811102C010922D0680911B12A8
:1090700090911C12181619060CF0E5C000912A06F2
:1090800010912B0620E6209FC001219F900D1124F6
:109090008D5A994F0E9482EB882309F43DC20F5FDD
:1090A0001F4F10932B0600932A0680911B1290915C
:1090B0001C12019790931C1280931B122DC2E12C5D
:1090C000F12C8CCF6EE470E0C80104960F946A2DE9
:1090D000009709F496CF7C0194CFC114D10401F11B
:1090E00080E0F12CF801E80FF11D90819A3219F01F
:1090F0008F5FF926F7CF4AE050E060E070E0C601EC
:1091000001960F949520CF2CD12CE12CF12C6C15CD
:109110007D058E059F0541F061E08AE697E09ACFD4
:1091200061E080E497E096CF8091C3059091C405FB
:10913000A091C505B091C6058093051B9093061BB1
:10914000A093071BB093081B06C0892B21F060E099
:1091500086E197E07FCF80910B02811122C067E406
:1091600070E0C8010F946A2D0097D9F04AE050E0F2
:1091700060E070E001960F9495206430710588F4EA
:10918000EFE9F6E084917F012FEFE21AF20A8823DB
:1091900019F028DDF701F6CF60E085E996E00E943E
:1091A000CFB36FE473E0C8010F94752D892B21F4C0
:1091B0001092940210921A1264E573E0C8010F94A1
:1091C000752D892B21F48CE896E00E94116769E5E2
:1091D00073E0C8010F94752D892B11F40E949E5ADB
:1091E00061E087EC95E04BDBCCCE0F3511050CF040
:1091F000C8CE9C35A1F40E94394097FDC2CE209183
:1092000029062111BECE98012F5F3F4F30932806CB
:1092100020932706F801E953FA4F8083B2CE9B339F
:1092200019F481E080932906809129068111A9CE45
:10923000C80101969093280680932706F801E95308
:10924000FA4F20839ECEEE24E39440915C16509119
:109250005D1660915E1670915F1680915816909120
:109260005916A0915A16B0915B16481759076A070C
:109270007B0708F4E12C00E010E09924939480E649
:10928000882E95ECA92E97E0B92E21EC622E27E0CE
:10929000722E8091CF11843008F03EC1E1103CC1A4
:1092A00080912D06811138C180919415909195156A
:1092B000A0919615B091971580935C1690935D16CA
:1092C000A0935E16B0935F1641E050E0BE016F5F61
:1092D0007F4F8CE895E10E9406D1019719F48981AE
:1092E00090E002C08FEF9FEFF82E20905C16309038
:1092F0005D1640905E1650905F1640915816509142
:10930000591660915A1670915B16EE24E394241658
:1093100035064606570608F4E12C2416350646069F
:109320005706B0F4019609F4AAC0FAE0FF1609F452
:10933000C3C02DE0F21609F4BFC083E2F81619F09D
:109340009AE3F912CFC080912C068111CBC0AFC037
:10935000E0EEF7E084916F012FEFC21AD20A882362
:1093600019F040DCF601F6CF0E94717F8CE895E1A0
:109370000E947ECE8091C615882369F1815080932A
:10938000C615EDE8E89FC001112441E061E0855376
:109390009A4E0E94918CE091C61524E0E29FF00164
:1093A0001124E953FA4E40815181628173814093C7
:1093B0005C1650935D1660935E1670935F168CE892
:1093C00095E10E94FFFE8091C213882309F447C0F3
:1093D0009092C11344C01092C1136AE580E299E1F2
:1093E0000E940AEB1092E8161092301940E050E00B
:1093F000BA018BEA95E10E94FFFE49E452E068EE73
:1094000076E18BEA95E10E9495FF019669F43EE5CD
:10941000C32E33E0D32EF60181916F01882311F022
:10942000E1DBF9CF8AE0DEDB8BEA95E10E947ECEBC
:1094300010921C1210921B12B092F70FA092F60F0E
:109440003ADA0E94B1E80E94528A6D3371058105B3
:10945000910528F07092F70F6092F60F2CDA1092B7
:1094600064168091C213882319F00E945B881FC084
:109470000E940A898091C2138111F7CF18C0E0EED3
:10948000F2E284916F012FEFC21AD20A882319F0F9
:10949000A9DBF601F6CFE1EDF7E084916F019FEFD4
:1094A000C91AD90A882319F09DDBF601F6CFE3E249
:1094B000FE1202C090922D0610922C060115110585
:1094C00009F4E7CE80912E10889E000D111D112405
:1094D000F801E25BFF4E108280E00E94204000E035
:1094E00010E0D7CE0F35110508F0D3CEFBE3FF1205
:1094F00002C090922C0680912C068111CACE8091D8
:109500002E10F801889EE00DF11D1124E25BFF4E44
:10951000F0820F5F1F4FBDCE0F90DF91CF911F9153
:109520000F91FF90EF90DF90CF90BF90AF909F9002
:109530008F907F906F905F904F903F902F90089505
:109540008F929F92AF92BF92CF92DF92EF92FF9253
:10955000CF936B017C01B42E20E030E0A9010F9481
:109560007B2387FF06C08DE23DDBF7FAF094F7F826
:10957000F094C0E060E070E080E09FE3CB1541F044
:109580002DEC3CEC4CEC5DE30F94E023CF5FF6CF89
:109590009B01AC01C701B6010F94152A6B017C0138
:1095A0000F945E2B4B015C014AE0DEDBCC2379F1AA
:1095B000C501B4010F947F239B01AC01C701B60123
:1095C0000F94142A6B017C018EE20CDB20E030E06A
:1095D00040E251E4C701B6010F94E0234B015C0166
:1095E0000F94592B6B01770FEE08FF08C701B601E6
:1095F00062DCC701B6010F9481239B01AC01C50158
:10960000B4010F94142A6B017C01C150F9F6CF917B
:10961000FF90EF90DF90CF90BF90AF909F908F9092
:1096200008958F929F92AF92BF92CF92DF92EF9266
:10963000FF920F931F93CF93DF93EDEEF8E08491A9
:10964000EF012196882319F0CDDAFE01F8CFC12C65
:10965000D12C7601C0E080E2C5DACF5FC830D9F7FF
:10966000C701B60128DC8FEFC81AD80AE80AF80A41
:1096700095E0C916D104E104F10461F78AE0B2DA99
:1096800000E816E1C12CD12C760180E2ABDAC701EB
:10969000B60111DCC0E0D0E080E2A4DAF801EC0F02
:1096A000FD1F80809180A280B380A5019401C50137
:1096B000B4010F94C32C811110C020E030E0A90147
:1096C000C501B4010F943B2C87FD02C08BE28ADAFE
:1096D00045E0C501B40134DF08C0B12C80E282DA74
:1096E000B3948DE398E0B912FACF6496C436D105ED
:1096F00099F68AE077DA8FEFC81AD80AE80AF80AEA
:109700000C5F1F4F95E0C916D104E104F10409F084
:10971000BCCF8AE067DA8AED98E09093F70F8093E8
:10972000F60FDF91CF911F910F91FF90EF90DF9097
:10973000CF90BF90AF909F908F90BDC81F920F9217
:109740000FB60F9211240BB60F922F938F939F9306
:10975000EF93FF93E091031B81E08E0F8F77909141
:10976000C6002091041B821731F0F0E0ED57F54E52
:1097700090838093031BFF91EF919F918F912F9185
:109780000F900BBE0F900FBE0F901F9018950F9368
:109790001F93CF93DF938C01EFE1F9E08491EF0108
:1097A0002196882319F01EDAFE01F8CFF801849182
:1097B000EF012196882319F015DAFE01F8CFE6E0D3
:1097C000F9E08491EF012196882319F00BDAFE016C
:1097D000F8CFDF91CF911F910F910895FF920F93D2
:1097E0001F93CF93DF938C01EB01F42E80E2FAD923
:1097F0008FEFF81611F084E501C082E4F3D98AE313
:10980000F1D9F801608171818281938142E098DE13
:10981000488159816A817B818CE19AE0DF91CF9107
:109820001F910F91FF900D94EA0C0F931F93CF930C
:10983000DF93CDB7DEB728970FB6F894DEBF0FBE23
:10984000CDBF60912F1070913010072E000C880B47
:10985000990B0F9481236D837E838F8398878091EA
:10986000211290912212A0912312B0912412898387
:109870009A83AB83BC834EEFBE016B5F7F4FCE01FB
:109880000196ACDF60916B1B70916C1B072E000C76
:10989000880B990B0F9481236D837E838F83988728
:1098A0008091700890917108A0917208B09173082E
:1098B00089839A83AB83BC834FEFBE016B5F7F4F7D
:1098C000CE0101968BDFE4E2FAE084918F010F5F15
:1098D0001F4F882319F086D9F801F7CFE091B8051A
:1098E000F0E0E35AFD4E608170E080E090E0E3DA62
:1098F000EFE1FAE084918F010F5F1F4F882319F089
:1099000071D9F801F7CF60915C1270E080E090E0CF
:10991000D2DA28960FB6F894DEBF0FBECDBFDF9126
:10992000CF911F910F9108952F923F924F925F9286
:109930006F927F928F929F92AF92BF92CF92DF925F
:10994000EF92FF920F931F93CF93DF93CDB7DEB7C4
:109950002F970FB6F894DEBF0FBECDBF8091471290
:1099600083FD66C160E084E69AE00E94CFB383E5A0
:10997000E4D88887811105C082E5DFD8882309F4FF
:1099800057C179D80F94592B6E37710514F06DE7D4
:1099900070E070936C1B60936B1B0E945BC26BD872
:1099A00020E030E040EA50E40F943B2C181614F409
:1099B0000E9467F281E08093940280916C0880930A
:1099C000B805412C512C32011C821D821E821F823F
:1099D0001B8219862CE32A873CE13B8746E44C87AF
:1099E00010E000E050E859838FEB8A83812C912CA2
:1099F000540160916B1B70916C1B072E000C880B3F
:109A0000990B0F9481237B018F879D879B01AC016C
:109A1000612F702F89819A810F947B23882309F409
:109A200049C020917008309171084091720850919E
:109A300073089885B7018F8591110EC09D850F948D
:109A40007B23881F8827881F8B831E2D0F2DAF85B2
:109A5000A983BD85BA832EC09D850F947B2387FF84
:109A600022C080919402882309F4E2C060E086E578
:109A70009AE02F960FB6F894DEBF0FBECDBFDF91F0
:109A8000CF911F910F91FF90EF90DF90CF90BF90FB
:109A9000AF909F908F907F906F905F904F903F908E
:109AA0002F900C94CFB31E2D0F2D2F8529833D852C
:109AB0003A831B820E947EF76B017C01DC01CB01A3
:109AC0002C813D814E815F81821B930BA40BB50BD2
:109AD000B7FD37C0D701C60188519C4FAF4FBF4F6C
:109AE0008C839D83AE83BF83A0DEE0E6FAE08491A1
:109AF000DF011196BE87AD87882321F073D8ED85ED
:109B0000FE85F5CF81149104A104B104B1F0D50113
:109B1000C401805F984DAF4FBF4FBC01CD016C19A0
:109B20007D098E099F0928EE33E040E050E00F9454
:109B3000B729CA01B901BFD902C08FE353D88AE05F
:109B400051D880E00E947C670AD82090700830903D
:109B50007108B0917208BF87209173082D87910119
:109B60004B2F5D85612F702F89819A810F94142A64
:109B70009F7781149104A104B10449F420E030E0FE
:109B800040E85FE30F947B2387FF0BC008C020E011
:109B900030E040E450E40F943B2C181614F44601D6
:109BA00057013B81332361F1411451046104710475
:109BB00041F0D701C60184199509A609B709B7FD77
:109BC0001FC091014F855D8569857A858B859C8550
:109BD0000F94142A20E030E040EC5FE30F947B23E5
:109BE00087FD3FCF2601370140E6440E4AEE541E62
:109BF000611C711C29863A865F855B878D858C8701
:109C000080919402882309F42CCF81149104A1043B
:109C1000B10409F4EECE90E1C91A97E2D90AE1083D
:109C2000F108C818D908EA08FB08F7FE1ACFE1CEF8
:109C30002F960FB6F894DEBF0FBECDBFDF91CF9148
:109C40001F910F91FF90EF90DF90CF90BF90AF905A
:109C50009F908F907F906F905F904F903F902F904C
:109C600008952F923F924F925F926F927F928F92C0
:109C70009F92AF92BF92CF92DF92EF92FF920F939B
:109C80001F93CF93DF93CDB7DEB72F970FB6F8941E
:109C9000DEBF0FBECDBF8DE690E0D1D8811192C15D
:109CA0008091471283FD8EC183E50E949D45888780
:109CB000811106C082E50E949D45882309F482C176
:109CC0000E943B450F94592BCB010E943BB30E944D
:109CD0003B4520E030E04AEA52E40F947B2318161B
:109CE00044F00E94B1E860E086E49AE00E94CFB3BD
:109CF00002C00E9467F260912F1070913010072E01
:109D0000000C880B990B0F94812320912112309124
:109D1000221240912312509124120F943B2C1816BA
:109D200084F483E393E09F938F938AE39AE09F9375
:109D30008F931F920E9467EB0F900F900F900F90E0
:109D40000F900F94CB0D81E080939402412C512C05
:109D500032011C821D821E821F821B8219862CE307
:109D60002A873CE13B8746E44C8710E000E050E85E
:109D700059838FEB8A83812C912C540160912F1091
:109D800070913010072E000C880B990B0F948123D3
:109D90007B018F879D879B01AC01612F702F89818B
:109DA0009A810F947B23882309F449C020912112C2
:109DB0003091221240912312509124129885B701BC
:109DC0008F8591110EC09D850F947B23881F882756
:109DD000881F8B831E2D0F2DAF85A983BD85BA8368
:109DE0002EC09D850F947B2387FF22C08091940213
:109DF000882309F4E7C060E088E29AE02F960FB666
:109E0000F894DEBF0FBECDBFDF91CF911F910F91B0
:109E1000FF90EF90DF90CF90BF90AF909F908F908A
:109E20007F906F905F904F903F902F900C94CFB3A6
:109E30001E2D0F2D2F8529833D853A831B820E947D
:109E40007EF76B017C01DC01CB012C813D814E81D1
:109E50005F81821B930BA40BB50BB7FD3BC0D701F1
:109E6000C60188519C4FAF4FBF4F8C839D83AE83FB
:109E7000BF83DBDCE6E3FAE08491DF011196BE8765
:109E8000AD87882329F00E94F245ED85FE85F4CF49
:109E900081149104A104B104B9F0D501C401805F1B
:109EA000984DAF4FBF4FBC01CD016C197D098E0994
:109EB0009F0928EE33E040E050E00F94B729CA0133
:109EC000B9010E945B4703C08FE30E94F2458AE01C
:109ED0000E94F24580E00E947C670E94AF4520907E
:109EE000211230902212B0912312BF8720912412A8
:109EF0002D8791014B2F5D85612F702F89819A816C
:109F00000F94142A9F7781149104A104B10449F499
:109F100020E030E040E85FE30F947B2387FF0BC035
:109F200008C020E030E040E450E40F943B2C1816C9
:109F300014F4460157013B81332361F1411451046C
:109F40006104710441F0D701C60184199509A6097D
:109F5000B709B7FD1FC091014F855D8569857A8579
:109F60008B859C850F94142A20E030E040EC5FE361
:109F70000F947B2387FD3ACF2601370140E6440E3C
:109F80004AEE541E611C711C29863A865F855B87E8
:109F90008D858C8780919402882309F427CF8114C2
:109FA0009104A104B10409F4E9CE90E1C91A97E241
:109FB000D90AE108F108C818D908EA08FB08F7FE31
:109FC00015CFDCCE2F960FB6F894DEBF0FBECDBFF7
:109FD000DF91CF911F910F91FF90EF90DF90CF9085
:109FE000BF90AF909F908F907F906F905F904F90B9
:109FF0003F902F900895CF92DF92EF92FF92CF93F0
:10A0000081E080939402C1E081E0909194029923D1
:10A0100009F449C0882309F446C080E00E947C67A7
:10A0200060912F10709130106115710581F1072E2C
:10A03000000C880B990B0F9481239B01AC0160915C
:10A0400021127091221280912312909124120F9468
:10A05000142A6B017C0120E030E0A9010F943B2C15
:10A0600018165CF020E030E040E450ECC701B60187
:10A070000F947B2387FD0DC00AC020E030E040E450
:10A0800050E4C701B6010F943B2C181614F080E081
:10A09000BCCFC093111240E050E0BA018FED93E9BC
:10A0A0000E948F74B1CFCF91FF90EF90DF90CF904F
:10A0B0000895CF92DF92EF92FF920F931F93CF9369
:10A0C000DF9300D01F92CDB7DEB7182F662351F073
:10A0D0001092380610923406109235061092360609
:10A0E000109237060E947EF7C0903406D090350655
:10A0F000E0903606F09037069B01AC012C193D0923
:10A100004E095F0957FD3EC017FD16C04091380645
:10A11000212F012E000C330B2C5F3F4FE42F042E18
:10A12000000CFF0B2E173F076CF141172CF000E9D4
:10A1300011E020E030E004C004EC19E020E030E061
:10A14000DC01CB01800F911FA21FB31F8093340647
:10A1500090933506A0933606B093370680ED97E0CE
:10A160009C838B838CE291E09A838983BE016D5F2F
:10A170007F4FCE0101960E9459F1809138068F5F82
:10A18000809338060F900F900F900F90DF91CF9132
:10A190001F910F91FF90EF90DF90CF900895CF9295
:10A1A000DF92EF92FF920F931F93CF93DF9381EB98
:10A1B000E82E82E0F82E0FE318E0C1E4D9E199EB34
:10A1C000C92E95E0D92EF70181917F010E946E453D
:10A1D0008823E1F00E943B459B01AC01F6018081A0
:10A1E000811104C08091BD05882329F0688179819F
:10A1F0008A819B8103C060E070E0CB010F94152A37
:10A20000F801608371838283938309C08881998177
:10A21000AA81BB81F80180839183A283B3830C5F01
:10A220001F4F2496FFEFCF1ADF0A85EBE81682E076
:10A23000F80649F686E40E949D458823C9F00E94ED
:10A240003B4520E030E0A9010F943B2C181684F424
:10A250000E943B4520E030E040E752E40F94F12AB1
:10A2600060938C0270938D0280938E0290938F0284
:10A27000DF91CF911F910F91FF90EF90DF90CF90E2
:10A2800008954F925F926F927F928F929F92AF92BA
:10A29000BF92CF92DF92EF92FF920F931F93CF93D3
:10A2A000DF93CDB7DEB72C970FB6F894DEBF0FBEA5
:10A2B000CDBF7C012A013B01B22EA32E82E0E8161D
:10A2C000F10449F420E030E0A901C301B2010F9488
:10A2D0007B2387FD8CC0D12CEE0CFF1CEE0CFF1CE9
:10A2E000F701EF5BF64E4F0110821182128213824A
:10A2F0000E94B444F4014082518262827382C09011
:10A300006C0820E030E0A901B8018B2D9A2D0F9444
:10A310007B2381110CC0F701E758F04F859195918F
:10A32000A591B491982E892EBA2EAB2E02C0902EF4
:10A33000812E8091491990914A19A0914B19B091A1
:10A340004C194091451950914619609147197091E7
:10A3500048190091411910914219209143193091E7
:10A36000441909831A832B833C834D835E836F8357
:10A37000788789879A87AB87BC87AE01475F5F4F35
:10A38000BE016B5F7F4FCE0101960E940EE2E92C69
:10A39000F82C0B2D1A2D2DE439E1AE01475F5F4FEC
:10A3A000BE016B5F7F4FCE0101960E94F1D40E94E7
:10A3B000717FDD2019F080E00E94F94510924D1068
:10A3C0002C960FB6F894DEBF0FBECDBFDF91CF91B4
:10A3D0001F910F91FF90EF90DF90CF90BF90AF90C3
:10A3E0009F908F907F906F905F904F90089581E045
:10A3F0000E94F945DD24D3946FCFCF92DF92EF9284
:10A40000FF926091D5117091D611072E000C880B28
:10A41000990B0F9481236B017C012DEB37E346E808
:10A4200055EB0F943B2C87FD0AC02DEB37E346E834
:10A4300055E3C701B6010F947B2318164CF4A7010E
:10A44000960160E070E080E89FE30F94F12A03C07A
:10A4500060E070E0CB016093091B70930A1B80934E
:10A460000B1B90930C1B6091D7117091D811072E84
:10A47000000C880B990B0F9481236B017C012DEB51
:10A4800037E346E855EB0F943B2C87FD0AC02DEBD4
:10A4900037E346E855E3C701B6010F947B2318164E
:10A4A0004CF4A701960160E070E080E89FE30F9410
:10A4B000F12A03C060E070E0CB0160930D1B709344
:10A4C0000E1B80930F1B9093101BFF90EF90DF905B
:10A4D000CF9008952F923F924F925F926F927F920A
:10A4E0008F929F92AF92BF92CF92DF92EF92FF92A4
:10A4F0000F931F93CF93DF93CDB7DEB7E1970FB6DE
:10A50000F894DEBF0FBECDBF00916D0881E0082733
:10A51000B0906E08B82610916F081827011104C07A
:10A52000B11002C009F47FC0EBEEFCE484917F011E
:10A530002FEFE21AF20A811103C0E7E4F9E004C048
:10A540000E94F245F701F2CF84917F013FEFE31AB9
:10A55000F30A882321F00E94F245F701F5CF00238A
:10A5600069F0E5E4F9E084917F019FEFE91AF90AC7
:10A57000882321F00E94F245F701F5CFBB2069F056
:10A58000E3E4F9E084917F01AFEFEA1AFA0A882345
:10A5900021F00E94F245F701F5CF112319F0E1E413
:10A5A000F9E003C0E9E3F9E00BC084917F01BFEF5C
:10A5B000EB1AFB0A8823B1F30E94F245F701F5CFAD
:10A5C00084917F012FEFE21AF20A882321F00E9482
:10A5D000F245F701F5CF112319F046E955E002C025
:10A5E00044E254E0BB2019F023E833E002C024E247
:10A5F00034E0002319F085E893E002C084E294E09F
:10A600005F934F933F932F939F938F9387E299E0AC
:10A610009F938F931F920E9467EB0FB6F894DEBF53
:10A620000FBECDBF28C52090AB1287E50E946E45B6
:10A63000882309F429C18091D5119091D611892BD5
:10A64000D1F4E0EEF2E284918F010F5F1F4F811190
:10A6500003C0E0EDF9E004C00E94F245F801F3CF39
:10A6600084918F010F5F1F4F882309F404C50E9456
:10A67000F245F801F5CFC0904919D0904A19E09001
:10A680004B19F0904C1980907C1690907D16A090FC
:10A690007E16B0907F168AE50E949D45811107C005
:10A6A000A5019401C701B6010F94142A02C00E94AB
:10A6B0003B456B017C0120E030E040E251EC0F941F
:10A6C0003B2C87FD0AC020E030E040E251E4C701A6
:10A6D000B6010F947B231816D4F4E0EEF2E28491D5
:10A6E0008F010F5F1F4F811103C0E3ECF9E004C03D
:10A6F0000E94F245F801F3CF84918F010F5F1F4F45
:10A70000882309F4B8C40E94F245F801F5CF88E522
:10A710000E949D45882329F00E943B452B013C0166
:10A7200006C0412C512C60EC662E6FE7762E89E531
:10A730000E949D45882329F00E943B454B015C0106
:10A7400006C0812C912C50ECA52E5FE7B52E89E434
:10A750000E949D45882319F00E941B4501C08FEF80
:10A76000082F8AE40E949D45882319F00E941B450A
:10A7700001C08FEF182FA3019201C301B2010F9402
:10A78000C32C811162C0A5019401C501B4010F94CD
:10A79000C32C81115AC06091D1117091D211072E32
:10A7A000000C880B990B0F94812320917416309123
:10A7B000751640917616509177160F94152A9B01C5
:10A7C000AC01C301B2010F94142A20E030E0A901CA
:10A7D0000F94152A20E030E0A9010F94F12A0F947C
:10A7E000592B062F6091D3117091D411072E000CB4
:10A7F000880B990B0F94812320917816309179164C
:10A8000040917A1650917B160F94152A9B01AC014A
:10A81000C501B4010F94142A20E030E0A9010F947F
:10A82000152A20E030E0A9010F94F12A0F94592B4A
:10A83000E02F05300CF0E4E00E2FE7FD00E0162FCE
:10A8400065300CF014E017FD10E0053008F013C47B
:10A85000163008F010C480E00E943D4195E00902E6
:10A86000F0011124E10FF11D17FDFA95EE0FFF1F06
:10A87000EE0FFF1FE058F94EC082D182E282F382D0
:10A88000822D0E943D41F7C38AE40E946E458823D1
:10A8900019F00E947941EFC386E50E949D45882307
:10A8A00029F00E940B4579A768A702C019A618A62F
:10A8B000A8A5B9A5159768F0EBE9F9E084918F0197
:10A8C0000F5F1F4F882309F4D6C30E94F245F80199
:10A8D000F5CF84E40E946E45382E882319F00E943B
:10A8E0002C45382E8AE50E949D45882339F00E9428
:10A8F0003B456EA77FA788AB99AB04C01EA61FA6D9
:10A9000018AA19AA83E50E949D45882319F00E9480
:10A910003B4504C060E070E88BE395E420E030E064
:10A9200040E752E40F94F12A609387027093880203
:10A930008093890290938A0220E030E048E452E458
:10A9400060917416709175168091761690917716B5
:10A950000F94152A4B015C018CE40E949D458823CD
:10A9600021F00E943B454B015C01C501B4010F94ED
:10A97000592B69877A878B879C8709851A8520E000
:10A9800030E04AE753E46091741670917516809137
:10A990007616909177160F94152A4B015C0182E58B
:10A9A0000E949D45882321F00E943B454B015C019C
:10A9B000C501B4010F94592B6D877E878F87988BC3
:10A9C000ED85FE85FE8FED8F20E030E048E452E417
:10A9D000609178167091791680917A1690917B1615
:10A9E0000F94152A4B015C0186E40E949D45882343
:10A9F00021F00E943B454B015C01C501B4010F945D
:10AA0000592B698B7A8B8B8B9C8B29893A893BA339
:10AA10002AA320E030E04AE753E460917816709171
:10AA2000791680917A1690917B160F94152A4B0116
:10AA30005C0182E40E949D45882321F00E943B45F1
:10AA40004B015C01C501B4010F94592B6D8B7E8BBA
:10AA50008F8B988F8D899E899BA78AA7A985BA8598
:10AA6000BD01BB0F880B990B0F9481236CA37DA3B1
:10AA70008EA39FA38090741690907516A090761662
:10AA8000B090771620E030E04CE352E4C501B40109
:10AA90000F94152A9B01AC016CA17DA18EA19FA1F1
:10AAA0000F947B2387FD0AC0B1E0B9A38D859E85F5
:10AAB00009970817190724F419A202C0E1E0E9A3D5
:10AAC0002D853E85B901330F880B990B0F94812397
:10AAD0002B013C0120E030E04BE953E4C501B40117
:10AAE0000F94152A9B01AC01C301B2010F943B2CBA
:10AAF00001E018164CF089859A850996AD8DBE8DBA
:10AB00008A179B070CF400E0E989FA89BF01FF0F5F
:10AB1000880B990B0F9481236D8F7E8F8F8F98A355
:10AB20008090781690907916A0907A16B0907B1647
:10AB300020E030E0A901C501B4010F94152A9B0162
:10AB4000AC016D8D7E8D8F8D98A10F947B2311E0CC
:10AB500087FD09C08D899E8909972AA13BA12817E5
:10AB600039070CF410E0AD89BE89BD01BB0F880B1D
:10AB7000990B0F9481232B013C0120E030E04BE93D
:10AB800053E4C501B4010F94152A9B01AC01C30124
:10AB9000B2010F943B2CBB24B39418164CF0898956
:10ABA0009A890996EAA5FBA58E179F070CF4B12C8C
:10ABB000F9A1F1110CC0002329F08CE899E00E9462
:10ABC000C74B0BC011110BC0B11010C014C084E9E9
:10ABD00099E00E94C74B0111F0CF112321F084E8C6
:10ABE00099E00E94C74BBB2009F445C28DE799E06C
:10ABF0000E94C74B40C228A539A5232BD1F0E6E619
:10AC0000F9E084918F010F5F1F4F882321F00E948C
:10AC1000F245F801F6CF332061F0EDE4F9E08491DC
:10AC20008F010F5F1F4F882321F00E94F245F8012A
:10AC3000F6CF0E94717F1092AB12311006C084E6ED
:10AC400090E00F94F1070E94B44481E00E94B24268
:10AC5000882319F02092AB120EC2AD84BE84898580
:10AC60009A85A81AB90AB7FE03C093E0A90EB11CD1
:10AC7000B594A794B594A794B5010B2C000C880B40
:10AC8000990B0F9481236AA77BA78CA79DA70D8999
:10AC90001E89A989BA890A1B1B0B17FF02C00D5F09
:10ACA0001F4F1595079515950795B801012E000CB6
:10ACB000880B990B0F9481232B013C010E94D345F3
:10ACC0006091D5117091D611072E000C880B990B4D
:10ACD0000F9481239B01AC016AA57BA58CA59DA542
:10ACE0000F947B2381114EC06091D7117091D811C0
:10ACF000072E000C880B990B0F9481239B01AC014C
:10AD0000C301B2010F947B2381113CC06091D1112A
:10AD10007091D211072E000C880B990B0F94812390
:10AD200020917416309175164091761650917716D1
:10AD30000F94152A9B01AC016CA17DA18EA19FA14E
:10AD40000F947B2381111EC06091D3117091D41197
:10AD5000072E000C880B990B0F94812320917816F5
:10AD60003091791640917A1650917B160F94152ADE
:10AD70009B01AC016D8D7E8D8F8D98A10F947B23EF
:10AD80008823B1F131102092AB120E947941B09228
:10AD9000D611A092D5111093D8110093D7112091FC
:10ADA00074163091751640917616509177166CA1F5
:10ADB0007DA18EA19FA10F94142A0F94592B7093FB
:10ADC000D2116093D111209178163091791640916B
:10ADD0007A1650917B166D8D7E8D8F8D98A10F9474
:10ADE000142A0F94592B7093D4116093D311212CF2
:10ADF00085E40E946E45898B882319F00E942C45BA
:10AE0000898B1E861D86B1E0BD8BA7019601C70107
:10AE1000B6010F94C32C8111C5C03D89332309F4B9
:10AE2000BAC0E1E0EAA3F5E0F9A319862D8931E083
:10AE300023272D8B8D859E85092E000CAA0BBB0B1D
:10AE4000898F9A8FAB8FBC8F99A1A9859A1709F426
:10AE500097C06A2FAA0F770B880B990B0F94812349
:10AE60002AA53BA54CA55DA50F94E0232CA13DA1EF
:10AE70004EA15FA10F94152A4B015C01698D7A8D5B
:10AE80008B8D9C8D0F948123A30192010F94E0235D
:10AE90002D8D3E8D4F8D58A10F94152A6B017C018D
:10AEA00020E030E0A901C501B4010F947B2387FFA6
:10AEB00004C060E070E0CB0104C060E070E080E0BE
:10AEC0009FE3A50194010F94152A0F948A2B69839F
:10AED0007A838B839C8320E030E0A901C701B6010F
:10AEE0000F947B2387FF04C060E070E0CB0104C0B7
:10AEF00060E070E080E09FE3A70196010F94152ABF
:10AF00000F948A2B6D837E838F83988728A5498928
:10AF1000BE016B5F7F4FCE0101960E9440F36B0133
:10AF20007C019B01AC010F94C32C882319F0209263
:10AF3000AB1226C025E039853203800111248D85AE
:10AF40009E85080F191F000F111F000F111F0058B9
:10AF5000194E2EA53FA548A959A9C701B6010F94BE
:10AF6000152AD8016D937D938D939C93139780E060
:10AF70000E947C67BAA1E985BE0FB987212C64CFF6
:10AF80002D853E852F5F3F4F3E872D87253031052C
:10AF900009F03BCF07C08FEF8AA39FEF99A3A4E0EE
:10AFA000A98744CF80E00E94B242882319F0209202
:10AFB000AB1253C0A7019601C701B6010F94C32C71
:10AFC00081114BC0332009F10E94114B0E94BFA494
:10AFD00014DA31103FC081E499E10F943D089B01E0
:10AFE000AC016091491970914A1980914B19909167
:10AFF0004C190F94142A6093491970934A1980933D
:10B000004B1990934C1981E026C012E084E0F82E91
:10B0100002E0EF2CE11ADF2CD01A21E041E0602F92
:10B02000812F0F94A91021E04FEF602F8E2D0F94E8
:10B03000A9102FEF41E06D2D812F0F94A9102FEF54
:10B040004FEF6D2D8E2D0F94A910015020F7115048
:10B05000F8F6BACF822D8093AB120E94BA4527D35F
:10B0600081E090E090934606809345068091AB1274
:10B0700081110E94B444E1960FB6F894DEBF0FBE72
:10B08000CDBFDF91CF911F910F91FF90EF90DF9097
:10B09000CF90BF90AF909F908F907F906F905F9078
:10B0A0004F903F902F9008958F929F92AF92BF92B2
:10B0B000CF92DF92EF92FF920F931F93CF93DF9384
:10B0C000CDB7DEB7AC970FB6F894DEBF0FBECDBFDD
:10B0D0008091C213882309F4D8C08CE895E10E94BE
:10B0E000CDFE8CE895E10E947ECE1092C0131092A6
:10B0F000BF138091C213882309F4C7C0E090B6053E
:10B10000F090B7051092C11380918F15882321F01C
:10B110008CE895E10E947ECECE0101966C010E94E2
:10B1200071FC8EEE93E190930E1480930D14F70151
:10B1300080818F3209F05AC06FE270E0C7010F942E
:10B140006A2D8C010F5F1F4F09F456C06FE270E04B
:10B15000C8010F946A2D5C01009709F44EC00817CE
:10B16000190708F04AC04C01801A910AA401B801DD
:10B17000CE0180960F94932DE0E2F0E0EC0FFD1FDE
:10B18000E80DF91D10828E01005E1F4FF8018191BC
:10B190008F01882319F00E94F245F8CF8AE00E94BF
:10B1A000F24560910D1470910E146115710511F046
:10B1B0006C5F7F4F21E0AE01405E5F4FCE01059690
:10B1C0000E9413D481110CC0BE01605E7F4F88E0E5
:10B1D0009AE00F94200D8EE20E94F2458AE050C062
:10B1E000D0920E14C0920D148501ACCF8FE094E183
:10B1F00090930E1480930D14870180910D149091FB
:10B200000E14009709F00496B8010F9423018823C7
:10B2100009F1E2EEF9E084917F019FEFE91AF90A62
:10B22000882321F00E94F245F701F5CFF8018191C2
:10B230008F01882319F00E94F245F8CF8AE00E941E
:10B24000F24510925C1610925D1610925E161092E6
:10B250005F1618C0E0EFF9E084917F019FEFE91AD3
:10B26000F90A882321F00E94F245F701F5CFF80191
:10B2700081918F01882319F00E94F245F8CF8EE268
:10B280000E94F245C6010E943B64AC960FB6F8944A
:10B29000DEBF0FBECDBFDF91CF911F910F91FF9009
:10B2A000EF90DF90CF90BF90AF909F908F900895D8
:10B2B000FF920F931F93CF93DF9389E40E949D45E4
:10B2C000882321F00E940B45062F01C00FEF8AE46E
:10B2D0000E949D45882321F00E940B45C62F01C086
:10B2E000CFEF8AE50E946E45D82F811105C081E518
:10B2F0000E946E45F82E01C0F12C07FD06C0C7FD67
:10B3000004C0D1111AC0F11018C0E0EEF2E284912D
:10B31000EF012196811103C0E1E0FEE004C00E942C
:10B32000F245FE01F4CF8491EF012196882309F4C0
:10B3300055C00E94F245FE01F6CF053010F4C5302D
:10B34000B8F0E0EEF2E28491EF012196811103C0A2
:10B35000E2EEFDE004C00E94F245FE01F4CF8491CC
:10B36000EF0121968823D1F10E94F245FE01F7CF2B
:10B37000002E000C110B0C2E000CDD0B0E943B4527
:10B380009B01AC01FF2099F085E0809FF001819F37
:10B39000F00D1124EC0FFD1FEE0FFF1FEE0FFF1F2E
:10B3A000E058F94E608171818281938103C060E031
:10B3B00070E0CB01A5E0A09FF001A19FF00D11244A
:10B3C000CE0FDF1FCC0FDD1FCC0FDD1FC058D94EB5
:10B3D0000F94152A688379838A839B83DF91CF91A9
:10B3E0001F910F91FF900895CF92DF92EF92FF92FD
:10B3F000CF93DF9386E50E946E45882341F08091CC
:10B40000D5119091D611892B11F00E94114B83E533
:10B410000E946E45C82F882319F00E942C45C82F22
:10B4200083E50E946E45882319F08C2F0E943D41D0
:10B430008AE50E946E45882321F00E943B450E94C8
:10B44000F540F090AB12C11103C0EBEEFCE418C064
:10B45000F110FBCFE0EEF2E28491EF012196882318
:10B4600021F00E94F245FE01F7CFE3ECFDE084916C
:10B47000EF012196882349F30E94F245FE01F7CFA0
:10B480008491EF012196882321F00E94F245FE016C
:10B49000F7CFF11003C06BE873E002C067E873E018
:10B4A00085EB9DE00F94200D8AE00E94F245EBEEC3
:10B4B000FCE48491EF012196882321F00E94F2455B
:10B4C000FE01F7CFE8EAFDE08491EF0121968823A1
:10B4D00021F00E94F245FE01F7CFC090A712D09054
:10B4E000A812E090A912F090AA1220E030E0A90181
:10B4F000C701B6010F943B2C181674F442E0C70143
:10B50000B6010E94A04A8AE0DF91CF91FF90EF90B0
:10B51000DF90CF900C94F245E3EAFDE08491EF01D7
:10B520002196882321F00E94F245FE01F7CFDF919A
:10B53000CF91FF90EF90DF90CF90089588E893E14E
:10B540009093800D80937F0D80916F008D7F80930D
:10B550006F009091211380912213981719F00F9486
:10B560008C0BF7CF1092820D1092810D80916F009D
:10B57000826080936F008FB7F89410920D12109232
:10B580000E1210920F12109210128FBF0E94717F34
:10B5900084E690E00F94F1070C94B444CF93DF93CA
:10B5A000EDE6FBE08491EF012196882321F00E94D3
:10B5B000F245FE01F7CFEFE5FBE08491EF01219624
:10B5C000882321F00E94F245FE01F7CFE8E4FBE07A
:10B5D0008491EF012196882321F00E94F245FE011B
:10B5E000F7CFE8E3FBE08491EF012196882321F077
:10B5F0000E94F245FE01F7CFE7E2FBE08491EF0104
:10B600002196882321F00E94F245FE01F7CFE6E162
:10B61000FBE08491EF012196882321F00E94F245FE
:10B62000FE01F7CFE7E0FBE08491EF01219688234C
:10B6300021F00E94F245FE01F7CFE2EFFAE084919B
:10B64000EF012196882321F00E94F245FE01F7CFF9
:10B65000ECEDFAE08491EF012196882321F00E941D
:10B66000F245FE01F7CFE7ECFAE08491EF01219675
:10B67000882321F00E94F245FE01F7CFEAEAFAE0C2
:10B680008491EF012196882321F00E94F245FE016A
:10B69000F7CFE2E9FAE08491EF012196882321F0C7
:10B6A0000E94F245FE01F7CFDF91CF9108954F92AE
:10B6B0005F926F927F928F929F92AF92BF92CF9242
:10B6C000DF92EF92FF92CF93DF93EFE8FAE084915D
:10B6D000EF012196882321F00E94F245FE01F7CF69
:10B6E00060914119709142198091431990914419C8
:10B6F00042E00E94A04AEBE8FAE08491EF01219633
:10B70000882321F00E94F245FE01F7CF6091451990
:10B7100070914619809147199091481942E00E9412
:10B72000A04AE7E8FAE08491EF012196882321F00E
:10B730000E94F245FE01F7CF6091491970914A19B4
:10B7400080914B1990914C1942E00E94A04AE3E885
:10B75000FAE08491EF012196882321F00E94F245BE
:10B76000FE01F7CF60914D1970914E1980914F19DC
:10B770009091501942E00E94A04A8FB7F8944090EF
:10B7800031195090321960903319709034198090AB
:10B79000351990903619A0903719B0903819C0908B
:10B7A0003919D0903A19E0903B19F0903C198FBFAD
:10B7B000E9E7FAE08491EF012196882321F00E94C5
:10B7C000F245FE01F7CFC301B2010E945B47E5E7F6
:10B7D000FAE08491EF012196882321F00E94F2453E
:10B7E000FE01F7CFC501B4010E945B47E1E7FAE033
:10B7F0008491EF012196882321F00E94F245FE01F9
:10B80000F7CFC701B6010E945B478AE0DF91CF9175
:10B81000FF90EF90DF90CF90BF90AF909F908F9070
:10B820007F906F905F904F900C94F2452F923F92D3
:10B830004F925F926F927F928F929F92AF92BF9240
:10B84000CF92DF92EF92FF920F931F93CF93DF93EC
:10B85000CDB7DEB72A970FB6F894DEBF0FBECDBFC7
:10B860008DE698E09E838D8384E7882E86E1982E6E
:10B8700091E4A92E99E1B92E29E3C22E26E0D22E19
:10B8800039E2232E32E0332E4DE6E42E4FE0F42E43
:10B8900000E010E0ED81FE818191FE83ED8388233D
:10B8A00009F480C0F5014080518062807380F1010D
:10B8B0002081318142815381F601608171818281D1
:10B8C00093810F94152A20E030E040E05FE30F946D
:10B8D000E0239B01AC01C301B2010F943B2C18166D
:10B8E00054F4F70185919591A591B4918F83988730
:10B8F000A987BA8704C01F82188619861A86F401A0
:10B900002081318142815381C301B2010F94142AF5
:10B910009B01AC016F81788589859A850F94142AE3
:10B920002B013C0120E030E040EA51EC0F943B2C2D
:10B9300087FD0AC020E030E040EA51E4C301B201D3
:10B940000F947B2318161CF4E0EEF2E209C0B30159
:10B95000A201C8010E94034425C00E94F245F801DB
:10B9600084918F010F5F1F4F8111F7CFEFE3FEE04E
:10B9700084918F010F5F1F4F882321F00E94F245B1
:10B98000F801F6CF61E081E39EE00E94CFB30E9410
:10B99000B27488E290E09C838B8388EC90E09A8379
:10B9A000898332C00F5F1F4FF4E08F0E911C84E03B
:10B9B000A80EB11C94E0C90ED11CE4E02E0E311C7F
:10B9C000F4E0EF0EF11C0330110509F063CF0E9483
:10B9D000B4446DDE60E081E29EE00E94CFB383E973
:10B9E00092E09C838B8304E610E01A830983BE01F6
:10B9F0006D5F7F4FCE0101960E9459F18AEB92E074
:10BA00009C838B831A830983BE016D5F7F4FCE01B8
:10BA100001960E9459F12A960FB6F894DEBF0FBE28
:10BA2000CDBFDF91CF911F910F91FF90EF90DF90ED
:10BA3000CF90BF90AF909F908F907F906F905F90CE
:10BA40004F903F902F9008952F923F924F925F9288
:10BA50006F927F928F929F92AF92BF92CF92DF921E
:10BA6000EF92FF920F931F93CF93DF93CDB7DEB783
:10BA7000E1970FB6F894DEBF0FBECDBF85E40E94FC
:10BA80009D45882321F00E940B458B0102C000E0F8
:10BA900010E083E40E949D45882329F00E940B4515
:10BAA0007BA76AA704C025E030E03BA72AA785E56D
:10BAB0000E946E4589A3882319F00E942C4589A312
:10BAC00017FD07C0C12CD12CB6E1EB2EB3E4FB2E41
:10BAD00006C0C12CD12CACE8EA2EA2E4FA2E83E5F4
:10BAE0000E949D45882321F00E943B456B017C010B
:10BAF0000115110511F41092B8050E947EF72B0173
:10BB00003C01C8010196029748F143E953E05A838A
:10BB10004983A981BA818D91BA83A983882319F0B9
:10BB20000E94F245F6CF8AE0E1960FB6F894DEBFA8
:10BB30000FBECDBFDF91CF911F910F91FF90EF907E
:10BB4000DF90CF90BF90AF909F908F907F906F903D
:10BB50005F904F903F902F900C94F245ECEBF3E008
:10BB6000FA83E983A981BA818D91BA83A983882355
:10BB700019F00E94F245F6CF8AE00E94F2450E9439
:10BB8000A7C28FE70F3FBFEF1B0719F480935C122A
:10BB900002C080935D12C701B6010F94592B072E86
:10BBA000000C880B990B0F9481236D8B7E8B8F8BF0
:10BBB000988F81E0809394024AA25BA26CA27DA23E
:10BBC0004CA65DA66EA67FA6198EE0E4EA8FFCE186
:10BBD000FB8F26E42C8F1D8E1E8E1F8E18A2198AB5
:10BBE0001A8A1B8A1C8A1D861E861F86188AC12CEB
:10BBF000D12C7601FFE78F2E912CA12CB12C8FE751
:10BC000090E0A0E0B0E08D839E83AF83B8871EA252
:10BC10001FA218A619A691E099871C861B86212CC5
:10BC2000312C19AA18AA80919402882309F4D0C152
:10BC30000E947EF769837A838B839C8380915B1259
:10BC4000882309F4A0C00E94B0C30115110559F45E
:10BC50002090211230902212A0912312A9ABB09112
:10BC60002412B8AB0AC02090700830907108E0919F
:10BC70007208E9ABF0917308F8AB910149A958A992
:10BC80006D8D7E8D8F8D98A10F947B2387FF06C0CD
:10BC90002D8E3E8E29A92F8F38A938A3298D3A8D54
:10BCA0004B8D5C8DB10189A998A90F947B2387FFE7
:10BCB00006C0298E3A8E49A94B8F58A95C8F898579
:10BCC000910149A958A96D897E89882309F441C049
:10BCD0008F89988D0F947B2387FF55C049815A81A6
:10BCE0006B817C814419550966097709DB01CA011A
:10BCF00088589341A109B109B7FD45C08D819E8146
:10BD0000AF81B88588199909AA09BB09B595A79586
:10BD1000979587950F3FEFEF1E0719F480935C12FC
:10BD200002C080935D124EA35FA368A779A7FD8927
:10BD3000FD8F2E892E8F3F893F8F488D48A38981A3
:10BD40009A81AB81BC818AA39BA3ACA3BDA31986B6
:10BD50001AC08F89988D0F943B2C1816A4F48981F2
:10BD60009A81AB81BC812AA13BA14CA15DA1821B20
:10BD7000930BA40BB50BAC01BD01485853416109AD
:10BD8000710977FF43C120E030E040EA51E46D895A
:10BD90007E898F89988D0F94152A910149A958A9F8
:10BDA0000F947B2387FF0FC0EFE2FDE08491DF015A
:10BDB0001196BA83A983882309F47CC20E94F245B4
:10BDC000E981FA81F3CF80E398EFAFEFBFEF2CA5C5
:10BDD0003DA54EA55FA5821B930BA40BB50B298136
:10BDE0003A814B815C81820F931FA41FB51FB7FD61
:10BDF0000DC00E94154C8AE00E94F24589819A810B
:10BE0000AB81BC818CA79DA7AEA7BFA789819A8172
:10BE1000AB81BC81880F991FAA1FBB1F2AA13BA120
:10BE20004CA15DA1821B930BA40BB50B8419950942
:10BE3000A609B70981349747AB41B10580F0E1E12C
:10BE4000FDE08491AF014F5F5F4F5A8349838823A0
:10BE500009F430C20E94F245E981FA81F2CF8AA545
:10BE60009BA5AB85BC858A179B070CF0AEC0E4EBA5
:10BE7000FCE084919F012F5F3F4F3A832983882301
:10BE800029F00E94F245E981FA81F3CF0F3F3FEF9D
:10BE9000130729F044E254E05A83498304C08FE831
:10BEA00093E09A83898369817A8182EA9CE00F9486
:10BEB000200DB701A6018EE99CE00F94EA0C8AE000
:10BEC0000E94F24569817A818CE89CE00F94200DF4
:10BED0004D855E856F85788988E89CE00F94EA0C33
:10BEE0008AE00E94F24569817A8186E79CE00F949E
:10BEF000200D49895A896B897C8982E79CE00F94DF
:10BF0000EA0C8AE00E94F24599A1992309F4D2C172
:10BF10000F3F1F4F69F5C0928B0DD0928C0DE092B0
:10BF20008D0DF0928E0D2CEA35EC47E25EE36D85C7
:10BF30007E858F8598890F94E0236093870D709399
:10BF4000880D8093890D90938A0D2CEA35EC47E299
:10BF50005EE369897A898B899C890F94F12A6093C1
:10BF6000830D7093840D8093850D9093860DA2C1EF
:10BF7000C092930DD092940DE092950DF092960D93
:10BF80002CEA35EC47E25EE36D857E858F859889E6
:10BF90000F94E02360938F0D7093900D8093910D1B
:10BFA0009093920D2CEA35EC47E25EE369897A8939
:10BFB0008B899C890F94F12A6093970D7093980D4B
:10BFC0008093990D90939A0D75C10E94FCB32BCE6E
:10BFD0008091940281116EC1E1960FB6F894DEBF94
:10BFE0000FBECDBFDF91CF911F910F91FF90EF90CA
:10BFF000DF90CF90BF90AF909F908F907F906F9089
:10C000005F904F903F902F900C94A7C24B855C851A
:10C01000141615060CF024C14EA05FA068A479A4E4
:10C02000480E591E6A1E7B1E2EA13FA148A559A588
:10C03000281B390B4A0B5B0BC501B4010F94A829CF
:10C04000A30192010F94D9298D809E80AF80B8847E
:10C05000820E931EA41EB51E54E185169104A10400
:10C06000B1040CF18CEE88169104A104B1043CF4E7
:10C0700090E889169104A104B10434F422C05BEE67
:10C08000852E912CA12CB12C8D829E82AF82B886F8
:10C090002EEF30E040E050E0281939094A095B09E9
:10C0A00049015A0112C084E190E0A0E0B0E08D8324
:10C0B0009E83AF83B88744E1842E912CA12CB12CB0
:10C0C00004C08D829E82AF82B886EBE9FDE0849148
:10C0D000DF011196BA87A987882329F00E94F245CB
:10C0E000E985FA85F4CF6D817E818F8198850E94E4
:10C0F0005B47E6E9FDE084919F012F5F3F4F3A8760
:10C100002987882329F00E94F245E985FA85F3CF33
:10C11000C501B4010E945B47498D5A8D6B8D7C8DA2
:10C120008FE89DE00F94EA0C4D8D5E8D6F8D78A1A8
:10C1300088E89DE00F94EA0C4B855C8543305105FF
:10C140000CF48EC0C501B4010F94812320E030E0CF
:10C1500040E850E40F94E0236B017C01298D3A8D77
:10C160004B8D5C8D6D8D7E8D8F8D98A10F94142AD3
:10C170002BED3FE049E450E40F94E02320E030E071
:10C1800040E05FE30F94E0239B01AC01C701B601DF
:10C190000F94F12A6B017C01C301B2010F9481233A
:10C1A0002FE632E143E85AE30F94E0232B013C01F0
:10C1B000B701A60182E89DE00F94EA0CB301A20149
:10C1C0008CE79DE00F94EA0C2AE939E949E15FE345
:10C1D000C701B6010F94E0236B017C019B01AC0108
:10C1E0000F94152AA30192010F94F12A6D877E877F
:10C1F0008F87988BA7019601C301B2010F94E023AA
:10C2000020E030E040E05EE30F94E023698B7A8B1E
:10C210008B8B9C8BECE6FDE084913F015FEF651A10
:10C22000750A882321F00E94F245F301F5CFB7018A
:10C23000A60186E69DE00F94EA0C4D855E856F852C
:10C24000788980E69DE00F94EA0C49895A896B89C8
:10C250007C898AE59DE00F94EA0C8AE00E94F24511
:10C260008D819E81AF81B885880D991DAA1DBB1D4A
:10C27000B595A795979587950F3FEFEF1E0719F492
:10C2800080935C1202C080935D122B853C852F5FEA
:10C290003F4F3C872B873D89398F4E894A8F5F8975
:10C2A0005B8F888D8C8F49805A806B807C8091E079
:10C2B000998769CDE1960FB6F894DEBF0FBECDBF6A
:10C2C000DF91CF911F910F91FF90EF90DF90CF9072
:10C2D000BF90AF909F908F907F906F905F904F90A6
:10C2E0003F902F900895CF93DF9385E40E949D4562
:10C2F000811110C080E50E946E45882391F00E9454
:10C300003B456093930D7093940D8093950D90939E
:10C31000960D07C00E941B45882361F3E0EEF2E210
:10C320006AC089E40E946E45882381F00E943B45E3
:10C330002CEA35EC47E25EE30F94E02360938F0D27
:10C340007093900D8093910D9093920D84E40E94D0
:10C350006E45882381F00E943B452CEA35EC47E28C
:10C360005EE30F94F12A6093970D7093980D80937C
:10C37000990D90939A0DEBEEFCE48491EF012196D8
:10C38000882321F00E94F245FE01F7CF4091930DE2
:10C390005091940D6091950D7091960D8EE69CE0F4
:10C3A0000F94EA0C2CEA35EC47E25EE360918F0DC6
:10C3B0007091900D8091910D9091920D0F94F12AB2
:10C3C000AB01BC018AE69CE00F94EA0C2CEA35EC48
:10C3D00047E25EE36091970D7091980D8091990D01
:10C3E00090919A0D0F94E023AB01BC0186E69CE08E
:10C3F0000F94EA0C11C08491EF012196882321F05B
:10C400000E94F245FE01F7CFCEE3D3E08991882365
:10C4100019F00E94F245FACF8AE0DF91CF910C9497
:10C42000F245CF93DF93EBEEFCE48491EF0121968C
:10C43000882321F00E94F245FE01F7CF83E50E9498
:10C440006E45882321F00E942C4580938B02E6E5FF
:10C45000FCE08491EF012196882321F00E94F245AF
:10C46000FE01F7CF80918B02811103C0E2E5FCE071
:10C4700002C0EEE4FCE08491EF012196882321F0D4
:10C480000E94F245FE01F7CFE6E4FCE08491EF0163
:10C490002196882321F00E94F245FE01F7CF4091BA
:10C4A000390650913A0660913B0670913C0684E44F
:10C4B0009CE00F94EA0C40913D0650913E0660913D
:10C4C0003F067091400681E49CE00F94EA0C409195
:10C4D00041065091420660914306709144068EE3F6
:10C4E0009CE00F94EA0CE6E3FCE08491EF012196D6
:10C4F000882321F00E94F245FE01F7CF40912902E6
:10C5000050912A0260912B0270912C0284E39CE0EE
:10C510000F94EA0C40912D0250912E0260912F024F
:10C520007091300281E39CE00F94EA0C409131025B
:10C530005091320260913302709134028EE29CE09D
:10C540000F94EA0C8AE0DF91CF910C94F2458FEFC3
:10C550008EBD0DB407FEFDCF8EB508954F925F924C
:10C560006F927F928F929F92AF92BF92EF92FF92C3
:10C570000F931F93CF93DF93EC01FC01EA53F04F2D
:10C580001491029729F481E00E94B242811114C1F2
:10C590007E01EE0CFF1CEE0CFF1CF701E654F04F81
:10C5A0004590559065907490612F110F770B880B13
:10C5B000990B0F9481234B015C0120E030E040ECAB
:10C5C0005FE3C301B2010F94E023A50194010F942E
:10C5D000E023AB01BC0100E010E09801CE010E9415
:10C5E0004151C230D10589F406EB1FE0F801659195
:10C5F00075918591949120E030E040EA50E40F94E9
:10C600007B2387FD0EC0F80103C0F701E255F04F10
:10C6100085919591A591B491E82F792F6A2F8B2F51
:10C6200004C0E0E070E060EA80E42E2F372F462F50
:10C63000582FC501B4010F94E0234B015C0120E0A9
:10C6400030E0A9010F947B23882309F449C000E05E
:10C6500010E09801B501A4017058CE010E9441512B
:10C66000FE01E555F04F6491611119C0EBEEFCE459
:10C6700084918F010F5F1F4F882321F00E94F245A4
:10C68000F801F6CFE9E8FFE084918F010F5F1F4FBB
:10C69000882321F00E94F245F801F6CF6AE0F70105
:10C6A000E758F04F459055906590749070E080E0A9
:10C6B00090E00F9481239B01AC01C301B2010F9460
:10C6C000F12A2B013C01A5019401C501B4010F948D
:10C6D000152AAB01BC0193018201CE010E94415198
:10C6E00081E0FE01E359F74F8083FE01EA5EFF4ED1
:10C6F0008083F701ED5CF74F108211821282138262
:10C70000CE010E94AD43F701E359F04F25913591D9
:10C710004591549187010F5B164EF701EC58F94E85
:10C7200060817181828193810F94152AF801608361
:10C73000718382839383C230D105D1F42091E416B2
:10C740003091E5164091E6165091E716609149192F
:10C7500070914A1980914B1990914C190F94142A99
:10C760006093491970934A1980934B1990934C190F
:10C770000E94B444F701E15CF74FD701AF5BB64EBE
:10C780008D919D910D90BC91A02D80839183A2836A
:10C79000B383229789F480E0DF91CF911F910F91AD
:10C7A000FF90EF90BF90AF909F908F907F906F9091
:10C7B0005F904F900C94B242DF91CF911F910F91F7
:10C7C000FF90EF90BF90AF909F908F907F906F9071
:10C7D0005F904F900895CF92DF92EF92FF92CF93A8
:10C7E000DF93EC01C0902902D0902A02E0902B0246
:10C7F000F0902C02A7019601688179818A819B8142
:10C800000F943B2C181624F4C882D982EA82FB824A
:10C81000C0902D02D0902E02E0902F02F0903002B6
:10C82000A70196016C817D818E819F810F943B2CA5
:10C83000181624F4CC82DD82EE82FF82C090310291
:10C84000D0903202E0903302F0903402A7019601BA
:10C85000688579858A859B850F943B2C181624F46E
:10C86000C886D986EA86FB86DF91CF91FF90EF904C
:10C87000DF90CF90089525EC32E0FC0131832083D6
:10C8800004960C94A9457F928F929F92AF92BF928B
:10C89000CF92DF92EF92FF920F931F93CF93DF938C
:10C8A000CDB7DEB7C055D1090FB6F894DEBF0FBEC5
:10C8B000CDBF89E492E0E8EEF6E1DF019C011D9234
:10C8C00021503040E1F780EE91E0E3E5F6E0DF0152
:10C8D0009C011D9221503040E1F78091C2138111DB
:10C8E00002C00E940A898091C213882309F484C27D
:10C8F0000FEC13E0D8018D918D01882319F00E946F
:10C90000F245F8CF8AE00E94F2450AEE13E0F80102
:10C9100081918F01882319F00E94F245F8CF8AE0B7
:10C920000E94F2454AE069E472E080E090E00E94F3
:10C93000B4468AE00E94F2454FE050E069E67FE0AD
:10C9400080E299E10F94EC2221E040E259E162EFAC
:10C9500073E18BEA95E10E9413D4882309F44CC259
:10C9600061E080E299E10E940AEB49E452E068EE5E
:10C9700076E18BEA95E10E9406D18BEA95E10E946F
:10C980007ECE01EF13E0D8018D918D01882319F03F
:10C990000E94F245F8CF8AE00E94F2456091E816C5
:10C9A00070E080E090E04AE00E94B4468AE00E9495
:10C9B000F2456091301970E080E090E04AE00E941A
:10C9C000B4468AE00E94F2458091E816882309F473
:10C9D00001C2909130198913F5C19FB7F8948091E5
:10C9E00008018E7F809308019FBF0EEF13E0F801CE
:10C9F00081918F01882319F00E94F245F8CF8AE0D7
:10CA00000E94F24509EE16E1D8016D917D918D915C
:10CA10009D918D0142E00E94A04A8AE00E94F24569
:10CA2000B6E1093F1B0781F76091F9167091FA167C
:10CA30008091FB169091FC1660938C0270938D028E
:10CA400080938E0290938F0242E00E94A04A8AE077
:10CA50000E94F24501E017E1F801619171918F01A7
:10CA6000072E000C880B990B0E945B478AE00E94FE
:10CA7000F245F7E109301F0779F7609103177091CC
:10CA80000417072E000C880B990B0E945B478AE065
:10CA90000E94F24505E214E0D8018D918D018823B2
:10CAA00019F00E94F245F8CF8AE00E94F2456091A9
:10CAB000051770910617072E000C880B990B0E9422
:10CAC0005B478AE00E94F245609107177091081752
:10CAD000072E000C880B990B0E945B478AE00E948E
:10CAE000F2456091091770910A17072E000C880B08
:10CAF000990B0E945B478AE00E94F24500E010E03B
:10CB0000F801E55FF84E7F01D7018D917D01882303
:10CB100019F00E94F245F8CF8AE00E94F245005ACF
:10CB20001F4F0038B1E01B0759F78E010F5B1F4FF5
:10CB300080E1F801282F11922A95E9F74E0131E39F
:10CB4000830E911CD401E82F1D92EA95E9F77E012E
:10CB5000F1E2EF0EF11CD701E82F1D92EA95E9F7FB
:10CB60006E01F1E1CF0ED11CD601E82F1D92EA959E
:10CB7000E9F79E012F5F3F4F5901D9011D928A9518
:10CB8000E9F76091E9167091EA168091EB169091A1
:10CB9000EC1623E041E00F94801E6091ED16709139
:10CBA000EE168091EF169091F016840123E041E09B
:10CBB0000F94801E6091F1167091F2168091F31619
:10CBC0009091F416870123E041E00F94801E20E04D
:10CBD00030E040EA50E46091F1167091F2168091D5
:10CBE000F3169091F4160F94152A850123E041E085
:10CBF0000F94801E20E030E040E450E46091F51690
:10CC00007091F6168091F7169091F8160F94142AE9
:10CC1000860123E041E00F94801EDF92CF92FF92C5
:10CC2000EF928DE59FE09F938F9383E596E09F932E
:10CC30008F930F94152383E596E00E9482EB81E0A9
:10CC400090E090931C1280931B1283E5E82E86E0FF
:10CC5000F82E0FB6F894DEBF0FBECDBF670190E689
:10CC6000792E24E0A22EB12C8090091790900A17FB
:10CC7000F0E6CF0ED11C1814190444F500910517E5
:10CC800010910617709EB001719E700D1124655FA2
:10CC9000784EC6010F947E2D80911B1290911C122C
:10CCA000019690931C1280931B1221E0821A910826
:10CCB00090920A1780920917C8010196B5010F9446
:10CCC000022D9093061780930517CECF00E010E059
:10CCD00080911B1290911C120817190794F4670198
:10CCE000D6018D916D01882319F00E94F245F8CF8D
:10CCF0008AE00E94F2450F5F1F4FB0E6EB0EF11C79
:10CD0000E7CF0AE314E0F80181918F01882319F03D
:10CD10000E94F245F8CF8AE00E94F24560918F1898
:10CD20007091901880919118909192184AE00E9409
:10CD3000B4468AE00E94F24503E918E1D8018D91DA
:10CD40008D01882319F00E94F245F8CF8AE00E94F5
:10CD5000F24560918B1870918C1880918D1890918C
:10CD60008E184AE00E94B4468AE00E94F245809103
:10CD70008F1890919018A0919118B091921880936B
:10CD80002A1090932B10A0932C10B0932D1040E0FC
:10CD900061E083E998E10E94918C40918B18509159
:10CDA0008C1860918D1870918E1840935C1650937A
:10CDB0005D1660935E1670935F168CE895E10E9495
:10CDC000FFFE1AC08AE49FE09093F70F8093F60F5E
:10CDD0000E945B4489E492E0E8EEF6E1DF019C0109
:10CDE0001D9221503040E1F74FE050E066E47FE0D3
:10CDF00080E299E10F94EC22C05BDF4F0FB6F8940C
:10CE0000DEBF0FBECDBFDF91CF911F910F91FF907D
:10CE1000EF90DF90CF90BF90AF909F908F907F90DA
:10CE200008958C01E0EEF2E28491EF0121968823CF
:10CE300021F00E94F245FE01F7CFE6E2FFE0849187
:10CE4000EF012196882321F00E94F245FE01F7CFE1
:10CE50000E94A7C20F94F7060E94B2B761E0C80112
:10CE60000E94CFB30E94B2740E94D1E9C4E00E9434
:10CE70002EB3C09312128091C4128695869510929B
:10CE8000FA128093FB120E9456E98091C412869593
:10CE90008695880F1092FA128093FB1287E19FE02B
:10CEA0000E94C1C68091C41286958695982F990FCD
:10CEB000890F1092FA128093FB128AE09FE00E9481
:10CEC000C1C60E94CAE88111D2CF2FEF8BE49DE149
:10CED000215080409040E1F700C00000F8942FEF0F
:10CEE00084E39CE0215080409040E1F700C00000C6
:10CEF0000E94A7C2A895FECF4F925F926F927F9239
:10CF00008F929F92AF92BF92CF92DF92EF92FF9259
:10CF10000F931F93CF93DF93082F0E94FCB30E94BF
:10CF20007EF76B017C0110910002112309F465C0AA
:10CF30008091450690914606009709F45EC04091A5
:10CF40004F08509150086091510870915208460165
:10CF50005701841A950AA60AB70AB7FC60C0833045
:10CF6000910509F130F4019708F447C0EBEEFCE4B9
:10CF700006C0049709F041C0EBEEFCE42AC084919E
:10CF8000EF012196882321F00E94F245FE01F7CFA0
:10CF9000ECE8FEE08491EF012196882371F10E9474
:10CFA000F245FE01F7CFEBEEFCE48491EF01219610
:10CFB000882321F00E94F245FE01F7CFE5E7FEE06D
:10CFC0008491EF0121968823C1F00E94F245FE0171
:10CFD000F7CF8491EF012196882321F00E94F2453A
:10CFE000FE01F7CFEDE5FEE08491EF012196882365
:10CFF00021F00E94F245FE01F7CF212F30E0A8EE8C
:10D00000B3E00F94052AC60ED71EE81EF91EC09283
:10D010004F08D0925008E0925108F0925208C09107
:10D020004B06CC2391F00E947EF7C0904706D0902B
:10D030004806E0904906F0904A06DC01CB018C19C5
:10D040009D09AE09BF09B7FFCBC18091CF118430D4
:10D0500010F40E94A9470E947EF780904F0690909E
:10D060005006A0905106B090520681149104A1047C
:10D07000B10469F1C0902A10D0902B10E0902C10D0
:10D08000F0902D10C80CD91CEA1CFB1C9B01AC01B4
:10D090002C193D094E095F0957FD19C0E0EEF2E277
:10D0A0008491EF012196882321F00E94F245FE0130
:10D0B000F7CF60914D0670914E0680ED9EE00F9483
:10D0C000200D8AE00E94F24587EC9EE05DC0209131
:10D0D0004C0621112AC08090010290900202A0907B
:10D0E0000302B090040281149104A104B104E9F098
:10D0F000C0902A10D0902B10E0902C10F0902D10A2
:10D10000C80CD91CEA1CFB1CDC01CB018C199D0945
:10D11000AE09BF09B7FD09C0011107C090912113E5
:10D1200080912213981709F477C180915708909144
:10D130005808909902C0019604C0181619062CF4DC
:10D1400001979093580880935708809157089091C1
:10D1500058088E3E9240CCF0E0EEF2E28491EF016E
:10D160002196882321F00E94F245FE01F7CFE7EADD
:10D17000FEE08491EF012196882321F00E94F24580
:10D18000FE01F7CF8EE99EE04CDE60916D1B909121
:10D19000211380912213981791F0E09122134DE40E
:10D1A000E49FF0011124EB50F74F6081809122132E
:10D1B00090912113981719F08F5F8F70F9CF70E05D
:10D1C00089E00E947EF680915A12882309F4F2C009
:10D1D0000091A3021091A402D091A502C091A602D1
:10D1E00060912F10709130106E5F7F4F072E000CF2
:10D1F000880B990B0F94812398014D2F5C2F0F946E
:10D200007B2387FDD7C0F0902213912CA12CB12C49
:10D21000E12C8DE4882E809121138F1509F45AC0DA
:10D220008F2D90E0889EF001899EF00D1124E2552B
:10D23000F74F4281538164817581452B462B472BE3
:10D2400081F44681578160857185452B462B472B9C
:10D2500041F44285538564857585452B462B472BC4
:10D26000A1F1889E9001899E300D1124C90182553B
:10D27000974F6C01FC0166857785808991890F94B1
:10D2800081232B013C01F601628973898489958988
:10D290000F947F239B01AC01C301B2010F94F12ACB
:10D2A000F60123A134A145A156A10F94E0233B012F
:10D2B0006C01292D3A2D4B2D5E2D0F943B2C181609
:10D2C00024F4962CA72CBC2CED2C81E08F0D8F70B4
:10D2D000F82EA1CF2091A7023091A8024091A90277
:10D2E0005091AA02692D7A2D8B2D9E2D0F94E0234B
:10D2F00098014D2F5C2F0F94152A6B017C019B0127
:10D30000AC01B8018D2F9C2F0F943B2C1816A4F064
:10D3100000919F021091A002D091A102C091A2029F
:10D3200098014D2F5C2FB601C7010F943B2C1816A6
:10D330001CF08601DE2DCF2DC0905308D0905408EC
:10D34000E0905508F090560898014D2F5C2FC701CA
:10D35000B6010F943B2C1816D4F420E037ED43EAC5
:10D360005CE3B8018D2F9C2F0F94E0234B015C01EF
:10D3700028E431EE4AE75FE3C701B6010F94E023EA
:10D38000A50194010F94152A8B01D82FC92FC8012C
:10D39000AD2FBC2F8093530890935408A093550849
:10D3A000B0935608B8018D2F9C2F0F94592BCB01A9
:10D3B0000E943BB30E94D47B83E993E1DF91CF913C
:10D3C0001F910F91FF90EF90DF90CF90BF90AF90A3
:10D3D0009F908F907F906F905F904F900C94A8409B
:10D3E0000E947EF76B017C012C2F30E0A8EEB3E0A9
:10D3F0000F94052AC60ED71EE81EF91EC0924706D6
:10D40000D0924806E0924906F0924A060E94154CD6
:10D410008AE00E94F24519CE5F9A109216108A9AFD
:10D42000109217109FB7F894809108018160809343
:10D4300008019FBF109218100F94F50676CE4F92F8
:10D440005F926F927F928F929F92AF92BF92CF9294
:10D45000DF92EF92FF920F931F93CF93DF93CDB79D
:10D46000DEB76A970FB6F894DEBF0FBECDBF9A8FB6
:10D47000898F5B018A01DC01D7966D917D918D9139
:10D480009C91DA970F947F236B017C01F501208139
:10D490003181428153810F94E0230F94DB2A0F9452
:10D4A0005E2B69877A878B879C87D8012D913D9168
:10D4B0004D915C91C701B6010F94E0230F94DB2AD4
:10D4C0000F945E2B6D877E878F87988B29853A8591
:10D4D0004B855C85283731054105510540F488E7C7
:10D4E00090E0A0E0B0E089879A87AB87BC872D8564
:10D4F0003E854F855889283731054105510540F44F
:10D5000088E790E0A0E0B0E08D879E87AF87B88B7A
:10D51000E98DFA8DED5BFF4F20813181428153818E
:10D520002D833E834F835887CA01B9010F9481230D
:10D5300069837A838B839C8369857A858B859C85B7
:10D540000F947F23698B7A8B8B8B9C8B20E030E050
:10D55000A90169817A818B819C810F947B23882327
:10D5600039F1A7019601C701B6010F94E0234B01E1
:10D570005C0129893A894B895C89CA01B9010F94F8
:10D58000E0239B01AC01C501B4010F94142A4B01A7
:10D590005C0129813A814B815C81CA01B9010F94F8
:10D5A000152A9B01AC01C501B4010F94F12A03C0F7
:10D5B00060E070E0CB010F94DB2A0F94592B2B0114
:10D5C0003C016D817E818F819885909580957095C5
:10D5D00061957F4F8F4F9F4F0F9481234B015C01CB
:10D5E0006D857E858F8598890F947F236D837E83DB
:10D5F0008F83988720E030E0A901C501B4010F9422
:10D600007B23882349F12D813E814F815885CA01B2
:10D61000B9010F94E0236D8B7E8B8F8B988FA701C0
:10D620009601C701B6010F94E0239B01AC016D89FF
:10D630007E898F89988D0F94142A6B017C01A50136
:10D640009401C501B4010F94152A9B01AC01C701D7
:10D65000B6010F94F12A03C060E070E0CB010F9493
:10D660008A2BA98DBA8D52968D909D90AD90BC90CD
:10D67000559775016401C418D508E608F7080F949A
:10D68000592BC61AD70AE80AF90AF7FE6BC020E040
:10D6900030E0A90169817A818B819C810F947B2381
:10D6A000882309F447C0C501B4010F947F236B019F
:10D6B0007C0129813A814B815C81CA01B9010F94B7
:10D6C000152A9B01AC01C701B6010F94E0236B0141
:10D6D0007C0129893A894B895C89CA01B9010F9477
:10D6E000E0239B01AC01C701B6010F94142A6B0122
:10D6F0007C012D813E814F815885CA01B9010F946B
:10D70000E0239B01AC01C701B6010F94152A6B0100
:10D710007C0120E030E040E850E469817A818B812F
:10D720009C810F94E0239B01AC01C701B6010F94CB
:10D73000F12A03C060E070E0CB010F94DB2A0F9464
:10D74000592B2B013C0197FF03C0412C512C320176
:10D75000481459046A047B0410F024013501C12CDB
:10D76000D12C76018FB7F894E98DFA8D908193FDD5
:10D770001DC0468A578A608E718EC40CD51CE61C6B
:10D78000F71CC28ED38EE48EF58E29853A854B85A3
:10D790005C8523AF34AF45AF56AFFF962D853E85F0
:10D7A0004F85588920833183428353838FBF6A9684
:10D7B0000FB6F894DEBF0FBECDBFDF91CF911F91A2
:10D7C0000F91FF90EF90DF90CF90BF90AF909F9020
:10D7D0008F907F906F905F904F9008950F931F935D
:10D7E000CF93DF93E091810DF091820D828193813F
:10D7F000A481B581181619061A061B06E4F4809157
:10D800007E0D80FF18C09CB180915A0895FB992726
:10D8100090F98E7F892780935A08909159089170CA
:10D82000892349F080914D10816080934D1080E0F4
:10D8300090E00E942F7FE091810DF091820D868112
:10D840009781A085B185181619061A061B061CF5C6
:10D8500080917E0D81FF1FC09091030180915A0835
:10D8600091FB002700F910E0119501951109082797
:10D8700002701127082700935A0880915908827076
:10D88000082349F080914D10826080934D1081E013
:10D8900090E00E942F7FE091810DF091820D8285B2
:10D8A0009385A485B585181619061A061B0644F536
:10D8B00080917E0D82FF24C080911910882301F190
:10D8C00099B180915A0892FB992790F9C92F90E05D
:10D8D000D92FD195C195D109C827C470DD27C82794
:10D8E000C0935A08809159088470C82349F08091E8
:10D8F0004D10846080934D1082E090E00E942F7F55
:10D9000080915A0880935908DF91CF911F910F9110
:10D910000895CF93DF93EEE6F2E18491EF01219633
:10D92000882321F00E94F245FE01F7CFE6E6F2E1FE
:10D930008491EF012196882321F00E94F245FE0197
:10D94000F7CF659903C0C1E6D4E002C0C6E6D4E0D3
:10D950008991882319F00E94F245FACF8AE00E944B
:10D96000F245EEE5F2E18491EF012196882321F062
:10D970000E94F245FE01F7CF8091030181FD03C0B3
:10D98000C1E6D4E002C0C6E6D4E08991882319F04C
:10D990000E94F245FACF8AE00E94F245E6E5F2E104
:10D9A0008491EF012196882321F00E94F245FE0127
:10D9B000F7CF4A9903C0C1E6D4E002C0C6E6D4E07E
:10D9C0008991882319F00E94F245FACF8AE0DF910D
:10D9D000CF910C94F245AF92BF92CF92DF92EF922B
:10D9E000FF920F931F93CF93C82F882319F0EEE374
:10D9F000F2E10CC0EBEEFCE484918F010F5F1F4F4E
:10DA00008823A9F30E94F245F801F6CF84918F0193
:10DA10000F5F1F4F882321F00E94F245F801F6CFD7
:10DA2000CC2319F0E1E2F2E10CC0EBEEFCE48491CE
:10DA30008F010F5F1F4F8823A9F30E94F245F80161
:10DA4000F6CF84918F010F5F1F4F882321F00E9432
:10DA5000F245F801F6CF8AE00E94F245C1112CC0D0
:10DA6000EBEEFCE484918F010F5F1F4F882321F0C0
:10DA70000E94F245F801F6CFEEE0F2E184918F01C9
:10DA80000F5F1F4F882321F00E94F245F801F6CF67
:10DA900080910910882321F08AE00E94F2453AC063
:10DAA000E3E0F2E184918F010F5F1F4F882391F132
:10DAB0000E94F245F801F6CF4091051050910610F2
:10DAC00060910710709108108AEF91E10F94EA0CB1
:10DAD0008AE00E94F24580910910811127C0CC2371
:10DAE00019F0EFEEF1E10CC0EBEEFCE484918F0154
:10DAF0000F5F1F4F8823A9F30E94F245F801F6CF6C
:10DB000084918F010F5F1F4F882381F00E94F2459F
:10DB1000F801F6CFEBEEFCE484918F010F5F1F4F0D
:10DB2000882351F20E94F245F801F6CFC11124C0BA
:10DB3000EBEEFCE484918F010F5F1F4F882321F0EF
:10DB40000E94F245F801F6CFEEEDF1E184918F01EC
:10DB50000F5F1F4F882321F00E94F245F801F6CF96
:10DB6000EBEEFCE484918F010F5F1F4F882321F0BF
:10DB70000E94F245F801F6CF409151195091521987
:10DB8000609153197091541986ED91E10F94EA0C4C
:10DB90004091551950915619609157197091581923
:10DBA00083ED91E10F94EA0C4091591950915A1963
:10DBB00060915B1970915C1980ED91E10F94EA0C12
:10DBC00040915D1950915E1960915F1970916019D3
:10DBD0008DEC91E10F94EA0C8AE00E94F245C111AC
:10DBE00024C0EBEEFCE484918F010F5F1F4F88236C
:10DBF00021F00E94F245F801F6CFEFEAF1E18491BD
:10DC00008F010F5F1F4F882321F00E94F245F8011A
:10DC1000F6CFEBEEFCE484918F010F5F1F4F88235A
:10DC200021F00E94F245F801F6CF40918F125091F9
:10DC30009012609191127091921286EA91E10F9484
:10DC4000EA0C409193125091941260919512709148
:10DC5000961283EA91E10F94EA0C40919712509149
:10DC600098126091991270919A1280EA91E10F9442
:10DC7000EA0C40919B1250919C1260919D12709100
:10DC80009E128DE991E10F94EA0C8AE00E94F24520
:10DC9000C11124C0EBEEFCE484918F010F5F1F4F94
:10DCA000882321F00E94F245F801F6CFEBE7F1E17D
:10DCB00084918F010F5F1F4F882321F00E94F2454E
:10DCC000F801F6CFEBEEFCE484918F010F5F1F4F5C
:10DCD000882321F00E94F245F801F6CF4091DA1135
:10DCE0005091DB116091DC117091DD1182E791E1BF
:10DCF0000F94CD0C4091DE115091DF116091E01135
:10DD00007091E1118FE691E10F94CD0C4091E211F9
:10DD10005091E3116091E4117091E5118CE691E16D
:10DD20000F94CD0C4091E6115091E7116091E811EC
:10DD30007091E91189E691E10F94CD0C8AE00E947F
:10DD4000F245C11124C0EBEEFCE484918F010F5F1A
:10DD50001F4F882321F00E94F245F801F6CFEFE132
:10DD6000F1E184918F010F5F1F4F882321F00E9402
:10DD7000F245F801F6CFEBEEFCE484918F010F5FE2
:10DD80001F4F882321F00E94F245F801F6CF409101
:10DD9000F2115091F3116091F4117091F51186E137
:10DDA00091E10F94EA0C4091EE115091EF116091C6
:10DDB000F0117091F11183E191E10F94EA0C40911F
:10DDC000EA115091EB116091EC117091ED1180E12D
:10DDD00091E10F94EA0C8AE00E94F245C11124C03F
:10DDE000EBEEFCE484918F010F5F1F4F882321F03D
:10DDF0000E94F245F801F6CFECE9F0E184918F0141
:10DE00000F5F1F4F882321F00E94F245F801F6CFE3
:10DE1000EBEEFCE484918F010F5F1F4F882321F00C
:10DE20000E94F245F801F6CF40918B1250918C126E
:10DE300060918D1270918E1283E990E10F94EA0C3B
:10DE400040918712509188126091891270918A12C4
:10DE500080E990E10F94EA0C4091AC125091AD1220
:10DE60006091AE127091AF128DE890E10F94CD0CDD
:10DE70004091F6115091F7116091F8117091F911DC
:10DE80008AE890E10F94EA0C4091FA115091FB114D
:10DE90006091FC117091FD1187E890E10F94EA0CFC
:10DEA0004091FE115091FF1160910012709101128A
:10DEB00084E890E10F94EA0C409102125091031211
:10DEC000609104127091051281E890E10F94EA0CC0
:10DED0008AE00E94F245C11124C0EBEEFCE484917B
:10DEE0008F010F5F1F4F882321F00E94F245F80138
:10DEF000F6CFE3E7F0E184918F010F5F1F4F882396
:10DF000021F00E94F245F801F6CFEBEEFCE484919B
:10DF10008F010F5F1F4F882321F00E94F245F80107
:10DF2000F6CF40911A1050911B1060911C10709107
:10DF30001D108AE690E10F94EA0C40911E1050915A
:10DF40001F10609120107091211087E690E10F94CE
:10DF5000EA0C40912210509123106091241070918E
:10DF6000251084E690E10F94EA0C8AE00E94F245C5
:10DF7000C11124C0EBEEFCE484918F010F5F1F4FB1
:10DF8000882321F00E94F245F801F6CFE0E5F0E1A8
:10DF900084918F010F5F1F4F882321F00E94F2456B
:10DFA000F801F6CFEBEEFCE484918F010F5F1F4F79
:10DFB000882321F00E94F245F801F6CF6091AB1260
:10DFC00070E087E490E10F94070D4091A712509103
:10DFD000A8126091A9127091AA1284E490E10F94A2
:10DFE000EA0C8AE00E94F245CC2379F08FE7A82E54
:10DFF00082E1B82E9BE7C92E92E1D92E23E8E22ECA
:10E0000022E1F22E00E010E024C0EBEEFCE484916B
:10E010008F010F5F1F4F882321F00E94F245F80106
:10E02000F6CFE7E2F0E184918F010F5F1F4F882365
:10E0300021F00E94F245F801F6CFEBEEFCE484916A
:10E040008F010F5F1F4F882389F20E94F245F8016C
:10E05000F6CFB8018EE190E10F94070DF5016191C3
:10E0600071915F018BE190E10F94070DF6016191D1
:10E0700071916F0188E190E10F94070DF7016191B3
:10E0800071917F0185E190E10F94070D8AE00E9474
:10E09000F2450F5F1F4F02301105D9F6C11124C0A0
:10E0A000EBEEFCE484918F010F5F1F4F882321F07A
:10E0B0000E94F245F801F6CFE6E0F0E184918F018D
:10E0C0000F5F1F4F882321F00E94F245F801F6CF21
:10E0D000EBEEFCE484918F010F5F1F4F882321F04A
:10E0E0000E94F245F801F6CF4091930D5091940DA6
:10E0F0006091950D7091960D8DEF9FE00F94EA0C55
:10E100002CEA35EC47E25EE360918F0D7091900D43
:10E110008091910D9091920D0F94F12AAB01BC0169
:10E120008AEF9FE00F94EA0C2CEA35EC47E25EE3BD
:10E130006091970D7091980D8091990D90919A0D25
:10E140000F94E023AB01BC0187EF9FE00F94EA0C32
:10E150008AE00E94F245C1110CC0EBEEFCE4849110
:10E160008F010F5F1F4F882321F00E94F245F801B5
:10E17000F6CF40918B0D50918C0D60918D0D70916B
:10E180008E0D8EEE9FE00F94EA0C2CEA35EC47E200
:10E190005EE36091870D7091880D8091890D90915B
:10E1A0008A0D0F94F12AAB01BC018BEE9FE00F9416
:10E1B000EA0C2CEA35EC47E25EE36091830D709146
:10E1C000840D8091850D9091860D0F94E023AB0115
:10E1D000BC0188EE9FE00F94EA0C8AE00E94F245B1
:10E1E000C11124C0EBEEFCE484918F010F5F1F4F3F
:10E1F000882321F00E94F245F801F6CFE2EDFFE01E
:10E2000084918F010F5F1F4F882321F00E94F245F8
:10E21000F801F6CFEBEEFCE484918F010F5F1F4F06
:10E22000882321F00E94F245F801F6CF4091E416D0
:10E230005091E5166091E6167091E71689EC9FE023
:10E240000F94EA0C8AE0CF911F910F91FF90EF900D
:10E25000DF90CF90BF90AF900C94F2452F923F92F9
:10E260004F925F926F927F928F929F92AF92BF92E6
:10E27000CF92DF92EF92FF920F931F93CF93DF9392
:10E28000CDB7DEB764970FB6F894DEBF0FBECDBF33
:10E2900085E40E946E45882329F00E943B456B016E
:10E2A0007C0105C0C12CD12CE12C30ECF32E8AE589
:10E2B0000E949D45882329F00E943B452B013C018B
:10E2C00003C0412C512C320188E50E949D458823D2
:10E2D00019F00E943B4503C060E070E0CB01698704
:10E2E0007A878B879C8789E50E949D45882319F052
:10E2F0000E943B4503C060E070E0CB016D877E87E4
:10E300008F87988B85E50E946E45882329F00E94AF
:10E310003B454B015C0106C0812C912C28ECA22EC0
:10E3200022ECB22E8CE40E946E45882339F00E94C4
:10E330003B45698B7A8B8B8B9C8B04C0198A1A8A1C
:10E340001B8A1C8A82E40E949D45882321F00E943A
:10E350000B45162F01C015E02090B1133090B21379
:10E3600080914C06811194C28091471283FD3EC07A
:10E3700020E030E0A901C501B4010F947B23811195
:10E3800009C020E030E0A901C701B6010F947B234A
:10E39000882361F180912512811126C020912F10D0
:10E3A0003091301080911702909118022817390788
:10E3B000DCF4E0EEF2E284917F019FEFE91AF90AC2
:10E3C000882321F00E94F245F701F5CFE8E8F2E159
:10E3D00084917F019FEFE91AF90A882309F458C252
:10E3E0000E94F245F701F4CF0E94FB4F81E0809339
:10E3F0004C069091C113992321F01092C113809380
:10E400005B080E948DF181E08093111240E050E0A2
:10E41000BA0185E095E983D20E94717F80E1E1E451
:10E42000F9E1ACE5B8E001900D928A95E1F720E0C2
:10E4300030E0A901C701B6010F947B238823F1F0D6
:10E440000E943E43A701960160914B0870914C08D1
:10E4500080914D0890914E080F94152A60934B08B7
:10E4600070934C0880934D0890934E0860E070E0E4
:10E4700080E792E40E9452430E94717F20E030E0E6
:10E48000A901C301B2010F943B2C1816FCF480E0E3
:10E4900090E0A0EAB0E48D839E83AF83B887A301A8
:10E4A00092016091491970914A1980914B1990918C
:10E4B0004C190F94152A69837A838B839C83BE0140
:10E4C0006B5F7F4FCE0101960E94AB4280E090E0EF
:10E4D000A8ECB2E489839A83AB83BC839E012F5F4F
:10E4E0003F4F49E459E1BE01635F7F4FCE0109967A
:10E4F0000E94BA4120E030E0A901C501B4010F94A7
:10E500007B23882351F181E08093111240E050E099
:10E51000BA0182E794E903D280E00E947C670E94FE
:10E520003E43A501940160914B0870914C08809185
:10E530004D0890914E080F94152A60934B087093E4
:10E540004C0880934D0890934E0860E070E080E2A4
:10E5500091E40E9452430E94717F01E000931112E6
:10E5600040E050E0BA0189EB92E9D9D161E0812F16
:10E570000E94595080E00E947C670F94F50664E683
:10E5800070E080E090E00E940EB10E947EF7DC0116
:10E59000CB0188539045AF4FBF4F80939B0D909315
:10E5A0009C0DA0939D0DB0939E0D1092750883E075
:10E5B00090E0909346068093450600931A1280914E
:10E5C0001A12882309F44CC060E0812F0E94595030
:10E5D00080917508882309F43FC00093111240E030
:10E5E00050E0BA018CE493E99AD180911A1281111A
:10E5F0002FC010929B0D10929C0D10929D0D1092A9
:10E600009E0D109275080E94CAC20E94FB4F009393
:10E61000111240E050E0BA0189EB92E980D10E94EA
:10E620007EF7DC01CB0188539045AF4FBF4F8093FD
:10E630009B0D90939C0DA0939D0DB0939E0D1092F9
:10E64000750800931A1261E0812F0E94595004C08E
:10E6500081E00E947C67C9CF81E00E947C67AFCFD8
:10E6600081E090E0909346068093450680914C06A9
:10E67000882309F40DC1F090750810929B0D10923B
:10E680009C0D10929D0D10929E0D1092750880E0C9
:10E690000E94CAC2F1100E94FB4F61E0812F0E94CC
:10E6A00059500E943E4320E030E0A90169897A89EF
:10E6B0008B899C890F947B23882309F446C0FF2013
:10E6C00049F081E08093111240E050E0BA0189EBFB
:10E6D00092E925D183E090E0909346068093450629
:10E6E00081E080931A1280911A12882311F0F110A0
:10E6F000D5C081E090E090934606809345068093D4
:10E70000111240E050E0BA0186E292E908D129896D
:10E710003A894B895C8960914B0870914C088091D3
:10E720004D0890914E080F94152A60934B087093F2
:10E730004C0880934D0890934E0860E070E080ECA8
:10E7400090E40E9452430E94717F11E083E0C82E42
:10E75000D12CEE24E394F12C1093111240E050E000
:10E76000BA0183E991E9DBD020E030E048E452E4EB
:10E7700060914B0870914C0880914D0890914E0823
:10E780000F94152A60934B0870934C0880934D08A2
:10E7900090934E0860E070E080E490E40E94524361
:10E7A0000E94717FD0924606C092450610921A12BE
:10E7B000109311121092F90F1092F80F40E050E0F0
:10E7C000BA0188E995E9ABD08091F80F9091F90FE3
:10E7D000009721F481E00E947C67F6CFF092460614
:10E7E000E0924506019709F4B7CF11E0109311129A
:10E7F00040E050E0BA0182E291E991D0809168084E
:10E8000090916908A0916A08B0916B0880934D19A6
:10E8100090934E19A0934F19B093501980934B08C1
:10E8200090934C08A0934D08B0934E080E94A6F117
:10E8300080E090E0A8ECB2E489839A83AB83BC8348
:10E840009E012F5F3F4F49E459E160E678E08CE597
:10E8500098E00E94BA4180E090E0A0EAB0E48983A9
:10E860009A83AB83BC83BE016F5F7F4F84E698E0E1
:10E870000E94AB4277D080915B08882339F0809169
:10E88000C21381111093C11310925B0810924C06B1
:10E890002A94232859F40E9467F208C060E0812F6F
:10E8A0000E94595081E00E947C671DCF64960FB68C
:10E8B000F894DEBF0FBECDBFDF91CF911F910F91B6
:10E8C000FF90EF90DF90CF90BF90AF909F908F9090
:10E8D0007F906F905F904F903F902F900895809120
:10E8E0009B088630D8F496E0899FF0011124E958FE
:10E8F000F74F2091AB023091AC02318320834091DD
:10E90000581B5091591B60915A1B70915B1B42839D
:10E910005383648375838F5F80939B080895209150
:10E92000AB023091AC0228173907D9F09093AC02B2
:10E930008093AB024093581B5093591B60935A1B12
:10E9400070935B1B8A50964721F41092111210921B
:10E950009B0882E08093350281E08093FA0F109249
:10E960001812089540E050E0BA018AE096E7D7CF48
:10E97000E0919B08EE2381F0E150E0939B0886E054
:10E98000E89FF0011124E958F74F428153816481D7
:10E99000758180819181C3CFE5CFCF93DF93809143
:10E9A0003502882349F0609113027091140220E02F
:10E9B00041E081E00E9408F180917608811118C041
:10E9C00081E080937608C091AB02D091AC0240E028
:10E9D00050E0BA018DEC94E7A2DF0E94717F1092A3
:10E9E000760840E050E0BA01CE01DF91CF9197CF99
:10E9F000DF91CF910895CF92DF92EF92FF920F9324
:10EA00001F93CF93DF939C017B0180E090E0F9019D
:10EA1000E80FF91FE491EE2311F00196F8CFF7010A
:10EA2000AF014E195F0961916111FACF04E110E065
:10EA3000041B11099927081719071CF0DD24D3942A
:10EA400002C082E0D82E8091C41290E06D2D70E05B
:10EA50006F5F7F4F0F94022DC62EC6E0C60F8091C8
:10EA6000F712C81748F04091F91250E08C2F90E04F
:10EA70000B97481759078CF5D0E0E114F104B1F178
:10EA80008AE30E9404E982E0D8120FC0CC0D809185
:10EA9000F712C81758F12091F91230E08C2F90E04E
:10EAA0000B97281739071CF421C0DD23F9F0802FBC
:10EAB000880F080F000F0093FA12C093FB1280E238
:10EAC0000E9404E9C701DF91CF911F910F91FF9040
:10EAD000EF90DF90CF900C94CEC61092FA12C093B4
:10EAE000FB12C9010E94C1C6D1E0C7CFDF91CF910F
:10EAF0001F910F91FF90EF90DF90CF9008959CE0D1
:10EB0000899F802D112491E0980F909361192CE03A
:10EB1000280F209362194091F71250E030E02E5FE9
:10EB20003F4F24173507CCF0292F30E04091F912E0
:10EB300050E0241735078CF4662341F08E5F0E9465
:10EB4000F3F0809162198E5F0E94F3F08091621958
:10EB50001092FA128093FB1208950895FF920F937A
:10EB60001F93CF93DF931F92CDB7DEB783E690E07C
:10EB70000F94922980932612813011F48093AD086E
:10EB80008091FC12811105C081E08093FC120E94EB
:10EB90006AE96091C5127091C61219829E012F5FB9
:10EBA0003F4F4FE083EC92E10E9406F8809105020E
:10EBB000882349F1109205028091C31290E0805899
:10EBC000910997FD019695958795182F0E94D1E997
:10EBD00034E0F32E00E420E840E0612F83EC92E182
:10EBE0000E9422F8882339F021EB32E140E460E012
:10EBF000812F0E9403EA0E942EB3F09212120E940B
:10EC0000CAE88111E7CF0F90DF91CF911F910F914B
:10EC1000FF9008952F923F924F925F927F928F9232
:10EC20009F92AF92BF92CF92DF92EF92FF920F939B
:10EC30001F93CF93DF93CDB7DEB72A970FB6F89423
:10EC4000DEBF0FBECDBF109217128091191288231C
:10EC500041F084DF40E050E0BA0183E898EB5FDEEA
:10EC60002DC54091581B5091591B60915A1B7091B2
:10EC70005B1B20911B0230911C02C901840F951F60
:10EC80002436310524F4853691053CF416C024362B
:10EC9000310531F08436910584F484E690E00DC0AE
:10ECA000473051056105710514F0069706C04A3FCB
:10ECB0005F4F6F4F7F4F6CF4069690931C028093CA
:10ECC0001B021092581B1092591B10925A1B109243
:10ECD0005B1B80911B0290911C028A3091053CF0D5
:10ECE000883E23E092072CF087EE93E002C08AE092
:10ECF00090E090931C0280931B020E947AB7182F19
:10ED00000E942EB381E0809312128091F712853118
:10ED100008F5112359F080916D1B90916E1B892B82
:10ED200029F0BAE0EB2EB8E1FB2E04C0AAEDEA2EE2
:10ED3000A6E1FA2E03E120E841E060E083EC92E1F5
:10ED40000E9422F8882331F0970143E161E080E0DE
:10ED50000E9403EA8091F7128D3108F07DC188305E
:10ED600008F041C0809175081123D9F160912F10EE
:10ED700070913010072E000C880B990B0F94812393
:10ED800020E030E040E05FE30F94152A0F94592B08
:10ED90009B01643671051CF52A303105F4F04CE016
:10EDA00022E130E0241B310937FF02C02F5F3F4FC3
:10EDB000359527953195219531092A5D2093FA12D1
:10EDC00027E02093FB12CB010E9463FB0E94CEC67A
:10EDD00087ED96E10E94C1C606C046E0E1CF42E160
:10EDE000DFCF882319F28091F7128D31D0F5809111
:10EDF000F9128531B0F120E030E040E05FE360914E
:10EE000021127091221280912312909124120F945A
:10EE1000152A0F94592B9B01643671050CF023C3FE
:10EE20002A3031050CF41DC34CE022E130E0241BF4
:10EE3000310937FF02C02F5F3F4F35952795319538
:10EE4000219531092A5D2093FA122CE12093FB12BF
:10EE5000CB010E9463FB0E94CEC687ED96E10E9423
:10EE6000C1C68091F712853108F58091F912813180
:10EE7000E8F060912F1070913010072E000C880B75
:10EE8000990B0F94812320912112309122124091ED
:10EE90002312509124120F943B2C18160CF4E5C247
:10EEA00022E042E061E18EE20F94E80F8091F712D8
:10EEB000883008F03FC080917408111102C08111A0
:10EEC00039C060916B1B70916C1B072E000C880B76
:10EED000990B0F94812320E030E040E05FE30F9432
:10EEE000152A0F94592B643671052CF46A3071057C
:10EEF00024F446E003C042E101C04CE022E130E0EE
:10EF0000241B310937FF02C02F5F3F4F35952795EE
:10EF1000319521953109285B2093FA1227E020933F
:10EF2000FB12CB010E9463FB0E94CEC687ED96E1E7
:10EF30000E94C1C68091F7128D31D0F58091F912EF
:10EF40008531B0F120E030E040E05FE3609170088F
:10EF50007091710880917208909173080F94152A2E
:10EF60000F94592B9B01643671050CF08CC22A302A
:10EF700031050CF086C246E022E130E0241B310965
:10EF800037FF02C02F5F3F4F35952795319521956B
:10EF90003109285B2093FA122CE12093FB12CB015C
:10EFA0000E9463FB0E94CEC687ED96E10E94C1C617
:10EFB0008091F712853130F58091F912813110F18D
:10EFC00060916B1B70916C1B072E000C880B990BCA
:10EFD0000F9481232091700830917108409172083C
:10EFE000509173080F943B2C18160CF04EC21092DF
:10EFF000E31222E042E062E18FE40F94E80F81E047
:10F000008093E3128091F7128C3130F58091F912E0
:10F01000843110F180916D1B90916E1B019644E636
:10F02000489F9001499F300D112437FF02C02150A5
:10F030003F4F832F932F990F990B009769F028E684
:10F040002093FA122BE12093FB120E9463FB0E9493
:10F05000CEC685E20E9404E94091AD08642F70E0BD
:10F060002091F71230E083E390E0861B970B821724
:10F0700093075CF02091F91230E08AE290E0861B61
:10F08000970B281739070CF007C24091AD08209163
:10F09000F71230E084E390E0841B91098217930714
:10F0A0002CF08091F912813308F024C28091C113B1
:10F0B000882309F453C04091AD082091F71230E045
:10F0C00083E390E0841B9109821793070CF446C0F8
:10F0D0008091F912823308F441C002E0041B2091B0
:10F0E0008F15222319F18091581690915916A091ED
:10F0F0005A16B0915B160097A105B10509F402C23A
:10F10000BC01CD016D597F4F8F4F9F4F24E630E0FA
:10F1100040E050E00F94B72960915C1670915D1645
:10F1200080915E1690915F160F94B72985E3289F12
:10F13000B0011124072E000C880B990B0F9481232A
:10F140002AE037ED43E25CE30F94E0230F945E2B5B
:10F15000462F202F62E387E30F94E80F8091F71288
:10F16000813308F079C08091F912893208F474C0B3
:10F170000E94528A4B015C0120E13EE040E050E0F9
:10F180000F94B729722E032FE22EF32E8CE3282E34
:10F19000312C412C512CC501B401A20191010F94D5
:10F1A000B729CA01B901A20191010F94B729CE0173
:10F1B00001966C0191E8891691E5990691E0A906FE
:10F1C000B10408F4A1C17F936F93C70168E170E0B7
:10F1D0000F94EE2C9F938F93C501B40120E831E585
:10F1E00041E050E00F94B7293F932F9383EC96E1D1
:10F1F0009F938F93DF92CF920F9415230FB6F894BD
:10F20000DEBF0FBECDBF8CE38093FA1280E3809304
:10F21000FB12C6010E94CEC680912A1090912B103D
:10F22000A0912C10B0912D10892B8A2B8B2B09F4D7
:10F23000ADC120918F15211184C188E68093FA1207
:10F2400083E38093FB12822F90E00E9463FB0F9474
:10F25000D60F85E20E9404E9E091BD12F091BE1242
:10F2600084818111CCC060914119709142198091C3
:10F270004319909144190F94592BCB010E94E2FA43
:10F28000BC0188EA98E00F947E2D60914519709139
:10F29000461980914719909148190F94592BCB0129
:10F2A0000E94E2FABC0183EA98E00F947E2D2CEADA
:10F2B00035EC47E257E36091491970914A19809102
:10F2C0004B1990914C190F94152A20E030E048EC2E
:10F2D00052E40F94E0230F94592B6B017C0197FDAE
:10F2E00019C090E1C91697E2D906E104F104E4F0EF
:10F2F000C701B60120E137E240E050E00F94D92980
:10F30000CA01B9012AE030E040E050E00F94D92969
:10F31000605D0BC0F094E094D094C094C11CD11CEB
:10F32000E11CF11C6DE201C060E26093701B28EEED
:10F33000C21623E0D206E104F10494F0C701B6013D
:10F3400028EE33E040E050E00F94D929CA01B9011A
:10F350002AE030E040E050E00F94D929605D01C020
:10F3600060E26093711BC701B60124E630E040E023
:10F3700050E00F94D9299AE0892E912CA12CB12C20
:10F38000CA01B901A50194010F94D929605D609368
:10F39000721BC701B601A50194010F94D929062F4C
:10F3A000662381F08EE28093731BCA01B901A50127
:10F3B00094010F94D929605D6093741B005D0093E4
:10F3C000751B17C0CA01B901A50194010F94D92971
:10F3D000662339F08EE28093731B605D6093741B2B
:10F3E00005C080E28093741B8093731B80E280933E
:10F3F000751B60E77BE18CE998E00F947E2D80918E
:10F40000F712883298F48091F9128D3178F02BE060
:10F4100040E86DE180E00F94A00F8091F7128732F1
:10F4200028F48091F9128F3108F0B9C08091F71259
:10F43000823328F48091F9128B3208F01BC180913D
:10F44000F712803408F03AC18091F912883308F439
:10F4500035C11092FA128FE38093FB120E9456E995
:10F460002DC146E0E2CC42E1E0CC1092E31222E072
:10F4700042E061E18EE20F94E80F81E08093E312B5
:10F4800015CD4CE079CD42E177CD22E042E062E15A
:10F490008FE40F94E80FB6CD6AE2641B27E048E0E2
:10F4A0008AE20F94E80F8091AD086CE2681B25E0BA
:10F4B00042E082E30F94E80F8091AD0861E3681B9E
:10F4C00024E04AE08AE20F94A00F9091AD088BE20D
:10F4D000891B6091C5127091C61292E39093DF125E
:10F4E0008093E0122FED32E142E383EC92E10E943F
:10F4F00006F8CBCD24E0241B45E361E386E30F94BB
:10F50000A00FD4CD20E012CE94E6E916F10460F409
:10F510007F936F93C70168E170E00F94EE2C9F9387
:10F520008F9389EB96E106C07F936F930F937F9241
:10F5300081EB96E19F938F93DF92CF920F941523E7
:10F540005DCE8091581690915916A0915A16B0919F
:10F550005B160097A105B105B9F0BC01CD016D594D
:10F560007F4F8F4F9F4F24E630E040E050E00F94F4
:10F57000B72960915C1670915D1680915E1690912E
:10F580005F160F94B72959CE20E057CE88E68093B6
:10F59000FA1283E38093FB1280E090E056CE83E082
:10F5A0008093FA1286E28093FB12112329F085EDF5
:10F5B00096E10E94C1C60DC080916D08811102C004
:10F5C0008FE305C0809116108111F1CF80E20E9477
:10F5D00004E98BE08093FA1206E20093FB1288EABA
:10F5E00098E00E94CEC68BE28093FA120093FB1241
:10F5F000112329F083ED96E10E94C1C60DC08091D0
:10F600006E08811102C08FE305C08091171081112F
:10F61000F1CF80E20E9404E983E38093FA1206E2CC
:10F620000093FB1283EA98E00E94CEC683E58093A4
:10F63000FA120093FB12112329F081ED96E10E944A
:10F64000C1C60DC080916F08811102C08FE305C053
:10F65000809118108111F1CF80E20E9404E98BE5BE
:10F660008093FA1286E28093FB128CE998E00E9464
:10F67000CEC6DCCE0E942EB384E08093121283E0CB
:10F680008093FA1212E31093FB1286E00E94ADC63B
:10F690000E942EB381E0809312128CE08093FA12C4
:10F6A0001093FB1280911B0290911C020E9463FB3D
:10F6B0000E94CEC685E20E9404E9C1CE2A960FB60A
:10F6C000F894DEBF0FBECDBFDF91CF911F910F9198
:10F6D000FF90EF90DF90CF90BF90AF909F908F9072
:10F6E0007F905F904F903F902F900895DF92EF9220
:10F6F000FF920F931F93CF93DF93F82ED62EE72E12
:10F700008A0180910B02882309F439C0E0EEF2E20D
:10F710008491EF012196882321F00E94F245FE0199
:10F72000F7CFED2DFE2D8491EF012196882321F056
:10F730000E94F245FE01F7CFEBE4F1E28491EF0184
:10F740002196882321F00E94F245FE01F7CFF7FCB5
:10F750000BC06F2DFF0C770B880B990B0E945B473A
:10F760008AE00E94F2450BC0E6E4F1E28491EF01E9
:10F770002196882321F00E94F245FE01F7CF809167
:10F78000C50D811108C010920B0281E08093C50D58
:10F79000C8010E941167DF91CF911F910F91FF90D7
:10F7A000EF90DF900C94A7C24F925F926F927F927E
:10F7B0008F929F92AF92BF92CF92DF92EF92FF9281
:10F7C0000F931F93CF93DF93CDB7DEB72C970FB670
:10F7D000F894DEBF0FBECDBF80915B12811117C0C0
:10F7E0002C960FB6F894DEBF0FBECDBFDF91CF9140
:10F7F0001F910F91FF90EF90DF90CF90BF90AF904F
:10F800009F908F907F906F905F904F9008950E948F
:10F81000B0C30E947EF72B013C01809175088111D5
:10F8200017C080919B0D90919C0DA0919D0DB09162
:10F830009E0D0097A105B10559F0A3019201281B67
:10F84000390B4A0B5B0B57FD03C081E080937508B1
:10F8500060912F1070913010072E000C880B990BBF
:10F860000F94812320912112309122124091231272
:10F870005091241214E0812E912C0CE3A02EB12C77
:10F88000C12CD12C7B018C0167EE7DE085EE9DE0E3
:10F890000E943BC18090211290902212A0902312CE
:10F8A000B09024126091131070911410072E000C68
:10F8B000880B990B0F9481239B01AC01C501B40106
:10F8C0000F943B2C18160CF008C160911002709137
:10F8D0001102072E000C880B990B0F9481239B01BA
:10F8E000AC01C501B4010F947B2387FFF6C04091A2
:10F8F0002F10509130105A83498320ED3CEC4CE49A
:10F900005DE36091970D7091980D8091990D9091A4
:10F910009A0D0F94E0236B017C012091DB0D309157
:10F92000DC0D4091DD0D5091DE0DC501B4010F9449
:10F93000142A9B01AC01C701B6010F94E0236B01AF
:10F940007C0123E333E343E75FE36091D70D7091DC
:10F95000D80D8091D90D9091DA0D0F94E0239B0181
:10F96000AC01C701B6010F94152A6B017C016093AD
:10F97000D70D7093D80D8093D90D9093DA0D8092A6
:10F98000DB0D9092DC0DA092DD0DB092DE0D80912A
:10F990007508811115C2A981BA81BD01BB0F880B01
:10F9A000990B0F948123A50194010F94142A4B0104
:10F9B0005C0120E030E040E251E40F943B2C18164B
:10F9C0000CF40FC220E030E040E251ECC501B4017C
:10F9D0000F947B2387FDF4C129813A81232B09F4FD
:10F9E000EFC18091D60D81111BC28091D20D9091F3
:10F9F000D30DA091D40DB091D50D89839A83AB839B
:10FA0000BC832091930D3091940D4091950D5091B0
:10FA1000960DC501B4010F94E0236D837E838F831F
:10FA20009887A501940169817A818B819C810F94CB
:10FA3000152A69837A838B839C836093D20D70939C
:10FA4000D30D8093D40D9093D50D20918F0D3091CF
:10FA5000900D4091910D5091920D0F94E0232D81C6
:10FA60003E814F8158850F94152AA70196010F9466
:10FA7000142A6B017C0120E030E04FE753E40F943F
:10FA80003B2C20E030E0A90118160CF4D0C1C701CE
:10FA9000B6010F947B2387FD07C0C701B6010F9401
:10FAA000592B759567951AC020E030E0A901C50172
:10FAB000B4010F947B2387FF10C0A50194016981D5
:10FAC0007A818B819C810F94142A6093D20D70935C
:10FAD000D30D8093D40D9093D50D60E060935D12AB
:10FAE00080914E1290914F12A0915012B0915112EC
:10FAF0000097A105B10509F1A3019201281B390B5B
:10FB00004A0B5B0B57FD19C0609152127091531252
:10FB100080E090E00F947F239B01AC016091211263
:10FB20007091221280912312909124120F947B23C2
:10FB300087FD3FC180E00E94CAC28091541290911B
:10FB40005512A0915612B09157120097A105B10518
:10FB500011F1481A590A6A0A7B0A77FC1CC06091A5
:10FB600058127091591280E090E00F947F239B010E
:10FB7000AC01609170087091710880917208909149
:10FB800073080F947B2387FF11C149E651E268E7B0
:10FB900071E28FEFABDD60916B1B70916C1B072ED8
:10FBA000000C880B990B0F948123209170083091E1
:10FBB00071084091720850917308E2E08E2E912CEA
:10FBC000F8E7AF2EB12CCC24CA94DC2C7B018C013D
:10FBD0006FED7DE083EE9DE00E943BC18091740853
:10FBE0008111E1C0C0907008D0907108E090720857
:10FBF000F090730820E030E040EA50E4C701B6011D
:10FC00000F943B2C87FF04C060E060935C12E8CD4A
:10FC100020E030E04AEF52E4C701B6010F947B23A5
:10FC2000181694F360916B1B70916C1B072E000CDF
:10FC3000880B990B0F948123A70196010F94142A26
:10FC40004B015C0120918B0D30918C0D40918D0DFD
:10FC500050918E0D0F94E0236D837E838F83988760
:10FC60002091CE0D3091CF0D4091D00D5091D10DFE
:10FC7000C501B4010F94152A69837A838B839C8311
:10FC80006093CE0D7093CF0D8093D00D9093D10DD6
:10FC90002091870D3091880D4091890D50918A0DEA
:10FCA0000F94E02369877A878B879C8720ED3CEC53
:10FCB0004CE45DE36091830D7091840D8091850D1E
:10FCC0009091860D0F94E0232B013C012091CA0DE9
:10FCD0003091CB0D4091CC0D5091CD0DC701B601A7
:10FCE0000F94142A9B01AC01C301B2010F94E023CD
:10FCF0002B013C0123E333E343E75FE36091C60D4F
:10FD00007091C70D8091C80D9091C90D0F94E0239B
:10FD10009B01AC01C301B2010F94152A2B013C01D8
:10FD20006093C60D7093C70D8093C80D9093C90D55
:10FD3000C092CA0DD092CB0DE092CC0DF092CD0DB9
:10FD400029853A854B855C856D817E818F8198857B
:10FD50000F94152AA30192010F94142A6B017C01C0
:10FD600020E030E04FE753E40F943B2C20E030E0FC
:10FD7000A90118164CF5C501B4010F943B2C1816B7
:10FD800084F4A501940169817A818B819C810F940F
:10FD9000142A6093CE0D7093CF0D8093D00D909365
:10FDA000D10D6FE732CF10925C121ACD0E945BC268
:10FDB000F2CE47E851E266E971E280E097DCBDCE21
:10FDC00081E08093D60D89CEC701B6010F947B23C5
:10FDD00087FD0CC0C701B6010F94592B7595679527
:10FDE00014CF81E08093D60D6FE778CE20E030E02D
:10FDF000A901C501B4010F947B2387FF05CFA5019D
:10FE0000940169817A818B819C810F94142A60937B
:10FE1000CE0D7093CF0D8093D00D9093D10DF4CE75
:10FE20001092D60D19821A821B821C82EACDC5015E
:10FE3000B4010F943B2C1816BCF6A50194016981FE
:10FE40007A818B819C810F94142A6093D20D7093D8
:10FE5000D30D8093D40D9093D50D6FE73FCE880FCF
:10FE6000991F880F991FFC01EF5CF64E408151816C
:10FE700062817381FC01EF5BFF4E4083518362839B
:10FE80007383E091810DF091820D82899389A48919
:10FE9000B5898093C10D9093C20DA093C30DB0930B
:10FEA000C40D0895CF93DF932FB7F894AC01440F9E
:10FEB000551F440F551FFA01EF5CF64E60817181AA
:10FEC000828193812FBFEA01CF5CDF4E0F948123A3
:10FED000288139814A815B810F94E023DF91CF91A2
:10FEE00008959091211380912213981721F080E0BA
:10FEF0000E947C67F6CF08951F920F920FB60F9263
:10FF000011240BB60F92BF92CF92DF92EF92FF9225
:10FF10000F931F932F933F934F935F936F937F9311
:10FF20008F939F93AF93BF93EF93FF93CF93DF9301
:10FF300000D000D0CDB7DEB780916E008B7F80936C
:10FF40006E0080916F008D7F80936F007894C090D9
:10FF5000BD0DD090BE0DE090BF0DF090C00DC1144E
:10FF6000D104E104F10409F442C08091151081111B
:10FF700004C0809119108823D1F10E94EE6BF9EB37
:10FF8000CF16FBE0DF06E104F10488F008EBC01AAD
:10FF90000BE0D00AE108F108C092BD0DD092BE0D71
:10FFA000E092BF0DF092C00D88EB9BE009C0C60146
:10FFB0001092BD0D1092BE0D1092BF0D1092C00D8B
:10FFC0009093890080938800209188003091890067
:10FFD000809184009091850040962817390708F099
:10FFE00074C08091840090918500409623C0009158
:10FFF0007F0D1091800D1A830983012B09F49AC09B
:020000021000EC
:1000000009811A81015011091093800D00937F0D11
:100010001092820D1092810D0F948C0B012B41F4E4
:100020008AE391E29093F70F8093F60F0E945B446E
:1000300088EC90E0909389008093880046C0898185
:100040009A810E94A5E824E630E08091151088236B
:1000500009F403C5C901293BBBE03B0708F03BC6D7
:1000600090938900809388008091AF0D9091B00D9E
:10007000A091B10DB091B20D820F931FA11DB11DC2
:100080008093AF0D9093B00DA093B10DB093B20DCE
:1000900020918800309189008091840090918500A2
:1000A00040962817390748F4809184009091850084
:1000B00040969093890080938800BB2031F0109285
:1000C000820D1092810D0F948C0BF89480915E122A
:1000D000882321F080916E008B7F03C080916E0099
:1000E000846080936E0080916F00826080936F00C7
:1000F00026960FB6F894DEBF0FBECDBFDF91CF912D
:10010000FF91EF91BF91AF919F918F917F916F91EF
:100110005F914F913F912F911F910F91FF90EF9021
:10012000DF90CF90BF900F900BBE0F900FBE0F903F
:100130001F9018950091810D1091820D01151105E8
:1001400009F0E4C19091211380912213981761F175
:10015000009122132DE4029F80011124F801E25541
:10016000F74FC0900D12D0900E12E0900F12F09049
:100170001012CF01875B9F4FDC014D915D916D9116
:100180007C91D701C601841B950BA60BB70B8093FE
:100190000D1290930E12A0930F12B0931012808143
:1001A000886080838F010BC08FB7F89410920D1276
:1001B00010920E1210920F12109210128FBF109305
:1001C000820D0093810D0115110509F49CC1F80100
:1001D00052A180917E0D418158130AC0242F30E036
:1001E00080910A02082E000C990B2817390731F06C
:1001F00050937E0D40930A020F94520B1092B90D4A
:100200001092BA0D1092BB0D1092BC0DD801D7966A
:100210000D90BC91A02DBA83A983A134ECE9BE074F
:1002200020F4A132BE4478F004C020E43CE93A83D3
:10023000298349815A8156954795569547955A8302
:10024000498384E00BC089819A818131A7E29A07B2
:1002500040F0969587959A83898382E08093B80DC4
:100260000BC081E08093B80DE981FA81B09720F44A
:1002700020E230E03A83298349815A814052510972
:100280005A834983411568E05607F0F0E52FFF27B0
:10029000EE0FFF1FEE0FFF1FCF01865C924EFC0199
:1002A000329645915491B981AA27B59F9001B49F88
:1002B000210D3A1F06942A1F3A1F1124FC01859133
:1002C0009491821B930B22C089819A819695879580
:1002D0008C7F865C964EFC0125913491FC01329610
:1002E0004591549169817A8167707727649FC00135
:1002F000659F900D749F900D112453E096958795FE
:100300005A95E1F7F901E81BF90BCF018436910505
:1003100090F430E7E32E34E0F32ED7018D917D0188
:10032000882319F00E94F245F8CF89819A810E94B2
:10033000A5E884E690E09093B70D8093B60D809188
:10034000B80D8093B50DF80103ACF4ADE02DFA8340
:10035000E983F093B40DE093B30DE1342CE9F20797
:1003600020F4E132FE4478F004C040E45CE95A83B2
:10037000498389819A8196958795969587959A83E1
:10038000898384E00BC0A981BA81A131E7E2BE076D
:1003900040F0B695A795BA83A98382E08093B80D03
:1003A0000CC081E08093B80D29813A81203231055B
:1003B00020F440E250E05A83498389819A818097F2
:1003C0009A8389838115A8E09A07F0F0E92FFF2727
:1003D000EE0FFF1FEE0FFF1FCF01865C924EFC0158
:1003E000329645915491B981AA27B59F9001B49F47
:1003F000210D3A1F06942A1F3A1F1124FC018591F2
:100400009491821B930B22C089819A81969587953E
:100410008C7F865C964EFC0125913491FC013296CE
:100420004591549169817A8167707727649FC001F3
:10043000659F900D749F900D112473E0969587959C
:100440007A95E1F7F901E81BF90BCF0184369105A4
:1004500090F450E7E52E54E0F52ED7018D917D0103
:10046000882319F00E94F245F8CF89819A810E9471
:10047000A5E884E690E0AC0160E070E04093AF0D49
:100480005093B00D6093B10D7093B20D90938900AD
:1004900080938800F80182899389A489B589B695EB
:1004A000A79597958795B095A095909581959F4F25
:1004B000AF4FBF4F8093AB0D9093AC0DA093AD0D9C
:1004C000B093AE0D8093A70D9093A80DA093A90DA6
:1004D000B093AA0D8093A30D9093A40DA093A50DA6
:1004E000B093A60D80939F0D9093A00DA093A10DA6
:1004F000B093A20D1092C10D1092C20D1092C30DB7
:100500001092C40D03C080ED97E094CD809115103A
:100510008111DEC3809119108111DAC32091B80DC9
:10052000222309F4AFC1E091810DF091820D428147
:1005300053816481758180919F0D9091A00DA09150
:10054000A10DB091A20D840F951FA61FB71F809318
:100550009F0D9093A00DA093A10DB093A20D18161E
:1005600019061A061B060CF4889AE091810DF09189
:10057000820D46815781608571858091A30D909190
:10058000A40DA091A50DB091A60D840F951FA61FD7
:10059000B71F8093A30D9093A40DA093A50DB093C6
:1005A000A60D181619061A061B060CF48E9AE09171
:1005B000810DF091820D428553856485758580910A
:1005C000A70D9091A80DA091A90DB091AA0D840F2F
:1005D000951FA61FB71F8093A70D9093A80DA093FA
:1005E000A90DB093AA0D181619061A061B0644F495
:1005F0009FB7F89480910B01886080930B019FBF97
:10060000E091810DF091820D468557856089718951
:100610008091AB0D9091AC0DA091AD0DB091AE0D50
:10062000840F951FA61FB71F8093AB0D9093AC0D41
:10063000A093AD0DB093AE0D181619061A061B0641
:100640000CF4149A80919F0D9091A00DA091A10D92
:10065000B091A20D181619061A061B0684F5E09132
:10066000810DF091820D4289538964897589841BBB
:10067000950BA60BB70B80939F0D9093A00DA093A5
:10068000A10DB093A20D80910602409131195091B5
:1006900032196091331970913419082E000C990B9E
:1006A000AA0BBB0B840F951FA61FB71F8093311990
:1006B00090933219A0933319B0933419889880918C
:1006C000A30D9091A40DA091A50DB091A60D1816A3
:1006D00019061A061B0684F5E091810DF091820D32
:1006E0004289538964897589841B950BA60BB70BC6
:1006F0008093A30D9093A40DA093A50DB093A60D88
:10070000809107024091351950913619609137193F
:1007100070913819082E000C990BAA0BBB0B840F93
:10072000951FA61FB71F8093351990933619A09374
:100730003719B09338198E988091A70D9091A80D14
:10074000A091A90DB091AA0D181619061A061B063C
:10075000BCF5E091810DF091820D42895389648945
:100760007589841B950BA60BB70B8093A70D9093EF
:10077000A80DA093A90DB093AA0D809108024091F5
:10078000391950913A1960913B1970913C19082E12
:10079000000C990BAA0BBB0B840F951FA61FB71F4C
:1007A0008093391990933A19A0933B19B0933C194F
:1007B0009FB7F89480910B01877F80930B019FBFB7
:1007C0008091AB0D9091AC0DA091AD0DB091AE0D9F
:1007D000181619061A061B0684F5E091810DF09192
:1007E000820D4289538964897589841B950BA60BF8
:1007F000B70B8093AB0D9093AC0DA093AD0DB09360
:10080000AE0D8091090240913D1950913E196091C1
:100810003F1970914019082E000C990BAA0BBB0BC5
:10082000840F951FA61FB71F80933D1990933E1903
:10083000A0933F19B093401914988091C10D9091E5
:10084000C20DA091C30DB091C40D0196A11DB11DA3
:100850008093C10D9093C20DA093C30DB093C40DAE
:100860002150E091810DF091820D42895389648974
:10087000758984179507A607B70708F451CEBB24DE
:10088000B39401C0B12CE091810DF091820D809163
:10089000C10D9091C20DA091C30DB091C40D4689B8
:1008A0005789608D718D481759076A077B0708F4CF
:1008B000DAC04091AF0D5091B00D6091B10D7091C3
:1008C000B20D068D178D20A131A1AA27419FB12D10
:1008D000529FC001629F900D619F800D911D429FAC
:1008E000B00D811D9A1F519FB00D811D9A1F609FF1
:1008F000B00D811D9A1F509FB10D8A1F9A1FB6958A
:100900008A1F9A1F349F800D911D359F900D1124D1
:1009100023AD34AD820F931F9093B40D8093B30D2C
:1009200047A950AD61AD72ADA0E0B0E048175907DE
:100930006A077B0720F45093B40D4093B30D0091E8
:10094000B30D1091B40D1A83098301342CE91207F9
:1009500020F401321E4478F004C040E45CE95A837C
:10096000498389819A8196958795969587959A83EB
:10097000898384E00BC0A981BA81A131E7E2BE0777
:1009800040F0B695A795BA83A98382E08093B80D0D
:100990000CC081E08093B80D09811A8100321105E5
:1009A00020F420E230E03A83298309811A81005241
:1009B00011091A830983011528E01207E8F0E12FD5
:1009C000FF27EE0FFF1FEE0FFF1FCF01865C924E39
:1009D000FC01329625913491AA27039FA001029F22
:1009E000410D5A1F06944A1F5A1F1124FC012591DC
:1009F0003491241B350B20C089819A819695879567
:100A00008C7F865C964EFC0125913491FC013296D8
:100A10004591549169817A8167707727649FC001FD
:100A2000659F900D749F900D1124B3E09695879566
:100A3000BA95E1F7281B390B2436310508F005CBB0
:100A4000F0E7EF2EF4E0FF2ED7018D917D01882392
:100A500009F4F5CA0E94F245F7CF8091191081116F
:100A6000F9CAC901FDCA8091C10D9091C20DA09132
:100A7000C30DB091C40D428D538D648D758D481793
:100A800059076A077B0708F0F0C00091B90D109173
:100A9000BA0D2091BB0D3091BC0D09831A832B83B5
:100AA0003C83468D578D60A171A1AA27059FB12D6A
:100AB000169F7001269FF00C259FE00CF11C069FED
:100AC000B00DE11CFA1E159FB00DE11CFA1E249F0B
:100AD000B00DE11CFA1E149FB10DEA1EFA1EB69568
:100AE000EA1EFA1E709FE00CF11C719FF00C11249D
:100AF0008091B30D9091B40DFF96E816F90680F43D
:100B00008E199F0940815181628173816C01E12CB2
:100B1000F12CC416D506E606F70620F4CA0102C079
:100B20008081918181341CE9910728F481322EE47F
:100B3000920748F002C080E49CE9969587959695C7
:100B4000879524E007C0813137E2930730F096950E
:100B5000879522E02093B80D08C021E02093B80DBE
:100B60008032910510F480E290E08C01005211096E
:100B70001E830D83011528E01207E8F0E12FFF27FF
:100B8000EE0FFF1FEE0FFF1FCF01865C924EFC01A0
:100B9000329625913491AA27039FA001029F410D0F
:100BA0005A1F06944A1F5A1F1124FC0125913491A3
:100BB000241B350B20C08D819E81969587958C7F57
:100BC000865C964EFC0125913491FC01329645914C
:100BD00054916D817E8167707727649FC001659F06
:100BE000900D749F900D112443E0969587954A953A
:100BF000E1F7281B390B2436310590F480E7E82E05
:100C000084E0F82ED7018D917D01882319F00E9490
:100C1000F245F8CF8D819E810E94A5E824E630E060
:100C200080911510811104C080911910882339F02A
:100C3000C901293BBBE03B0708F068C001C0C901FE
:100C4000909389008093880089819A81AB81BC81CF
:100C5000820F931FA11DB11D8093B90D9093BA0D02
:100C6000A093BB0DB093BC0D13CA2091B60D30916B
:100C7000B70D80911510811104C08091191088233F
:100C8000F1F0293BEBE03E07D0F0C90168EB7BE0D7
:100C90000F94EE2C883E53E0950708F052C088541C
:100CA000944FA901481B590B60E070E04093BD0DC3
:100CB0005093BE0D6093BF0D7093C00D9C01309397
:100CC0008900209388008091B50D8093B80DE0C90C
:100CD0000E94EE6B23CC68EB7BE00F94EE2C883EF9
:100CE00013E0910780F48854944FA901481B590BD5
:100CF00060E070E04093BD0D5093BE0D6093BF0D5A
:100D00007093C00DADC988EB9BE0EFCF68EB7BE043
:100D10000F94EE2C883E43E0940780F48854944F5F
:100D2000A901481B590B60E070E04093BD0D509342
:100D3000BE0D6093BF0D7093C00D82CF88EB9BE01A
:100D4000EFCF88EB9BE0ADCF8F929F92AF92BF9297
:100D5000CF92DF92EF92FF921F93CF93DF93C82F32
:100D600085E695E19093F50F8093F40F109281152D
:100D700082E090E0A0E0B0E080936A1590936B155C
:100D8000A0936C15B0936D151092F30F1092EF0FA6
:100D90001092F00F1092F10F1092F20F8FEF9FEF61
:100DA000DC018093EB0F9093EC0FA093ED0FB093C9
:100DB000EE0FCC2379F1C53008F0F8C040E060E0D8
:100DC00070E0CB010E94BBFC882309F4EFC020E156
:100DD000C29FC00111248552924FFC01E254FE4F84
:100DE00020812F7709F0E2C03C96408151816281D9
:100DF0007381443651056105710508F4D7C03497F5
:100E0000C080D180E280F380C114D104E104F104F8
:100E100021F4CCC0C12CD12C760140E0C701B60131
:100E20000E94BBFC182F882309F4C0C08091F60DE6
:100E30009091F70D8115924009F0B8C0A091FB0D7B
:100E4000AA2309F4B3C06091F90D7091FA0D6115F0
:100E5000710509F4ABC02091F80D222309F4A6C056
:100E6000A0937C1520936E1580E030E041E050E0C7
:100E7000C82FFA01082E02C0EE0FFF1F0A94E2F7F6
:100E80002E173F0739F08F5FC83091F789E08093C4
:100E900077158CC0809377152091010E3091020E4A
:100EA0002115310519F040E050E008C020910F0EE7
:100EB0003091100E4091110E5091120E20936F152B
:100EC0003093701540937115509372154601570178
:100ED000860E971EA11CB11C80927D1590927E15E6
:100EE000A0927F15B0928015E091FC0DF091FD0D60
:100EF000F0938315E0938215B0E00F94F529860EE8
:100F0000971EA81EB91E8092841590928515A092F6
:100F10008615B092871585E0EE0FFF1F8A95E1F7E1
:100F2000E150FE4FEF2FFF27E6958E0E9F1EA11C6E
:100F3000B11C8092781590927915A0927A15B09292
:100F40007B152091FE0D3091FF0D2115310521F00B
:100F5000A90160E070E008C040910B0E50910C0EAA
:100F600060910D0E70910E0ED701C6018819990976
:100F7000AA09BB09840F951FA61FB71F04C0B69509
:100F8000A79597958795CA95D2F7809373159093F7
:100F90007415A0937515B0937615853F2FE09207D1
:100FA000A105B10528F48CE08093811510E01AC0EA
:100FB000853F9F4FA105B10510F480E111C08091DC
:100FC000170E9091180EA091190EB0911A0E8093E1
:100FD000841590938515A0938615B093871580E2AC
:100FE00080938115812FDF91CF911F91FF90EF901A
:100FF000DF90CF90BF90AF909F908F900895CF9249
:10100000DF92EF92FF920F931F93CF93DF93CDB7B1
:10101000DEB7EDB6FEB6DC010D900020E9F79D01CC
:10102000281B390B2C5F3F4F4DB75EB7421B530B4C
:101030000FB6F8945EBF0FBE4DBF0DB71EB70F5F62
:101040001F4F9F938F9382E093E29F938F931F9301
:101050000F930F941523680154E0C50ED11C0F9017
:101060000F900F900F900F900F90F60180818823C2
:1010700049F0082E000C990B0F94272DF60181934F
:101080006F01F3CFC8010E9482EB8EEF92E2909342
:10109000F70F8093F60F0E945B440FB6F894FEBEE4
:1010A0000FBEEDBEDF91CF911F910F91FF90EF909A
:1010B000DF90CF900895AF92BF92CF92DF92EF92E0
:1010C000FF920F931F93CF93DF93CDB7DEB7AA970D
:1010D0000FB6F894DEBF0FBECDBF8091ED138F9396
:1010E0008091EC138F9385EF92E29F938F937E0113
:1010F00081E2E80EF11CFF92EF920F9415230F90FE
:101100000F900F900F900F900F9010E0F70101904B
:101110000020E9F73197EE19FF091E1784F46701E3
:10112000C10ED11C17FDDA94F6018081082E000C47
:10113000990B0F94272DF60180831F5FE7CF82EF75
:1011400093E10E94DBCF00E0CE0101966C0180911B
:10115000F513823080F08091FA139091FB13A091E7
:10116000FC13B091FD138F719927AA27BB27892BF8
:101170008A2B8B2BF9F0011103C08FEF9FEF05C075
:101180008091EC139091ED1301969093ED13809361
:10119000EC13AA960FB6F894DEBF0FBECDBFDF9159
:1011A000CF911F910F91FF90EF90DF90CF90BF9064
:1011B000AF90089540E050E0B60182EF93E10E94C5
:1011C0006BFE1816C4F6F60101900020E9F731977E
:1011D0001E2F1C19115068F05601A10EB11C17FDED
:1011E000BA94F501808190E00F94272DF50180835A
:1011F000F1CF8A858E3709F4AACF45E050E0B701D8
:10120000C6010F94852D892B09F0A1CFC701F7DE08
:1012100001E09DCFCF92DF92EF92FF921F93CF9389
:10122000DF931092C2138091F513882321F082EF8F
:1012300093E10E947ECE109269151092661585E3A7
:10124000809365150E947EF7EB01A89561E080917F
:1012500065150E9442F685E695E10E94E0CF23984D
:10126000229A219A209A289A85E08093671582E530
:101270008CBD1DBC1AE08FEF0E94E5CF1150D9F74D
:1012800020E030E0A90160E085E695E10E94EACF28
:10129000182F80936815813049F00E947EF76C1BEF
:1012A0007D0B613D774060F381E054C02AEA31E074
:1012B00040E050E068E085E695E10E94EACF82FFD9
:1012C00003C0109369150EC014E00E94A7628093BA
:1012D00068151150D1F78A3A11F082E03BC082E0E4
:1012E0008093691580916915823021F0C12CD12C31
:1012F000760105C0C12CD12CE12C80E4F82E20E031
:1013000030E0A90167E385E695E10E94EACFA701F5
:10131000960169E285E695E10E94EACF809368151F
:10132000882349F00E947EF76C1B7D0B613D77405E
:1013300030F38AE00FC080916915823011F520E00A
:1013400030E0A9016AE385E695E10E94EACF8823AF
:1013500051F088E08093661585E695E10E94E0CF24
:10136000EBEEFCE419C00E94A762807C803C19F47B
:1013700083E0809369150E94A7620E94A7620E9481
:10138000A76285E695E10E94E0CF1092671581E0A3
:10139000DBDC811131C015C08491EF0121968823D7
:1013A00021F00E94F245FE01F7CFE7EEF2E28491D0
:1013B000EF012196882309F456C00E94F245FE01F0
:1013C000F6CF80E0C1DC811117C0E0EEF2E284913B
:1013D000EF012196882321F00E94F245FE01F7CF0C
:1013E000ECECF2E28491EF012196882309F43BC0F2
:1013F0000E94F245FE01F6CF6AE675E182EF93E1C5
:101400000E942BCE811116C0E0EEF2E28491EF0132
:101410002196882321F00E94F245FE01F7CFEBEBE5
:10142000F2E28491EF0121968823E9F00E94F245CF
:10143000FE01F7CF81E08093C213EBEEFCE48491D0
:10144000EF012196882321F00E94F245FE01F7CF9B
:10145000EFEAF2E28491EF012196882321F00E94C5
:10146000F245FE01F7CF8BE1E2EFF3E1A3E1B4E156
:1014700001900D928A95E1F78091F0139091F1130C
:1014800090931214809311148EEE93E190930E14A6
:1014900080930D14DF91CF911F91FF90EF90DF901B
:1014A000CF9008950F931F938091B1139091B21331
:1014B000019719F40E947EF708C06091BB137091E8
:1014C000BC138091BD139091BE130091B71310917E
:1014D000B8132091B9133091BA13601B710B820BB2
:1014E000930B28EE33E040E050E00F94B729809151
:1014F000B3139091B413A091B513B091B613BC017E
:10150000CD01620F731F841F951F1F910F910895C6
:101510002F923F924F925F926F927F928F929F9203
:10152000AF92BF92CF92DF92EF92FF920F931F93F1
:10153000CF93DF93CDB7DEB7C057D1090FB6F8947C
:10154000DEBF0FBECDBF7C013B014A012DB73EB7C8
:10155000AF963FAF2EAFAF97AD961FAEAD972B01B5
:1015600034E0430E511C8E01015A1F4F80E490E07D
:101570008C0F9D1F0496E1969FAF8EAFE197F3010C
:101580008781823008F459C184859585A685B78501
:101590008F719927AA27BB27892B8A2B8B2B09F0C0
:1015A0004CC181ED93E1892B11F01092D11341EDE3
:1015B00053E1BE016F5F7F4FC2010E946BFE1816A0
:1015C0000CF03BC18C85982F9871903109F0AEC01A
:1015D000209165163091661621503109223031056F
:1015E00008F4A4C02DB63EB6BE016F5F7F4FC801A0
:1015F0000E945BFCF7018081882341F0F701019094
:101600000020E9F73197EE19FF0902C0E1E0F0E0B0
:10161000D8010D900020E9F7E01BF10BEA0FFB1F4A
:1016200031962DB73EB72E1B3F0B0FB6F8943EBF39
:101630000FBE2DBFEDB7FEB731965F01882311F0C5
:10164000B70102C064E874E0C5010F947E2DB801B3
:10165000C5010F945F2D64E874E0C5010F945F2D00
:10166000CE01805C9F4F0E9471FC21E0A801B20175
:10167000E1968EAD9FADE1970E9413D481112CC0ED
:101680008091651690916616892B31F5EBEEFCE49E
:1016900084916F012FEFC21AD20A882321F00E9491
:1016A000F245F601F5CFEBE9F2E284916F013FEFED
:1016B000C31AD30A882321F00E94F245F601F5CF20
:1016C0006801F60181916F01882319F00E94F245AB
:1016D000F8CF8AE00E94F2458BE1FE01EC5BFF4F00
:1016E000DE01959601900D928A95E1F724968EADD4
:1016F0009FAD24979CA38BA325EC32E03AA329A3AA
:1017000040E050E0BE016F5D7F4FC50101DFCE01BB
:1017100081960E943B64CE01805C9F4F0E943B6497
:101720000FB6F8943EBE0FBE2DBE29CF29812223CD
:1017300009F483C0253E09F422CF2E3209F41FCFCD
:101740002091D1132E3209F41ACF8A7009F017CFE5
:1017500081E0903109F080E08093C313903141F033
:101760008985873409F00BCF8A858E3709F407CF36
:1017700080916516909166168130910521F068F090
:101780000297A9F1FCCE8091671690916816019698
:101790009093681680936716F2CEBE016F5F7F4FFD
:1017A00084EC93E10E945BFC6701F60181916F017B
:1017B000882319F00E94F245F8CF84ECC82E83E10B
:1017C000D82EF60181916F01882319F00E94F2450D
:1017D000F8CF80E20E94F2456D8D7E8D8F8D98A1AD
:1017E0004AE00E94B4468AE00E94F245C8CEBE019B
:1017F0006F5F7F4F84EC93E10E945BFC8114910446
:1018000041F064EC73E1C4010F944C2D892B69F411
:1018100014C0AD96FFADAD978F2F90E02091671665
:10182000309168168217930741F0AD962FADAD97B2
:101830002F5FAD962FAFAD97A2CEAF962EAD3FAD39
:10184000AF970FB6F8943EBF0FBE2DBFC059DF4F04
:101850000FB6F894DEBF0FBECDBFDF91CF911F91C1
:101860000F91FF90EF90DF90CF90BF90AF909F903F
:101870008F907F906F905F904F903F902F90089542
:10188000EF92FF920F931F93CF93DF93CDB7DEB705
:101890006F970FB6F894DEBF0FBECDBF7B010DE092
:1018A00014E12FE034E1F8013183208322E030E0BD
:1018B000309366162093651690936816809367168A
:1018C00083E194E10E94DBCFF801808191812BE1DB
:1018D000FC013496DE01159601900D922A95E1F7F0
:1018E000FC01828193819C838B8385EC92E09A83B7
:1018F0008983A701BE016F5F7F4F84E294E008DE19
:10190000CE0101960E943B646F960FB6F894DEBF3D
:101910000FBECDBFDF91CF911F910F91FF90EF9040
:1019200008956F927F929F92AF92BF92CF92DF9273
:10193000EF92FF920F931F93CF93DF93CDB7DEB754
:10194000AC970FB6F894DEBF0FBECDBF2091C21387
:10195000222309F4C2C1962E7C0180918F15882321
:1019600009F474C0442309F48DC18091C6158823FD
:1019700029F1E0EEF2E284918F010F5F1F4F88237F
:1019800021F00E94F245F801F6CFE8E5F2E28491F9
:101990008F010F5F1F4F882321F00E94F245F8014D
:1019A000F6CF61E070E080E090E00E945B478AE063
:1019B0000E94F2458FE492E20E9411678BEC95E160
:1019C0000E9441EAEBEEFCE484918F010F5F1F4F10
:1019D000882321F00E94F245F801F6CFB70186E393
:1019E00092E20F94200D6091C6158DE8689FB001BA
:1019F000112465537A4E8BE292E20F94200D4091B0
:101A00005C1650915D1660915E1670915F1685E2CE
:101A100092E20F94CD0C8AE00E94F2458091C615A7
:101A200094E0899FF0011124E953FA4E40915C162D
:101A300050915D1660915E1670915F1640835183E0
:101A4000628373838F5F8093C6150DC01092C61595
:101A500082E0D82E19C1B70188E192E20F94200DDF
:101A60008AE00E94F2451092C11380918F1588235D
:101A700021F08CE895E10E947ECECE0101966C01AA
:101A80000E9471FC8EEE93E190930E1480930D14DE
:101A9000F70180818F3209F060C087010F5F1F4F0F
:101AA00009F461C06FE270E0C8010F946A2D5C0117
:101AB000009709F459C00817190708F055C03C01F0
:101AC000601A710AA301B801CE0180960F94932D7C
:101AD000E0E2F0E0EC0FFD1FE60DF71D1082CE01F5
:101AE00080963C018C01F80181918F01882319F0C7
:101AF0000E94F245F8CF8AE00E94F24560910D14F1
:101B000070910E146115710511F06C5F7F4F21E02B
:101B1000AE01405E5F4FCE0105960E9413D4811145
:101B200016C0E4E0F2E284918F010F5F1F4F88231B
:101B300021F00E94F245F801F6CFF30181913F01B7
:101B4000882319F00E94F245F8CF8EE285C0D0922A
:101B50000E14C0920D148501A1CF8FE094E19093F3
:101B60000E1480930D14870190910D1480910E1422
:101B7000692F782F992009F459C06115710511F06A
:101B80006C5F7F4F21E0A8018CE895E10E9413D49F
:101B9000882309F447C080919D1590919E15A091CE
:101BA0009F15B091A0158093581690935916A09345
:101BB0005A16B0935B16B80186EF91E20F94200D90
:101BC000409158165091591660915A1670915B16B3
:101BD0008EEE91E20F94CD0C8AE00E94F2451092B5
:101BE0005C1610925D1610925E1610925F16EFED65
:101BF000F1E284917F019FEFE91AF90A882321F02D
:101C00000E94F245F701F5CFB80180E090E038DEA0
